:020000040800F2
:10000000F0FF0010B19207085D000708A93202084E
:100010005193070851930708519307080000000007
:100020000000000000000000000000006100070860
:100030006500070800000000690007089DD6010858
:1000400051930708519307085193070851930708E4
:10005000519307085193070889B3000891B300082A
:1000600099B30008A1B30008A9B3000855B000086F
:1000700069B000087DB0000891B00008A5B0000884
:10008000B9B00008CDB00008519307085193070894
:10009000519307085193070851930708B1B300081B
:1000A00059CF0008B9CE000869CF0008A9CE0008D2
:1000B000E1CE0008F1CE000801CF000839A7000802
:1000C00075C2000841A7000879C2000851930708CB
:1000D00051930708D1CF0108D5D00108D9D1010823
:1000E000B9B30008519307085113070879CF0008E6
:1000F00031CF000889CF000821CF0008E1B0000807
:10010000519307085193070811CF0008519307082E
:10011000DDD20108E1D30108519307085193070884
:10012000F5B0000809B100081DB1000831B10008A0
:1001300045B10008519307085193070851930708E8
:100140005193070851930708519307086D0007085A
:1001500059B100086DB1000881B10008E5D401086B
:1001600049A700087DC2000851930708519307086A
:1001700051930708519307085193070851930708B3
:08018000519307085193070891
:10800000074BD0F8E4105B68D0F8F0205B1A9A4276
:10801000B8BFC0F8F030012380F81C310020704751
:10802000001000E0B74B00EB800270B503EBC20418
:1080300053F832205268B2F814C01CF0010F4FEA16
:1080400080016AD15FFA8CFE1EF0020F3DD0BFF3B3
:108050005F8F257F012D5FFA85FC00F0CC80148BAB
:10806000BFF35F8F0C1803EBC404257F022D00F0D3
:10807000E3800C1803EBC404257F032D06D1A47FF5
:1080800024B193F87940002C40F0E5809488A4B2A4
:1080900044F48064948093F978C001EB000E03EB04
:1080A000CE0E9EF81CE00EF1010EE6450CD1002428
:1080B00083F8794093F87A40002C40F0B680084469
:1080C00003EBC00300225A7670BD1EF0040F5BD193
:1080D0001EF0400E00F0C880158A93F978C0666AD9
:1080E000EDB206F80C505FFA8CFE267F0EF101040B
:1080F00064B2E51CAE4283F87840A44600F02A81C1
:108100000D1803EBC5052D7FAC42C6D10EF1020C54
:108110004FFA8CFC83F878C0BFE7B2F800C02CF4AB
:10812000006C4FEA0C4C4FEA1C4CA2F800C0B2F8AD
:1081300000C01FFA8CFC4CF4806CA2F800C0A57F34
:108140004FF0000C83F878C0002D46D093F879509A
:10815000002D3FD0012483F879400C1803EBC404B0
:10816000247F022C04D11488A4B244F40064148047
:108170000C1803EBC404A47E44F0010414820844E8
:1081800003EBC0031B7F70BDA57F4FF0010C83F88C
:108190007AC0002D6FD093F87950002D70D10C1853
:1081A00003EBC404647F002C00F0AE80148893F8C5
:1081B00078C0A4B244F400740CF1010C14804FFA9E
:1081C0008CF483F87840B2F800C01CF4807FFAD1B8
:1081D000A44662E7E47EFF2CBCD00C1803EBC40479
:1081E000A57E05F0FE051582E27EFF2AC7D0FF229C
:1081F00083F87820C3E7A47F002C3FF430AF93F8D6
:108200007940002C3FF42BAF148824F480642404BC
:10821000240C1480BFF35F8F148B148883F87AC00A
:10822000A4B244F40074148030E7948824F44074B9
:108230002404240C948042E7A47F002C3FF419AF5F
:1082400093F87940002C3FF414AF148824F4806430
:108250002404240C1480948824F480642404240CC2
:10826000948093F978C018E71FFA8CF52D0631D465
:1082700093F978C011E793F87940002C8FD095E7F7
:10828000257F022D15884AD925F480652D042D0CF3
:108290001580158A666A93F978C0EDB206F80C501D
:1082A000666A1488A4B244F4007414805FFA8CFCEB
:1082B000158A0CF1010464B2EDB2355595880CF1C4
:1082C000020CADB24FFA8CF445F4806583F8784027
:1082D000958078E793F978506E1C42D0266A765DD7
:1082E0001682247F05F1010C4FFA8CFC644583F85B
:1082F00078C07FF4D2AE948824F480642404240CE3
:108300009480CAE6F01E00201488A4B244F480745D
:108310001480012483F8794093F9784053E7ADB293
:1083200045F400751580158A666A93F978C0EDB238
:1083300006F80C505FFA8CFC666A158A0CF1010491
:1083400064B2EDB20CF1030C35554FFA8CF483F89E
:10835000784038E7958825F480652D042D0C9580AC
:10836000CEE6E57E1582A57F83F878E01DB9247FEF
:10837000002C7FF404AF948824F480642404240C3B
:108380009480FCE61B4B01681B4A03F5727C03E0FA
:1083900063452CD053F82C2F9142F9D170B593F846
:1083A00004E0427996450AD0634505D053F82C2F56
:1083B0009142F4D06345F9D14FF0FF3070BD9E4635
:1083C0008468DEF80C50A5424FF0000208D001325C
:1083D000032A0EF10C0EE7D0DEF80C50A542F6D1C0
:1083E000DEF81050C668B542F1D150B270BD4FF002
:1083F000FF30704714AE07080000014030B5EAB105
:108400008E464FEA014C034600F1C005002419686E
:108410009A6841EA0C0142EA0E029A60C3E900142C
:108420000C33AB42F3D1D0F8C030C0F8C44043EABB
:108430000E03C0F8C030C0F8C84030BD4FEA014E4E
:108440008C46E0E783691969B3F80CC00A6830B458
:108450009C6822F0010224680A60A28992B222EA92
:108460000C02A281027D04681F2A06D96568203AA1
:1084700008209040284245D0FEE72568082090401B
:108480002842F9D1202000FA02F2A260264A12788E
:10849000002A35D01A7E012A39D0D3F8F4200132CF
:1084A000C3F8F420EFF31181502282F31288586848
:1084B0005C6C026822EA04029C6C2243C9B202602E
:1084C00081F31188D3E90C401A6999681D6C096819
:1084D00014605061D3E90E40546090600024B3F8FA
:1084E000A800D5604C62C862106801242043106067
:1084F0001C7683F8F1408A899B8913439BB28B8158
:1085000030BC7047202000FA02F2E260BEE7002291
:1085100083F8F120D3F8F8000A68013022F0010254
:10852000C3F8F8000A60EBE70400001010B40C4C2C
:108530006368002B11DD002004F1080C0146DCF813
:10854000A03003F1C00259600C339342FBD1636841
:10855000013083420CF5807CF1DC5DF8044B704700
:1085600004000010F0B5494C04EB401C9CF8242496
:1085700002B9F0BD464B4FF08C0E0EFB003E93F857
:10858000DC6493F8DD249EF87E708CF80A749642C1
:108590004FF0000C4FEA40158EF87EC00ED002EB73
:1085A000420C03EBCC0C57009CF8E0C40CF1FF3EEE
:1085B000BEF1010F5CD9BCF1030F53D06019A0F8D4
:1085C0000814EFF31182902383F3128890F80A3491
:1085D000B0F8081443EA41030021D2B29BB280F8FC
:1085E0000A1482F311881A09217882EA13225A4068
:1085F000D9B1D0F82044D0F80C14D4F8A040D2431C
:108600001B019BB202F00F0201208840134304F1CA
:10861000C0015A0013F4004F93B202D162680243C2
:1086200062600C348C42F4D1F0BDD0F82014D0F844
:108630000C04D1F8A0401B0100F110019BB202F024
:108640000F0201208840134304F1C0015A0013F4C3
:10865000004F93B202D16268024362600C34A142BF
:10866000F4D1F0BD02F1010C0CF0030CB445A5D01F
:108670003A4403EBC202131893F8ED1400299DD07D
:108680006319012283F80A2498E700BF0400001050
:10869000F01E0020704700BF024B03EB401090F823
:1086A00025047047040000104368B0F8502010B44F
:1086B0001A83EFF31182502383F312884168446CCC
:1086C0000B6823EA0403C46C2343D2B20B6082F329
:1086D0001188D0E907418268036912681C605961FA
:1086E000D0E909415C60C46A9960B0F86010DC6050
:1086F0000023D1625DF8044B0376704710B4037D0C
:1087000001681F2B09D94C68203B202202FA03F391
:108710001C4215D15DF8044B70470C68202202FA08
:1087200003F31C42F6D00D4A4068002482F840450D
:1087300002685DF8044B22F0010202608B60704712
:10874000064A4068002482F8404502685DF8044B00
:1087500022F001020260CB60704700BFF01E0020D3
:10876000704700BF0B4890F83C1589B101EB4101FF
:10877000002310B4490000F244501C4650F8232056
:10878000063302B114608B42F8D15DF8044B704798
:10879000704700BF040000100B4890F83C1589B1E9
:1087A00001EB4101002310B4490000F244501C4683
:1087B00050F82320063302B114609942F8D15DF8D5
:1087C000044B7047704700BF040000100120704741
:1087D000034B00EB400003EBC00090F855057047D9
:1087E000040000101F4890F83C35002B39D00022BF
:1087F0002DE9F04300F244531B4E1C4D4FF0500E38
:108800004FF02C0C144607E053F8181B0C6090F83E
:108810003C150132914222DD197C0029F4D05F68B9
:10882000B90AA1F5801105EB010952294FF0FE08A4
:1088300098BF99F8F483EFF311898EF31288796A5F
:108840000CFB08680131C8F86C15B98A89B241F08F
:1088500001015FFA89F8B98288F31188D4E7BDE88D
:10886000F083704704000010F01E002014AE0708CB
:1088700007EE900AB8EE670A704700BFBCEEC00A68
:1088800010EE103A98B270470D4B0E49DB68DB438F
:10889000C3F30223C3F104030122DBB202FA03F3A0
:1088A00001EB000C1B0103F0F0038CF800334309CB
:1088B00000F01F0002FA00F041F82300704700BFEB
:1088C00000ED00E000E100E0037D1F2B08D9026805
:1088D000203B5168202202FA03F3194214D1704759
:1088E00001682022096802FA03F31942F7D00D4A01
:1088F00041684FF0000C82F8ACC70A68006822F0AB
:1089000001020A6083607047064A41684FF0000C1C
:1089100082F8ACC70A68006822F001020A60C360EE
:10892000704700BFF01E0020122301480B807047E3
:1089300088010020042301480B8070479C0100201F
:108940002048D0F8E837D0F8EC2730B59B184FF026
:108950001A040C8001D11C4830BD1B4AD0F8EA171C
:108960004FF0000E10467546B3F1204F4FEA137CCE
:108970000CF130040EF1020E2ABF0CF1370C84709A
:1089800080F802C0BEF1100FC5704FEA031300F16A
:108990000200E9D100200446B1F1204F4FEA1173E3
:1089A00003F1300C00F102002ABF373382F812C005
:1089B00093740828D4744FEA011102F10202EBD13A
:1089C000014830BD00F0FF1FA001002082B01F4B06
:1089D000002201920193019B1D4A04330193019BE4
:1089E0001968936803F00C03042B07D0082B0AD0F6
:1089F000184B194AC3F8B02702B07047154BC3F89B
:108A0000B01702B070475368506813F4800F00F03D
:108A10003F00536813D1C3F388130F49B1FBF0F142
:108A200001FB03F30A4A0B495268C2F301420132C7
:108A30005200B3FBF2F3C1F8B03702B07047C3F392
:108A40008813B1FBF0F101FB03F3EBE75028004082
:108A500000380240F01E00200024F4000123437778
:108A600000207047D0E90B2108B583690B4483616E
:108A70000AB108469047002008BD00BF436A1B6842
:108A80001B6A5B685B78024613F0010008BF5077F1
:108A9000704700BF70B5224A224C234B94B0054664
:108AA000CDE90042214A0992A4F108020A922A7FE4
:108AB0000493201D0023CDE905039A42CDE90E332E
:108AC0000B931093139314BF0520042011936B6A2A
:108AD0000C9002200122029018688DF80C200E469E
:108AE00007928DF820208DF834208DF848206EF004
:108AF0009FFD2B7F93B1330E04F8073C063C320CEC
:108B0000330A22706370A670686A694612F0BAFE72
:108B10006B6A18686EF08CFD14B070BD073CEEE710
:108B2000A4260020C40100207D8A00085D8A000878
:108B300010B5044694B050220649684672F0A2F877
:108B4000606A694612F09EFE636A18686EF070FDF6
:108B500014B010BD5CB20708C2628161704700BFEB
:108B60002DE9F0410446406A00681E460F469046D3
:108B70006EF05EFD237F002B3FD02A4DA0690523B8
:108B8000EB67030E85F8453005F146039870020C3B
:108B9000000A58701A703B68C5F888300020D8F871
:108BA0000030C5F89030012E2363C5F8A0002BD00B
:108BB000022E20D1D8F80420C5F89800796885F8ED
:108BC0009400C5F89C1013441749C5F8A42001204F
:108BD000236385F8A800C5F8AC10144B617F606A68
:108BE00003F11402002914BF1946114612F04AFE7F
:108BF000E36A8BB1206BBDE8F0810A4DA0690423C4
:108C0000EB6705F14503C1E7074B85F89460C5E9BB
:108C10002630C5F8A400E0E7636A18686EF008FD26
:108C2000E8E700BF88010020658A0008D401002021
:108C3000704700BF00B583B081610192049A009330
:108C4000C26201236A4601A9FFF78AFF03B05DF8FB
:108C500004FB00BF04307047C2628161704700BFEF
:108C6000436A1B681B6A5B689B78024613F001002D
:108C700008BF5077704700BF01234377002070473B
:108C8000D0E90B2108B583690B4483610AB108461A
:108C90009047002008BD00BF704700BF04307047F8
:108CA00010B4094CD4F8B8074FF0340C0CFB00F0AA
:108CB00004EB000C04F2BC742044DCF8BC47A4694B
:108CC000A4465DF8044B6047F01E0020064BD3F825
:108CD000B827342101FB02F203F2BC7013441044A4
:108CE000D3F8BC37DB691847F01E0020043070470A
:108CF0000D4B93F82828D3F824180244D2B283F8F5
:108D0000282893F8282808441206C3F8240805D513
:108D100093F8282882F0800283F82828034B012248
:108D200083F8C420704700BFF01E00208801002097
:108D30002DE9F047144FD7F82C58ED0A1ED0002625
:108D4000B04607F66409D7F830381048D3F828A0A1
:108D5000C7F85C88AC19641010234A46E102D0477A
:108D60000F280BDD0A4B03F1100C53F8041B0131E3
:108D700007D16345F9D12546B542E4DCE802BDE8F8
:108D8000F087661CF8E700BFF01E002020270020B7
:108D9000542700201C4BD3F87418D3F878288A1A6B
:108DA000322A16D8D3F88C288A4200D37047D3F8D9
:108DB000802822B31068928810B44469323122426C
:108DC00018BF42835DF8044B08BF0283C3F88C18B8
:108DD000704793F87C28D3F8801802F0010219B18B
:108DE00032B90A68898811830022C3F88C28704739
:108DF0000A68898851830022C3F88C287047323171
:108E0000C3F88C18704700BFF01E0020094A92F882
:108E10007C38D2F8802803F001031AB123B9136813
:108E200092881A8300207047136892885A83002022
:108E3000704700BFF01E00204FF40070034B10601D
:108E4000D3F898380B600020704700BFF01E002058
:108E500000207047012070470120704700207047B4
:108E600010B51C6994420DD396468A188C469442DC
:108E7000996938BFA4EB0E0C71446246BDE81040FE
:108E800071F000BF10BD00BF30B4194B00209C7BB7
:108E900014B11D688D4206D001300B2803F1100378
:108EA000F5D130BC70479AB1124B03EB40218A4296
:108EB00019D0114B93F8E4278AB1104B01225A7054
:108EC00000F5B17003EB00100123837130BC7047D3
:108ED0000A4B00F5B17003EB00108271E1E701224B
:108EE00083F8E427E9E7022CE3D1183BE8E700BF69
:108EF000785D002078470020605700206047002000
:108F000030B41D4C002384F8D03604F5C36004E06F
:108F100001330B2B00F1100015D005688D42F7D1FD
:108F200090F80EC0BCF1030FF2D1C2B1134901EBAE
:108F30004320824209D1A1F1180203F5B17302EB7B
:108F4000031301229A7130BC704794F8E42712B9D8
:108F5000012284F8E4270A4A01215170EDE708490B
:108F6000D4F8CC2603F5B17301EB031301320421CD
:108F70009971C4F8CC26E6E76057002078470020B6
:108F800060470020A8B183681BB10E4B07229A707E
:108F900070470C4A1178D36003294FF004000CBFCE
:108FA00080214FF48071C2E9011113611375907033
:108FB0007047044A02F580510123537081F8E43769
:108FC000704700BF604700200C4AF8B51368556928
:108FD0002B4003EA000555617DB1094F0126B5FA22
:108FE00085F4C4F11F0407EB840306FA04F4D3F8F4
:108FF000C80803689847A543F1D1F8BD003C01407B
:10900000F01E0020038A2DE9F047B0F80C901FFAFB
:1090100089F919EA03092BD005460E464FF000479F
:109020004FF00008B9FA89F327FA03F2D24391B25C
:109030001B3B298209EA0209042B16D8DFE803F05A
:10904000352C231A0300B36A002B37D003F1FF3A03
:109050001FFA8AFAC6F82880746A34B12368204659
:10906000514698476468002CF8D1B9F1000FD9D166
:10907000BDE8F0877068696B036889B29847B9F1F9
:10908000000FCFD1F4E7B068A96B036889B29847A5
:10909000B9F1000FC6D1EBE7F068E96B036889B25C
:1090A0009847B9F1000FBDD1E2E73069296C036838
:1090B00089B29847B9F1000FB4D1D9E7E96A1FFA2C
:1090C00081FAC9E72DE9F0430446406A344D00684F
:1090D00095B00E46914698466EF0AAFA314B019330
:1090E000314B049305F1D0030093217F02230293B7
:1090F00005F1C802012300278DF80C300592069770
:10910000002936D08DF834308DF84830CDE9097714
:10911000330ECDE90E77CDE9107785F8C9300523F8
:10912000CDF82C908DF82070CDF830801397CA358B
:109130000793330C1D4F2B70330A6B70AE70D7F84A
:109140000C09656A12F0FCFE637FA88033BB05A999
:10915000284612F097FB636A18686EF069FAD7F830
:10916000100912F0EDFE636A9880404615B0BDE824
:10917000F0838DF834308DF848300423CDE909119F
:10918000CDE90E11CDE91011CDF82C908DF82010FD
:10919000CDF830801391C9350793CAE76946D7E700
:1091A00088010020F82700207D8A0008F01E00209A
:1091B00070B5224B93F8DC2493F8DD349A4237D112
:1091C0001F4D95F80436E3B195F808461D4B002075
:1091D00040F20D3CB4B19A689989516016681968DB
:1091E00046F001061660A1F848C08A8992B242F49E
:1091F00080728A8195F804260130824203F11803B7
:10920000E8DC70BD1A68118821F080010904090C9E
:1092100011809988D162118889B241F08001118052
:109220005462998A9689314389B291819C82E1E79F
:109230006CF0BAFB0028C3D170BD00BFF01E002047
:1092400004000010042800202DE9F0411E4B93F883
:10925000DC2493F8DD349A422FD11C4F7D68002D19
:1092600012DD3846002410F8086BA046013416B110
:10927000037E012B1CD002691368AC4243F001034A
:1092800000F580701360F1D114F052FAD7F80C4653
:10929000002C0BDD0E4A02EBC40411689388888908
:1092A000083203439BB294428B81F6D1BDE8F08132
:1092B00080F8F080FFF7F8F9DDE76CF075FB002827
:1092C000CBD1BDE8F08100BFF01E002004000010EB
:1092D000140600102DE9F04F037D02681F2B83B0A8
:1092E000044609D95068A3F120052021A940014274
:1092F00007D103B0BDE8F08F1068202199400142EA
:10930000F7D05149514D4968C5F8301695F80816FF
:10931000A7694F4E19BB8C2101FB0761D1F884006E
:10932000D1F8FCE0D0F800C0DEF80000B1F8888089
:1093300020F00100CEF80000BCF80C1089B221EA40
:109340000801ACF80C10297801BB1F2B6FD9A3F1D1
:10935000200120238B40D36003B0BDE8F08F8C2127
:1093600001FB0761D1F88410D1F810C00868DCF85F
:10937000001021F00101CCF80010818921F48071E6
:109380000904090C818129780029DED04FF08C086E
:1093900008FB07F806EB08032E49D3F8FCA0D3F826
:1093A00084200193504608F11809D2F800B089448E
:1093B00060F01CF8019BD5F838262649012083F877
:1093C000D000002A3AD0BBF800309BB243F08003B3
:1093D000ABF8003008F174084FF0FF334144CBF88C
:1093E0002C30584660F06CFA8C2303FB0766002390
:1093F0004946C6F8A030504660F08EF8D6F8FC30EA
:1094000016225A601A6842F001021A60D6F88420C7
:10941000B6F88830126891890B439BB293810A4950
:10942000237D49682268C5F834161F2B8FD8202168
:1094300001FA03F3936003B0BDE8F08F14F078F9FC
:109440000449C5F83806BEE7001000E0040000102B
:10945000F01E00206C1F00202DE9F04114F068F987
:109460001F4F204E05464FF000087C68002C2ADD77
:1094700000231A4607EB0321013391F8F9109C42AF
:1094800042EA0102F6D142EA0804E4B29046736867
:10949000C3F30803A3B9EFF311838BB919F000F8F4
:1094A000431BB3F5FA6F02DCB8F1000FDDD124B134
:1094B0000D4B93F8D429542A09D02046BDE8F081F9
:1094C00014F00AF9ECE744464FF00008DFE7B3F880
:1094D000DC290132A3F8DC292046BDE8F08100BF79
:1094E0000400001000ED00E0F01E0020BC4B1B78D3
:1094F0000BB9012070472DE9F04FBA4DBA49D5F8A4
:109500007428BA4BA1FB02125209A3FB023A4FEA9C
:10951000DA0A0AEB8A0AA2EB4A0A85B0B04A5FFA75
:109520008AF3039302F61C1302F23C6701930023B3
:1095300007EB8A0A02F581699846A94BD3F8243AC9
:10954000434540F31781D9F81830D9F80460D3E9BE
:109550003A34029314F0ECF8029B95F8D4C90290C7
:109560004FEA860E95F8E8090EF1085E04F1806175
:109570000EEB431E3939BCF1540F0EEB81110EEB8B
:10958000801301D1A5F8DE09994240F26A811A6878
:10959000002A00F05E811A6C002A00F07081D3F876
:1095A0008020002A00F06D81D3F8C02003F580737D
:1095B000002AE9D1A3EB0E0E99424FEAAE1E40F20B
:1095C0005081A4EB0E0145294FF0000428BF45212E
:1095D00003EB81119B46204626460DE01A6C002ABB
:1095E00040F0D080D3F88020002A40F0F680D3F8F5
:1095F000C02003F580732AB9994206D91A68002A57
:10960000ECD04033994200F2C180112E344640F232
:109610002C81D6F1150200F128817549029ED1F8FE
:10962000D4309E45D5F8EC3938BFC1F8D4E0F11AF2
:10963000002919DB03F5F42303F590739E4288BFDC
:10964000029B6B4988BF0533C5F8EC39684BD3F8EA
:10965000D430052B86BF053BDBB2002385F8E83903
:109660004FF0FF33C1F8D43042B100FA02F2C4F136
:109670001404012000FA04F444EA02005D4BC0F334
:10968000C43203EB8202D2F8981400F01F0203EBFD
:109690008202D2F8982442EA0131C0F3441203EB6B
:1096A0008202C0F3842003EB8000D2F8983441EAB0
:1096B0000311D0F8983441EA032181EA112383EAA7
:1096C000131303F00F030F2B40F0B180B1F5803F6F
:1096D00080F0AD80BCF1540F4FEA111104D1B5F800
:1096E000D8390133A5F8D8393D4AD2F82439B1F533
:1096F000606F03F10103C2F8243900F0D480019BAC
:10970000998197F858300398834210D0DAF80820EE
:109710003B689B1A3B60DAF830207B689B1A7B60C1
:109720000023CAF80830CAF8303087F858003B6880
:1097300001333B60DAF808300133CAF808304FF6DD
:10974000FF73994207D17B6801337B60DAF83030D0
:109750000133CAF83030019B08F101081433B8F125
:10976000080F07F15C070AF15C0A019309F120096F
:109770007FF4E3AE1A4A0123012082F8203A05B0B3
:10978000BDE8F08F803399427FF63FAF5A469A1A70
:109790009211541C184A82FB04B2A2EBE472012A13
:1097A000B8BF0122904001241644013A04FA02F2A3
:1097B00010431C4622680AB3226C002A63D0D4F8F6
:1097C0008020002A61D0D4F8C02004F58074B2B1A2
:1097D000A142EFD89B4623460EE7C03312E700BFF5
:1097E00004000010F01E00201F85EB51CDCCCCCC26
:1097F0008801002014AE0708565555554034A14243
:10980000E8D9E31A9B115A1C2F4B83FB02B3A3EB3D
:10981000E273012BB8BF012398401E440122013B93
:1098200002FA03F3184323469B462346E4E6BCF1C1
:10983000540F2CD0254AD2F824390133C2F82439E8
:10984000224AD2F820390133C2F820394FF6FF718D
:1098500057E74033A3EB0E0E99424FEAAE1E3FF698
:10986000B0AE10B1013885F8E809BCF1540F7FF4AF
:1098700072AFB5F8DA390133A5F8DA396BE780331E
:1098800098E6C03396E68034B9E7C034B7E7B5F858
:10989000D8390E4A0133A5F8D839D2F82439013322
:1098A000C2F82439CCE795F8DD3403EB430305EB2C
:1098B000C303434493F8ED340D2B7FF420AF019A9A
:1098C000802393771DE700BF5655555504000010BF
:1098D00010B5044670F05EFC81B22046BDE8104031
:1098E000FEF740BE38B50B4D00EB400005F2445387
:1098F00003EBC00393ED027AD3ED037AE7EE007A2F
:10990000C4002C44B0EE670A70F044FCD4F844352F
:10991000186038BD040000100A4608B5054920B992
:10992000054860F0F3F8034808BD044860F0EEF81D
:10993000004808BDE0280020244908084C490808D0
:1099400010B5044C04480A46214660F0DFF8204672
:1099500010BD00BFE02800207449080810B5044C71
:1099600004480A46214660F0D1F8204610BD00BFE9
:10997000E02800208849080810B5044C04480A462D
:10998000214660F0C3F8204610BD00BFE02800204B
:109990009449080838B590F82830012B044604D0C3
:1099A000407F40B10023637738BD406A03681A7B6B
:1099B00092B9637F0BB9012038BD0A4D0A490223D1
:1099C00005F52F6212F072F895F8F13A03F00103F1
:1099D00083F001006377E7E71B6A002BE9D00020E2
:1099E00038BD00BFF01E0020600200202DE9F041CC
:1099F0000446154E90F82800637F144F06F52F6833
:109A0000012805D00BB1002363770120BDE8F08168
:109A1000606A05682A7B82B9002BF6D00223424691
:109A2000394612F043F896F8F13A03F001036377F0
:109A3000002BEAD094F82800E2E72A6A002AE8D14D
:109A4000002BE2D0EAE700BFF01E002060020020F9
:109A5000F0B511F0010583B00AD190F82860012E0D
:109A6000044607D0C368B3F1807F01D9012323776F
:109A700003B0F0BD0A4B476AD3F80C0912F060FA44
:109A8000E368B880B3F1807FF2D9B7218DF8041074
:109A9000267733462A46384601A912F007F8E7E749
:109AA000F01E002010B590F82830012B044603D09A
:109AB00000230120637710BD406A03681A7B3AB91E
:109AC0006DF0BAFD00F0010383F001006377F2E767
:109AD0001B6A002BF4D0002010BD00BF38B5114D1B
:109AE000044694F82830012B05D000236377002327
:109AF0002362012038BD606A03681A7B72B96DF079
:109B00009BFD00F0010060770028F0D0D5F8743894
:109B1000226A9B1A002BE4DB002038BD1B6A002B55
:109B2000EDD0F3E7F01E002010B5FF22044690F8B8
:109B30002810406A6EF09AFC0E4BD3F8743803F587
:109B4000FA7323622046FFF7C9FF94F82830012BEF
:109B500000D010BD606A0022A0216EF061FC94F874
:109B60002830012BF5D1606A1822BDE81040B021E1
:109B70006EF056BCF01E0020CB0700D5704710B524
:109B80000446FFF7D1FF94F82830012B00D010BD18
:109B9000024812F0D5F9636A988010BD00E1F5051E
:109BA00038B504460D46FFF799FF062294F82810B1
:109BB000606A6EF05BFC94F8283001229342627771
:109BC00005D0064BD3F874380F33236238BD606A72
:109BD000EA0AD8216EF000FCF3E700BFF01E002077
:109BE0008388002B4AD02DE9F04F8DB0DFF89080AC
:109BF0000446002606274FF001090DF1070509E08C
:109C000084F81D90D8F87438A28801360F33B24218
:109C1000236230D92046FFF761FF94F828A0D4F8DA
:109C200024B08DF80770BAF1010FE9D1002302A921
:109C30005846CDE90253CDE90633CDE908330B93FD
:109C4000CDF810A08DF814A08DF828A011F01AFE00
:109C5000DBF800006DF0ECFC94F8283084F81DA0CF
:109C60007204012B4FEAD2224FF0D801CAD1606AA8
:109C70006EF0B2FBC6E70DB0BDE8F08F704700BFD5
:109C8000F01E002070B5104D95F8F23A03B970BD82
:109C9000D5F8F46A0D4B0446F60AC3F8DC60FFF70A
:109CA0001DFF94F82830012B07D0D5F87438002216
:109CB0000233236285F8F22A70BD606A32461021B1
:109CC0006EF08AFBF1E700BFF01E00208801002043
:109CD0002DE9F047414F1E46D7F8DC30B3EBD12FCA
:109CE00090B00C460546904621D1DFF8F49095F8E7
:109CF0002830C4F30A04C4F50060B04234BF87B210
:109D0000B7B2012B3CD0D9F87438023328462B6205
:109D1000FFF7E4FE38B195F82830012B23D0384600
:109D200010B0BDE8F087002010B0BDE8F0874FEA22
:109D3000D12AFFF7D3FE0028F5D095F828304FF050
:109D4000FF32012BC7F8DC2042D0DFF89490D9F81D
:109D50007438023328462B62FFF7C0FE0028E2D099
:109D6000C7F8DCA0C3E7686A6DF066FCC0F30110B9
:109D700001380228D3D82846FFF7D6FE3846CFE769
:109D80008DF80240240A8DF801406C6A8DF8243069
:109D90008DF83830032300228DF80030204604234C
:109DA00001A9CDE90786CDE90522CDE90A22CDE951
:109DB0000C228DF8032002928DF810200F92CDF81E
:109DC00004D0039311F05EFD20686DF031FC9AE73A
:109DD000686A524613216EF0FFFAB6E78801002048
:109DE000F01E00202DE9F843436A394E04461868F6
:109DF0000F4690466DF01CFC96F8F23A002B37D0D7
:109E0000344DD6F8F83A85F88231C3F3022385F849
:109E1000813105F1E0093B68C5F88831D8F8003098
:109E20002D4AC5F89031606A00234946C5F898313B
:109E300012F0EEF8D6F8F83AD8F800201344C6F835
:109E4000F83AC3F30A07012386F8F23AFFB1234B2D
:109E5000C5F89831637F0BB909F11409606A226370
:109E6000494611F00FFDE36A53B3206BBDE8F88358
:109E7000A369184DC6F8F83AC6F8F43A85F8863161
:109E8000C3F3022385F8853105F59879C3E7D6F841
:109E9000F43A134A606AD90AC5F8DC10DB0C85F87D
:109EA000B311A2F12C0185F8B23112F0B1F8D6F855
:109EB000F83AD8F8002086F8F27AC6F8F43AC9E7FA
:109EC000636A18686DF0B4FB206BBDE8F88300BFCF
:109ED000F01E00208801002010030020818C000863
:109EE0003C03002033B910B51C46C36A204698478E
:109EF000204610BD76E700BF00B583B081610192B6
:109F0000049AC26201A96A460093FFF76BFF03B08F
:109F10005DF804FB2DE9F047089F884615460021AF
:109F2000202204461E4670F010FF4FB13B68E381CB
:109F30001B0C23827B687A89E3821B0C6282238359
:109F400040466EF0B5FAEB0619D4431EB8B108EBE3
:109F5000000701E0013B12D317F801CDBCF12E0F31
:109F6000F8D1C01A421E032AA8BF0322082B03F10E
:109F7000010AA8BF08239146C2441A4606E00828F1
:109F80000246C246A8BF08224FF000094FF0203316
:109F900041462360636004F10807204670F072FEBA
:109FA000174B23815146BB704A46384670F06AFE13
:109FB000611EE31D11F801CFACF1610EBEF1190F66
:109FC0009CBFACF1200C81F800C08B42F2D1384626
:109FD00004F10B0110F8013BA3F16102192A9CBFA7
:109FE000203B00F8013C8842F4D118232373330C42
:109FF000A382E572099B6683E361BDE8F08700BF39
:10A00000202020002DE9F04FDFF88894D9F874085B
:10A01000C9F8780887B0002B00F0DA8001F5FE78E7
:10A020001344DFF874B40393164601F12007C246C7
:10A0300021E0002E64D0D9F8A438B34200F0CC80DF
:10A04000D9F8A038B34200F0FF80D9F8A838D9F881
:10A05000AC18B3424BD8B14200F29981711A204634
:10A0600069F0D4FF039B01369E4207F500770AF59D
:10A07000007A00F0AD80D9F8B058B542A7F12004BD
:10A08000D7D8751BD9F8C08805F00702EB080492F1
:10A09000D8F830200233934203D3D8F838209342C3
:10A0A0000BD941461846059369F080FF059B804611
:10A0B000002800F08C81C9F8C00898F80420002A14
:10A0C00040F03481D8F82850002D00F07981D8F87C
:10A0D00030209B1A049A02EBC303D8F80C202046C8
:10A0E00002EB43224FF400714346A847BAE7B1425E
:10A0F000B4D920464FF40072002170F026FEB1E77B
:10A100004FF400723146204670F01FFE802387F81E
:10A110009E310C2387F8A231D9F8A038D44AD9F857
:10A120009818C4F8C6319342C4F8CA1100F33481B8
:10A13000D04AD14C82FB03021A44D817C0EB6212FA
:10A1400084FB0254CD4D85FB03C5C0EB2530C2EB2B
:10A15000821587F8A1015B1B801020F03F000133BE
:10A160000343144487F8A031D317C3EBE41422440B
:10A17000BF4B87F89F214A1E9A4200F31981BD4BBD
:10A18000BD4883FB02311144D317C3EB611180FB3F
:10A190000140BA4C84FB0254C3EB2433C1EB81145D
:10A1A00087F8A531121B9B1023F03F0301321343A4
:10A1B000084487F8A431CB17C3EBE010014487F8BB
:10A1C000A311552387F8DE31AA2387F8DF3149E749
:10A1D000002007B0BDE8F08F4FF0FF3384F8EC317A
:10A1E00084F8ED3184F8EE3184F8EF31D9F8B838DD
:10A1F000C4F8E8315223237063706123A37084F89C
:10A20000E73141230025E37084F8E631722384F8B6
:10A21000E43184F8E5314FF4F0722946A7F11C00CF
:10A2200070F093FD5523C7F8D051C7F8D451C7F843
:10A23000D85184F8FE316FF0550384F8FC5184F84E
:10A24000FD5184F8FF310DE700214FF400722046E4
:10A2500070F07BFD8A4A03CA47F81D0CEB2007F813
:10A26000200C582007F81F0C902047F8191C07F8FD
:10A270001E0C002302220821F820E372227307F843
:10A28000131CA273E37307F8102C07F80B0CD9F812
:10A29000A00884F82C20D9F898286376121A226234
:10A2A000D9F8A808D9F8AC28E376121A3F2020760E
:10A2B0004FF0FF30A0763E20207701206377A37710
:10A2C000E37784F82D3084F82E3084F82F306262E2
:10A2D00084F8300084F8313087F82610802187F820
:10A2E0002010292187F82210942187F823100E21AD
:10A2F00087F824100D21634A87F82510552187F827
:10A30000DE11AA2187F8DF1103CA5F4BC7F82700C7
:10A31000C7F82B1003CB1388A7F82F309378C7F812
:10A320003200C7F8361087F831309BE64FF40072E0
:10A330000021204670F009FD049B002B4ED1D8F877
:10A340004030002B00F0AA80049AD8F830304F49F2
:10A35000CDE9002220461122FFF7DCFDD8F840307D
:10A360001A6C002A00F0AD80049A1B6BCDE9002224
:10A37000474911223846FFF7CDFDD8F8448007F150
:10A3800020044FF4E075B8F1000F3FD16AE6F11AEE
:10A39000204669F03BFE65E6FF2387F89F3187F88A
:10A3A000A13187F8A031324B4A1E9A427FF7E7AEBF
:10A3B000FF2387F8A33187F8A53187F8A43100E798
:10A3C000294620464FF4007270F0BFFC4AE6A7F120
:10A3D000240343F804BF9A45FBD143E6D8F8403044
:10A3E000049AD8F84480002B0CBF01230223C3EB4E
:10A3F00002154346002B3FF435AE013D9B6CF9D16D
:10A4000098464FF40075002B3FF42CAE25442034C1
:10A41000234620354446049698460EE05CF81C1B03
:10A42000236BCDF800C000260196FFF773FDA46CE6
:10A4300008F12008CCB1A84517D02379A44604F12F
:10A440001C0E1122A8F12000002BE7D162792669A9
:10A45000236B216842F02102CDE900E6FFF75AFDA7
:10A46000A46C08F12008002CE5D1049EFAE500BF99
:10A47000FF03FB008320088281808080975545413F
:10A48000AC490808B8490808C4490808A44908089C
:10A49000A8490808F01E0020DEADBEEF049BD9F8E5
:10A4A0009C18CDE9003320460822FFF733FDD8F889
:10A4B0004480B8F1000F3FF4D5AD3C464FF4F07541
:10A4C000A4E7049BCDE9003352E700BF58B183886D
:10A4D0004FF00042B3FA83F332FA03F303D0024998
:10A4E0000A6813430B607047003C014090F8DB3072
:10A4F000052B03D890F81E31032B01D000207047A4
:10A5000090F8233103F0FB03022B0CBF002007203F
:10A510007047084B10B5D3F8FC3A18440C46807DC0
:10A5200011F0DCFF18B1828803680CB11A8310BDEA
:10A530005A83FCE7F01E002010B42A492A4A91F8F9
:10A5400004367BB3D2F81449A04239D0012B29D06C
:10A55000D2F82C49844239D0022B23D0D2F8444976
:10A56000A04235D0032B1DD0D2F85C49A04231D097
:10A57000042B17D0D2F87449A0422DD0052B11D04E
:10A58000D2F88C49A04229D0062B0BD0D2F8A4498E
:10A59000A04225D0072B05D0D2F8BC49844208BF81
:10A5A00007230ED003F1010C81F804C603EB43012D
:10A5B00002EBC1025DF8044BC2F81409184670475B
:10A5C0000023DBB218465DF8044B70470123F8E71F
:10A5D0000223F6E70323F4E70423F2E70523F0E779
:10A5E0000623EEE704000010F01E002038B5424CB0
:10A5F0008C2303FB004393F88B3003B938BD94F8E8
:10A60000DCC494F8DD349C450ED003EB430204EB2C
:10A61000C20292F8E0E40EF1FF35012D4FEA430249
:10A6200046D9BEF1030F3ED08C2202FB0042A2F8B5
:10A630007C10EFF31181902383F31288B2F87C50E1
:10A6400092F87E3043EA45030025C9B29BB282F8F6
:10A650007E5081F3118829491A090D7882EA132264
:10A660005A4005B1D2431B019BB202F00F021A43BC
:10A6700091F808365BBB8C2303FB0044D1F8283AE1
:10A68000D4F8040101219847D4F80011B4F8885097
:10A690008A8AD4F8FC302A438A8258601A6842F0C9
:10A6A00001021A6038BD5D1C05F003056545BBD08D
:10A6B000134404EBC303034493F8ED140029B3D00F
:10A6C0008C2303FB0043012283F87E20ACE78C231C
:10A6D00003FB0044D1F8285AD4F88430D4F8001190
:10A6E0005B79086903F0FC0318440421A847D4F8F7
:10A6F00000318000988138BDF01E00200400001059
:10A7000043680B4A23F0407323F4807343F480734F
:10A71000436083681A4042F002028260C36A0139D2
:10A72000CAB223F4700141EA0251C162704700BF0E
:10A73000FDF7FFC0704700BF0020FDF773BC00BFEE
:10A740000120FDF76FBC00BF0220FDF76BBC00BF0E
:10A7500010B1036882881A83704700BF30B1036864
:10A7600082881B691A4214BF01200020704700BF75
:10A7700010B1036882885A83704700BF10B404691F
:10A780008269E468416814604024D460446900230D
:10A790000C31C2E90433C2E90633C2E90833C2E925
:10A7A0000A33C2E90C3393609363516084B1C26988
:10A7B000E0689363C2E90233C2E90433C2E90633B5
:10A7C000C2E90833C2E90A33C2E90C33C2E9000125
:10A7D0005DF8044B704700BF436800221A60037D98
:10A7E0001F2B08D9203B2022016802FA03F343F013
:10A7F0001803CB6070472022016802FA03F343F08C
:10A8000018038B60704700BF0268136A11B1D969E1
:10A8100001B3143330B49C681D689169DDB14FF405
:10A82000806088618D60104640690C6180B1596814
:10A83000D369D9B10A464FF480619A609961224385
:10A8400012F0010F14BF00224FF400521A621C6173
:10A8500030BC704770478D61064D4FF0FF0C85F896
:10A8600004C205F5017500688D60DDE7024A9A6053
:10A870009961E4E788010020F02900200168F8B51B
:10A88000D1E9042304465568002B49D09861107D16
:10A890005E681F2831D81768202202FA00F040F0C5
:10A8A0001800B8601A7D1F2A32D91868203A202370
:10A8B00003FA02F242F01802C26000232B603360F8
:10A8C0003368896943F01003336028465EF024FE44
:10A8D00023683046D9695EF01FFE2B68226843F07A
:10A8E00001032B603368526843F00103336093889F
:10A8F0009BB243F003039380F8BD176820382022F1
:10A9000002FA00F040F01800F8601A7D1F2ACCD837
:10A910001868202303FA02F242F018028260CCE7A2
:10A92000137D90611F2B1CD81068202202FA03F3BC
:10A9300043F01803836000232B602B68896943F080
:10A9400010032B6028465EF0E7FD2B68226843F079
:10A95000010352682B6093889BB243F002039380FB
:10A96000F8BD1068203B202202FA03F343F01803DD
:10A97000C360E0E72DE9F0417F4D804E07463C681B
:10A9800097F888806368B888012284F824201A88A0
:10A9900022F040021204120C1A802289824223D033
:10A9A000198821F038010904AB424FEA114100F047
:10A9B000BF80734A934200F0BB800246B2F5807FAD
:10A9C000A8BF4FF48072022AB8BF0222002A92FA6E
:10A9D000A2F2B2FA82F208BF4FF0FF32013A41EA26
:10A9E000C20292B21A802081397BA27A8A420CD0AC
:10A9F0001A8822F003021204120C1A801A8892B2EA
:10AA0000002900F092801A80A1721A8892B242F056
:10AA100040021A80226A9168002900F0A3804FF05A
:10AA2000000C1432E64652F8100C8E4400EA06017F
:10AA300020B1B1F1805F23D0616909B352F8140CE1
:10AA4000143200EA060110B1B1F1805F18D052F85B
:10AA50000C1C0CF1010C0029E5D1227B82B1B8F16C
:10AA6000000F0DD0BCF1010F6FD8BEF1070F6CD8ED
:10AA70000CEB8C018900226A11440A7B002A64D005
:10AA8000226A92684FF00008002A53D0B8F1000FF4
:10AA900002D098F80C2022B1BA6812B111689288DD
:10AAA0004A83226AD2F800E0226A5168226A9268D8
:10AAB000501E9AB1BEF1000F23D01EF801CB1A89A7
:10AAC0009207FCD5A3F80CC01A89D207FCD59A8945
:10AAD00092B209B101F8012B0138EBD2236A1B7B3A
:10AAE000E3B9236A1B697BB1236AD7F894001B6919
:10AAF000984701280DD0022806D100232362BDE823
:10AB0000F0814FF0FF0CDAE7D4F82080236A143389
:10AB10002362236A9B686BB16368B7E7BB68002B4D
:10AB2000DFD01A689B881383DBE742F003026AE7F1
:10AB3000420843E7236A1B68DBB1236AD3E900724A
:10AB400022620022C3E9002219E700213846FFF7FC
:10AB50005BFEBB6813B11A689B8853833846BDE817
:10AB6000F0418BE6227B002A8AD0B8F1000F82D117
:10AB700086E72362C3E700BF003800400000FFFF04
:10AB8000003C004038B5D0F8E0102B4B04465A6822
:10AB9000D0F8D80071B1131A99420BDC94F8D03078
:10ABA000C4F8D820012B10D0D4F8D4300133C4F825
:10ABB000D43038BDD4F8E430C4F8D8200344C4F805
:10ABC000DC3094F8D030012BEED16168201D04F107
:10ABD000E805EFF3118C102383F3128863681B6A76
:10ABE0000BB3D4F8F0302A461BB1D3691432002BD2
:10ABF000FBD10B6A6BB1996839B9934209D01968D6
:10AC000029B15B6899680029F7D01433F3E7C3E9E9
:10AC100000055FFA8CFC8CF31188D4F8D430013332
:10AC2000C4F8D43038BD0D625FFA8CFC8CF3118807
:10AC3000FFF7A0FEB8E700BF001000E02DE9F041EB
:10AC4000826992F8DC30012B8AB005464CD0023B79
:10AC5000012B54D892F84C31D2F89C202E4C63F042
:10AC60007F0313708669D6F8A030D6F8108003F100
:10AC7000010E0FCCEC46ACE80F00D6F89C30CDE9C5
:10AC8000003E0FCCACE80F0094E8030006F110077B
:10AC90008CE80300EFF31180102383F312883369EB
:10ACA0001B6A002B2FD0029B6A461BB1D36914325A
:10ACB000002BFBD1D8F8203073B1996839B9934291
:10ACC0000AD0196829B15B6899680029F7D0143354
:10ACD000F3E71F60C3F804D0C0B280F31188AA69FB
:10ACE00011690B6A002BFCD1D2F8A0305A8852BAF5
:10ACF000EA819A8852BA2A82DB885BBA6B82012089
:10AD00000AB0BDE8F081C8F820D0C0B280F3118845
:10AD10003846FFF72FFEE2E72CB307082DE9F04194
:10AD200090F8DC30D0F8A050012B8AB0044672D0E5
:10AD300016D8D0F89C304FF0FF321A605A609A60F3
:10AD4000DA60D0F8E0300522B3F57A7FC0F8F02061
:10AD50007CD8032380F8DC3001200AB0BDE8F08104
:10AD6000023B012BF8D890F84D31D0F89C20524E80
:10AD700063F07F031370D0F8A030D0F8108003F197
:10AD8000010E00F110070FCEEC46ACE80F00D4F82E
:10AD90009C30CDE9003E0FCEACE80F0096E80300F2
:10ADA0008CE80300EFF31180102383F312882369EA
:10ADB0001B6A002B73D0029B6A461BB1D369143205
:10ADC000002BFBD1D8F8203073B1996839B9934280
:10ADD0000AD0196829B15B6899680029F7D0143343
:10ADE000F3E71F60C3F804D0C0B280F31188226972
:10ADF000136A002BFCD16B885BBAA4F8D030AB8807
:10AE00005BBAA4F8D230EB8801205BBAA4F8D43046
:10AE10000AB0BDE8F08190F84C2190F84D319B1AB2
:10AE20005B100133DBB205EB430235F813305BBA3C
:10AE3000A0F8D03053885BBAA0F8D23093885BBAC0
:10AE4000A0F8D43001200AB0BDE8F08103691A7B74
:10AE500072B35B6963B390F898304BB390F84C31A0
:10AE6000D0F89C20C4F8A40063F07F03137090F81E
:10AE70004C1190F84D31D0F8A0201048C4F80401CE
:10AE80005B1A07330121C4F8FC30D4F89C3084F8F5
:10AE900000110A44C4E93D3284F8DC105CE7C8F8CC
:10AEA00020D0C0B280F311883846FFF763FD9EE7DB
:10AEB000022384F8DC304FE72CB307080180000838
:10AEC00008B51D2011F00AFB08B183794BB11E2093
:10AED00011F004FB08B1837903B108BD5523C38089
:10AEE00008BD5523C380F2E7D3B2012B23D870B538
:10AEF00002EB4202114C4FEA820E4FF0000C224648
:10AF00000EF10805634604E00133152B11D012F849
:10AF10001CCF6045F8D192F801C08C45F4D1565948
:10AF2000002EF1D0C3EBC3030EEB83030433E01810
:10AF300070BD002070BD0020704700BF54B30708EB
:10AF400010B40C4C002304F6043C01E0152B0CD08B
:10AF500003EB430201331CF802108142F6D1224474
:10AF60005DF8044B92F9060B70474FF0FF305DF827
:10AF7000044B7047F01E0020D3B2022B21D830B50D
:10AF800002EB4202104D114C4FEA820C0CF10C0EF8
:10AF90002A46002304E00133172B10D052F82C4F1F
:10AFA000A042F8D114798C42F5D152F80E40002C11
:10AFB000F1D02C2202FB03C30833E81830BD002077
:10AFC00030BD0020704700BF14AE070800000140EC
:10AFD000002838D030B51C4D90F804C0002305F689
:10AFE000043401E0152B2CD003EB43020133A15CA8
:10AFF0006145F7D12A44046892F9063B90F805E0D0
:10B00000DAB2022A1DD803EB4303104810494FEA75
:10B01000830C02460CF10C05002304E00133172BCE
:10B020000FD052F82C1F8C42F8D111797145F5D10F
:10B0300051590029F2D02C2202FB03C308331844D3
:10B0400030BD002030BD7047F01E002014AE070850
:10B05000000001400348D0F8183213B100F5027027
:10B0600018477047880100200348D0F83C3213B1DC
:10B0700000F50B7018477047880100200348D0F88E
:10B08000603213B100F51470184770478801002032
:10B090000348D0F8843213B100F51D70184770478B
:10B0A000880100200348D0F8A83213B100F52670BB
:10B0B00018477047880100200348D0F8CC3213B1FC
:10B0C00000F52F7018477047880100200348D0F81A
:10B0D000F03213B100F5387018477047880100202E
:10B0E0000348D0F8143313B100F541701847704786
:10B0F000880100200348D0F8383313B100F54A70B6
:10B1000018477047880100200348D0F85C3313B11A
:10B1100000F5537018477047880100200348D0F8A5
:10B12000803313B100F55C70184770478801002028
:10B130000348D0F8A43313B100F565701847704781
:10B14000880100200348D0F8C83313B100F56E70B1
:10B1500018477047880100200348D0F8EC3313B13A
:10B1600000F5777018477047880100200348D0F831
:10B17000103413B100F58060184770478801002033
:10B180000348D0F8343413B100F224401847704714
:10B1900088010020094B0A4A013800EBC00003EB8C
:10B1A0008000116BD0F80832064883420CBF4FF480
:10B1B00000134FF480030B43136370478801002092
:10B1C000003802400060024070B501383C4C3D4DF3
:10B1D00000EBC00C04EB8C0C9646DCF808623A4A93
:10B1E000AE420CBF4FF400154FF48005166B35438B
:10B1F0001563CCF81812CCF820323449DCF80C3244
:10B200008B424FEAC0023ED001F580618B423AD0BA
:10B21000A1F57A718B4247D001F580618B4243D012
:10B22000A1F57A718B4241D001F580618B423DD00E
:10B23000A1F57A718B4235D001F580618B4231D016
:10B24000A1F57A718B4233D001F580618B422FD00A
:10B25000A1F57A718B422DD001F580618B4229D006
:10B26000A1F57A718B4227D001F580618B4223D002
:10B27000A1F57A718B4221D0154D01F580618B4289
:10B2800018BF002500E0134D104404EB8003CEF3FB
:10B290008711C3F8285293F81D02BDE870400022C0
:10B2A00069F004B90C4DEFE70C4DEDE70C4DEBE701
:10B2B0000C4DE9E70C4DE7E70C4DE5E7044DE3E7FE
:10B2C0008801002000600240003802401060024007
:10B2D00000800028208000100080001800880010E6
:10B2E0000080201020800020008800200080202086
:10B2F0000D4B984214D0A3F58063984210D003F50B
:10B30000804398420CD003F58063984208D003F53F
:10B310008063984204D0054BD3F8B00740087047CB
:10B32000024BD3F8B007704700040140F01E002024
:10B33000800AA0F58010522808D8054B184490F8D0
:10B34000F4330D2B02D8034AD056704700207047C3
:10B3500014AE0708A44A0808094910B54B6C094CFB
:10B3600043F480434B644022002104F6C8006FF090
:10B37000ECFC4FF0FF33C4F8443BC4F8473B10BD2E
:10B3800000380240F01E00200120FDF71DBE00BF66
:10B390000220FDF719BE00BF0420FDF715BE00BF57
:10B3A0000820FDF711BE00BF1020FDF70DBE00BF45
:10B3B0004FF47870FDF708BE4FF47C40FDF704BEF3
:10B3C00030B50C4683B0054618B3036803F13F431C
:10B3D00003F57E039B0A104A134493F88C0769F027
:10B3E000F1F9A988009104F00303C4F381028DF8F8
:10B3F000043028688DF80520C4F300136946C4F3AF
:10B4000041148DF806308DF807405DF057FF03B00A
:10B4100030BD4FF0FF33DEE714AE070800B1CFE7D1
:10B42000704700BF2DE9F04302691778012F85B0FE
:10B4300004460D4618D10B79013B13714B79002B53
:10B4400008BF682300F1100803754FF000093B4660
:10B450000DF10502752140468DF8059010F0F4F8C5
:10B46000064600283ED1226902231370EB7823B9E7
:10B470000026304605B0BDE8F08304F11008A97835
:10B48000404610F087FD06460028F1D0E87811F01C
:10B4900025F8A0612B780133DBB210B1C3712223F0
:10B4A00083710921FFF7BAFFA069FFF751F9424AFA
:10B4B000D2F87438632BFBD94048DFF80891404F2D
:10B4C00010F03EFDA08202E059F8047F5FB34046D1
:10B4D000B84703460028F7D0206984F8D8306CF0CC
:10B4E000D5F8C6E720696CF0D1F83B4649460DF126
:10B4F0000602404610F0A8F89DF8063003F07E03DF
:10B500008DF8063008B1682B14D09DF8053003F093
:10B510007E03682B8DF805300FD0702BA9D1042342
:10B5200084F8D830A5E7E87810F0D8FF11F036F8A5
:10B530003E469EE784F8D8709BE70222062384F8F3
:10B54000D820194602AA404610F07EF8E0B19DF8D6
:10B550000D309DF80B209B00520002F0020203F018
:10B56000040313439DF8092002F0010213430BD09A
:10B57000012B1DD0022B17D003F00303032B13D094
:10B58000032017F089FB74E701230DF10702404601
:10B590000C2110F059F80028F2D09DF8073013F074
:10B5A0000F03EDD0042B03D0012384F8D93060E7DA
:10B5B000002384F8D9305CE7F01E002040420F00E1
:10B5C0001D530608A8B507080B4B10B5D3F8FC3A75
:10B5D00003440446987D10F081FF60B12E228271F1
:10B5E000621CC2710121FFF719FF20460021BDE84E
:10B5F0001040FEF78EBF10BDF01E00202DE9F8436D
:10B600009DF8208000287AD004468088B0FA80F027
:10B6100020281546C0F11F0271D0DFF804913C4E7E
:10B6200009EB020706EB820297F8B877C2F8C81850
:10B630004FF00042C24005D03649086820EA0200B7
:10B6400008604A6119462046FFF7BAFEA2882368BF
:10B65000B2FA82F4C4F11F0101F0FC0202F180424F
:10B6600002F59C3203F13F4303F57E0301F0030131
:10B67000D2F808C08900C3F387234FF00F0E8B4028
:10B680000EFA01F12CEA0101916091680B4393607D
:10B69000204B4FF000421968E24021EA0201196094
:10B6A00059681D4C21EA02015960D4F8001C11436D
:10B6B000C4F8001C996809EB880821EA0201996026
:10B6C000D96898F8C80721EA02011028D96018D073
:10B6D00000F1804000F59E3003681A4302603E444A
:10B6E00096F8443BAB420ADD0C4B86F8445BD85DD0
:10B6F000C5F387110022BDE8F84368F0D7BEBDE866
:10B70000F883996811439960D9680A43DA60E6E7DB
:10B71000F01E0020003C014000300140B44A0808FF
:10B7200014AE07082DE9F843044690F8210144F2CD
:10B730003B33A4F84C3108B9BDE8F8830509013D55
:10B74000052D00F00F0000F29B804F4F07EB4503E3
:10B75000B3F8D42742FA00F3DB0740F191800123CC
:10B7600003FA00F0013810403D446DF0CDFB474E28
:10B7700095F8E087464A804406F64C3909EBC8053F
:10B780002621AB88E980B3FA83F3202BE260C3F172
:10B790001F02D1D0174406EB82020C34C2F8C8480D
:10B7A0004FF0004232FA03F397F8B84705D0394A10
:10B7B000116821EA03011160536100212846FFF757
:10B7C000FFFDAB8859F83820B3FA83F3C3F11F00AB
:10B7D00000F0FC0101F1804101F59C3102F13F4292
:10B7E00002F57E0200F003008F688000C2F387221A
:10B7F0004FF00F0C82400CFA00F027EA000088603E
:10B80000886802438A60234A234910684FF0004742
:10B8100027FA03F320EA03001060506820EA0300CF
:10B820005060D1F8000C1843C1F8000C906820EA71
:10B8300003009060D06820EA0300D060D1F8082CA3
:10B8400026441A43C1F8082C96F8442BF02A08D84D
:10B85000002B3FF471AF0F490A6813430B60BDE83A
:10B86000F883F02386F8443B0C4B0022185D03213B
:10B8700068F01CFEAB88B3FA83F327FA03F3E7E71B
:10B88000034BE36058E700BF14AE0708F01E00202A
:10B8900085AB0008003C014000300140B44A080874
:10B8A00070B50E4CD4F8246A002E15DD04F58164C1
:10B8B000002503E0B54204F120040DD0237F0135BB
:10B8C000002BF7D0E0680028F4D0217DFFF778FD49
:10B8D000B54204F12004F1D1012070BD0400001034
:10B8E000F8B5037D85691F2B04464DD90168A3F186
:10B8F00020024E6820209040064234D0102393400E
:10B90000C860CB604B68D340DE0700F18380EFF363
:10B910001183502282F312882A6C1168C9075AD405
:10B92000516889B271B9D5E90960864250D0AF69D2
:10B930000744D76073D9301A80B25060AE620021DC
:10B9400085F86410116841F00101DBB2116083F3E6
:10B95000118895F86430002B44D1237D1F2B27D903
:10B960002168A3F120024C6808209040044200D0D6
:10B97000C8604C68042000FA02F2224203D0203B47
:10B9800000FA03F3CB60F8BD0268202016689840E7
:10B99000064219460ED010219940906091601168BE
:10B9A000D940C807B3D5012101FA03F39360AEE78C
:10B9B00022681946106808238B40184200D0936013
:10B9C0001068042303FA01F10142DCD09160F8BD54
:10B9D000012285F86420DBB283F3118895F8643086
:10B9E000002BBAD095F87C30002BB6D195F87100B9
:10B9F00010F074FD2A6E938923F008031B040121C3
:10BA00001B0C938185F87C100028A6D02021FFF71D
:10BA1000D7FCA2E7012303FA02F2CA6077E72E6996
:10BA2000301A80B25060A96289E700BF70B50C4639
:10BA300082B015460646002839D0036803F13F431B
:10BA400003F57E039B0A1B4A134493F88C0768F0A6
:10BA5000B9FEB2880092B2FA82F304F003028DF8C4
:10BA60000420C4F3810230688DF80520C3F11F0360
:10BA7000C4F30012C4F341148DF80740C3F3CC049F
:10BA800000EB840403F007038DF806209B00226A74
:10BA90000F269D4006FA03F322EA03032362226A7B
:10BAA0001543694625625DF009FC02B070BD4FF098
:10BAB000FF33C8E714AE070800B1B7E7704700BF0F
:10BAC0002DE9F043774D05EB001683B0D6F84C3ED8
:10BAD000002B00F0938004464FEA001896F8540EAD
:10BAE00068F070FE96F8543E590903F01F020329CE
:10BAF0004FF0010303FA02F300F09880042900F0EC
:10BB0000858002297DD005EB0803013493F8500E9F
:10BB100010F0E4FCE4B2814610B112238371C471C9
:10BB200005EB080393F8510E10F0D8FC074610B14E
:10BB30001323C471837105EB080393F8520E10F0C0
:10BB4000CDFC064610B11423C471837145444846A8
:10BB500095F8532E01924A21FFF7AEFF019A38461D
:10BB60002A21FFF7A9FF019A0A213046FFF7A4FF17
:10BB7000D5F84C2E4C4B9A425DD04C4B9A424AD051
:10BB80004B4B9A4262D04B4B9A426AD04A4B9A42F4
:10BB900072D04A4B9A427AD049499088B1F84A44C7
:10BBA000B1F84834B1F852542343B1F84C4423431C
:10BBB000B1F84E4420F003002343B1F85044000490
:10BBC000000C2343B1F8544490802B431088234346
:10BBD000B1F85644B1F8581400F4415023430343DC
:10BBE0009BB21380938B23F400631B041B0C938381
:10BBF000118213889BB243F04003138003B0BDE869
:10BC0000F083304A516A0B4353627CE72D4A116935
:10BC10000B43136177E703F50033196A41F4804160
:10BC20001962196A21F480411962B5E7254A116A3F
:10BC30000B43136267E703F58433596A41F480517B
:10BC40005962596A21F480515962A5E703F5FE3320
:10BC5000196A41F400411962196A21F4004119621C
:10BC60009AE703F58233596A41F400515962596ADF
:10BC700021F4005159628FE703F56843596A41F492
:10BC800080115962596A21F48011596284E703F5E1
:10BC90006443596A41F400115962596A21F4001150
:10BCA000596279E7F01E0020003001400038004062
:10BCB000003C00400034014000500140005401406D
:10BCC0008801002000380240431C00F074812DE9F7
:10BCD000F04F00EB8003BE4FDA0087B057F80290B8
:10BCE00081000546019107EBC303B9F1000F05D0B0
:10BCF0009C68002C00F02F81A17911B107B0BDE83C
:10BD0000F08FD3F80CA0BAF1000F00F0A2819AF8DE
:10BD10000630002BF2D11832B818D9F80480BB5085
:10BD2000691CC0E90133C3601523A371C9B216238E
:10BD3000E1718AF807108AF8063099F8180068F05F
:10BD400041FDB8F804302268A18823F440731B0435
:10BD50001B0CA8F80430DAF800301183BAF804207C
:10BD60001A8311212046FFF72BFB11215046FFF7C4
:10BD700027FB09264FF0330B05E0BBF1010B00F068
:10BD8000158116F0AFFB0A20002CF6D02268A1889E
:10BD900013691942F1D05183052016F0A3FB2368E3
:10BDA000A2881A83052016F09DFB013EE2D13326BE
:10BDB00004E0013E00F0308116F094FB0A20002CD4
:10BDC000F7D02368A28819690A42F2D05A83052065
:10BDD00016F088FBBAF1000F00F05D81DAF8003050
:10BDE000BAF804205A83052016F07CFB002C00F0E2
:10BDF00024812368A2881A83052016F073FBDAF8E1
:10BE00000030BAF804201A83052016F06BFB236873
:10BE1000A2881B691A4240F0D580019B2B4407EB96
:10BE2000C3039A7C002A40F0CA801A7C1221204663
:10BE3000FFF7FCFD019B2B4407EBC3039B7C002B0E
:10BE400000F0C4803221BAF1000F07D0019B2B44CF
:10BE500007EBC30350465A7CFFF7E8FD5D4B98455E
:10BE600000F028815C4B984500F02F815B4B984592
:10BE700000F03681019B2B4407EBC3074FF47A7324
:10BE8000BC8A03FB04F4B8F8043023F440731B04A9
:10BE90001B0CA8F80430B8F800309BB243F0010343
:10BEA000A8F80030B8F8045002A85DF051FA25F067
:10BEB0003F0504994A4B2D04A3FB01232D0C45EAB1
:10BEC0009345A8F80450B8F8002022F001021204AB
:10BED000120CA8F80020434A980C9442034600F341
:10BEE00083806200B1FBF2F292B20133042A38BFC0
:10BEF0000422A8F82030A8F81C20B8F800309BB223
:10BF000043F00103A8F80030B8F8003023F481634F
:10BF100023F002031B041B0C4FF4804143F48063A5
:10BF2000A8F80030A8F80810B8F8003023F0800313
:10BF30001B041B0C0022A8F8003099F81A001146C7
:10BF400068F0B4FA002299F81900114607B0BDE86C
:10BF5000F04F68F0ABBAD3F80CA0BAF1000F00F0C4
:10BF6000D4809AF80630002B7FF4C8AE1832BB1884
:10BF7000D9F80480BC50C3E90144DC6016238AF878
:10BF800006306B1C8AF8073099F8180068F01AFC24
:10BF9000B8F80430BAF8042023F440731B041B0CD7
:10BFA000A8F80430DAF800301A83DEE624B9052058
:10BFB00016F098FAF6E67047A1882268EBE61A7C3C
:10BFC000322134E7DAF800301B6926E712213AE71C
:10BFD000F01E00200054004000580040005C00406B
:10BFE00083DE1B43A086010004EB4404B1FBF4F1A3
:10BFF0008AB2C1F30B0109B942F0010250494FF472
:10C00000967300FB03F3A1FB03139B09013342F476
:10C010000042A8F820306EE7002C40F08D8005200B
:10C0200016F060FABAF1000F65D0DAF80030BAF80D
:10C0300004205A83052016F055FA052016F052FA0E
:10C04000DAF80030BAF804201A83052016F04AFA0C
:10C05000F0E61832BB18D9F8048047F802A0C3E90B
:10C0600001AAC3F80CA01523A371431CE37199F82E
:10C07000180068F0A7FBB8F80430A28823F44073D6
:10C080001B041B0CA8F80430236811211A832046D6
:10C09000FFF796F96DE6052016F024FA2368A288CA
:10C0A0001A83052016F01EFA052016F01BFA2368E5
:10C0B0001B69B2E603F5F2331A6A42F400121A62FF
:10C0C0001A6A22F400121A62D4E603F5F0331A6AEF
:10C0D00042F480021A621A6A22F480021A62C9E6E5
:10C0E00003F5EE331A6A42F400021A621A6A22F465
:10C0F00000021A62BEE6052016F0F4F9052016F0DB
:10C10000F1F9052016F0EEF994E61832BB18D9F8CB
:10C11000048047F802A0C3E901AAC3F80CA099F86B
:10C12000180068F04FFBB8F8043023F440731B0488
:10C130001B0CA8F804301CE6A288236846E600BF62
:10C14000D34D62102DE9F843074611F0C5FADFF828
:10C150004C8007EB8709044608EBC90542F20F76CD
:10C1600004E011F0B9FA031BB3420ADC6B7E002B2A
:10C17000F7D108EBC90898F8180080F00100BDE875
:10C18000F883B8F87C3E013338469BB2A8F87C3E71
:10C19000FFF79AFD0020BDE8F88300BFF01E0020E5
:10C1A00010B582B08DF80730431C0CD0022804462D
:10C1B00009DC0DF1070368F077FA20B12046FFF79C
:10C1C000C1FF02B010BD002002B010BD70B500EB81
:10C1D0008003274D05EBC30255F833305C68A38A12
:10C1E00084B09BB20393039B13F4706F1CBF0123B5
:10C1F0001376039B13F4E06F4FEA80060CD1A38AF9
:10C20000304423F4706305EBC0051B041B0C0022B3
:10C21000A3826A7604B070BD238BA38823F4806365
:10C220001B041B0CA380039B9A05E8D423889B0561
:10C23000E5D42388D9050FD52388DA05FCD42388D3
:10C240009BB243F40073238023889B05FCD40190A8
:10C25000FFF73AFD0198D2E723889BB243F40073BD
:10C260002380A38823F440731B041B0CA380C6E720
:10C27000F01E00200020A9E70120A7E70220A5E783
:10C280002DE9F84F2F4F00EB800407EBC404D4F8DE
:10C290000480B8F1000F04D09A46637E03F0FF09D2
:10C2A00023B14FF000094846BDE8F88F0E4693468B
:10C2B000054611F011FA0A9B7600F6B2C4E908337C
:10C2C0000123A67684F81BB084F81D90A37784F828
:10C2D0001CA0637684F81890B8F8042091050646EF
:10C2E00022D4B8F80030DA0512D442F20F7404E018
:10C2F00011F0F2F9831BA3421ADCB8F800309B0559
:10C30000F6D4B8F800309BB243F48073A8F800303C
:10C31000B8F804309BB24FF0010943F44073A8F819
:10C3200004304846BDE8F88F99464846BDE8F88F86
:10C33000B7F87C3E01339BB22846A7F87C3EFFF756
:10C34000C3FCB0E7F01E0020F0B58569296995F8B7
:10C350004C210B78012B97B0044606D0022B01D15B
:10C360000B6A2BB3002017B0F0BD91F90460731C69
:10C37000F8D0022EF6DC04AB297D0093304606236C
:10C38000FFF77EFF0028EDD03046FFF7DBFE0028E8
:10C39000E8D0BDF81010BDF81220BDF8143049BA2D
:10C3A00052BA5BBA0120E1812282638217B0F0BDEC
:10C3B00062F07F028DF80F200DF10F02069201222C
:10C3C000CDE90732CDE90A338DF824308DF83820D5
:10C3D0008DF84C200F9304AA129314930623CDE9F1
:10C3E0000C2300220023CDE9102305F11000EFF308
:10C3F0001186102383F312882B691B6AFBB1089BFB
:10C4000006AF3A461BB1D3691432002BFBD10B6A3D
:10C410006BB1996839B9934209D0196829B15B6841
:10C4200099680029F7D01433F3E7C3E90007F6B29F
:10C4300086F311882A69136A002BFCD1A9E706ABA1
:10C44000F6B20B6286F31188FEF794FAF2E700BFAA
:10C4500070B5016990F84D210B78012B96B0044618
:10C4600006D0022B01D10B6A43B3002016B070BD79
:10C4700091F904506B1CF8D0022DF6DC04AB017D61
:10C48000009328460623FFF7FBFE0028EDD0284640
:10C49000FFF758FE0028E8D0BDF81010BDF81220B4
:10C4A000BDF8143049BA52BA5BBA0120A4F8D010D2
:10C4B000A4F8D220A4F8D43016B070BD62F07F0288
:10C4C0008DF80F200DF10F0206920122CDE90732FF
:10C4D000CDE90A338DF824308DF838208DF84C20C2
:10C4E0000F9304AA129314930623CDE90C23002280
:10C4F0000023CDE910231030EFF31185102383F3CF
:10C50000128823691B6AFBB1089B06AE32461BB139
:10C51000D3691432002BFBD10B6A6BB1996839B91E
:10C52000934209D0196829B15B6899680029F7D04E
:10C530001433F3E7C3E90006EDB285F311882269ED
:10C54000136A002BFCD1A7E706AB0B62EDB285F3B3
:10C550001188FEF70FFAF2E7F8B590F871301C0970
:10C56000013C052C0FD81B4E06EB44020546B2F8E1
:10C57000D40703F00F0340FA03F2D20703D595F86E
:10C580007C70012F01D00120F8BD07FA03F3013BB5
:10C59000184034446CF0B8FC94F8E0270E4C10447A
:10C5A00054F8302004EBC0041069A3881840EBD085
:10C5B000EB6E002285F87C2093F821202046022192
:10C5C000FFF734FA2A6E93899BB243F0080338468A
:10C5D0009381F8BD14AE07083C2A0020094BD3F81C
:10C5E000802ED3F8841E40F22A40002350604B6214
:10C5F0000B889BB243F001030B80136843F00103E7
:10C6000013607047F01E00201D4B1E48196C1E4A17
:10C6100010B441F080510124196404625321FF24B5
:10C62000CA205462506251625B6FDB0085B017D440
:10C6300016480423002102910290029A1A440292A1
:10C64000029A04331C2B1160F5D103910390039BD4
:10C650000393039B0E4A1A6005B05DF8044B7047C4
:10C660000A4B002201920193019B0193019A084B0E
:10C6700012689A42DCD105B05DF8044B704700BFE8
:10C680000038024000000E420028004050280040C0
:10C690003166654210B5174C84B00139002389B268
:10C6A000A042ADF80C30ADF806308DF80E30029196
:10C6B00013D0114B984210D003F5804398420CD010
:10C6C00003F58063984208D003F58063984204D054
:10C6D0000A4BD3F8B0375B0802E0084BD3F8B03709
:10C6E000B3FBF2F201A9013AADF804205DF09AF82B
:10C6F00004B010BD0004014000000140F01E002005
:10C7000030B50446006EA268838923F400531B04ED
:10C710001B0C8381637995B013F0040F4FF0000177
:10C72000019214BF4FF480520A46ADF808201A0354
:10C730001B0203F48063ADF80C302379ADF80E10C2
:10C7400002F40052ADF80A20DA0744BF0422ADF823
:10C750000E209B07ADF8101005D5BDF80E3043F044
:10C760000803ADF80E3001A95DF06EF96279236E11
:10C77000D50700F18B8012F0080F9A8A48D092B248
:10C7800042F008029A829A8992B242F400529A8147
:10C790002279D00732D5E06B002800F08980002391
:10C7A000E26D0893CDE90C33CDE91033CDE91233B6
:10C7B0004FF480750A936369E1680E9506920793BA
:10C7C000626C05924FF480634FF480350B930991AE
:10C7D0000F955CF00BFE05A9E06B5CF09DFEE26B33
:10C7E000216E136843F0010313608B8A9BB243F000
:10C7F00040038B82536822799BB2636591070DD405
:10C80000226E93899BB243F40053938115B030BDDF
:10C8100022F008021204120C9A82B4E7206C00285D
:10C8200052D02369A26D0993A36CCDE90532402350
:10C8300000254FF4803108934FF480630B930F91E0
:10C84000CDE90C55CDE91055CDE9125507950A955E
:10C850000E955CF0CBFD206C05A95CF05DFE236CB1
:10C86000226E586940F080005861186840F0160048
:10C8700018605D60938A9BB243F0800302F10C0163
:10C8800093820B6843F040030B60BAE71E498B426A
:10C8900024D0A1F54C418B421ED001F580618B4222
:10C8A0001ED102200121FDF734FE6279236E62E77A
:10C8B0004FF6DF711980D96841F02001D960D9683D
:10C8C00041F01001D96099E7226ED36843F08003EC
:10C8D00002F10C01D360D4E70120E3E70020E1E797
:10C8E00001F580618B420AD001F580618B4208D04E
:10C8F00001F544418B427FF43EAF0520D2E703208F
:10C90000D0E70420CEE700BF001001402DE9F84F2A
:10C910004D4C04EB8004D4F82C4A002C7DD0E56EFD
:10C92000002D76D01F46EB6A6361AB6AA3616B8E04
:10C93000E3602B8E23616B682366444B2360444B7A
:10C94000A160A36606462046904610F08BF994F845
:10C9500071000FF0C3FD824695F8200094F870B086
:10C96000A14600284ED102213A0784F87C1036D423
:10C9700018F0020F10D0BAF1000F0DD00B238AF877
:10C980000630731C8AF807303B0648D495F82120FE
:10C9900050462221FFF74AF818F0010F04D1E26B4C
:10C9A0009AB14846BDE8F88F58460FF097FD002829
:10C9B000F5D00C220136C671827195F82120222112
:10C9C000FFF734F8E26B002AEBD195F8241095F8C4
:10C9D0002200890967F06AFD4846BDE8F88F0136F4
:10C9E000F6B2BAF1000FDAD00B2317F0500F8AF825
:10C9F00007608AF8063008D095F821205046FFF7E6
:10CA000015F8CCE767F0DEFEADE795F8212012219E
:10CA1000F4E7A9464846BDE8F88FA146C1E794F877
:10CA200071000FF05BFD226E938923F008031B0455
:10CA300001211B0C938184F87C100028ACD02021AC
:10CA4000FEF7BEFCA8E700BF04000010FCB5070815
:10CA500059C50008BFF34F8F0549064BCA6802F459
:10CA6000E0621343CB60BFF34F8F00BFFDE700BF11
:10CA700000ED00E00400FA0508B572B6FFF7EAFF22
:10CA800000B583B00D49002200920091009B0C3349
:10CA90000093009B1B68012B02D003B05DF804FBE0
:10CAA00001920191019B06490C330193019B1A608D
:10CAB0000B6883F308884B689847FEE750280040CE
:10CAC0000000FF1F38B5FFF79FFDFFF7D9FF0120DA
:10CAD0005CF0B4FD714A936823F00303936093689C
:10CAE00013F00C0FFBD113686C49002842D143F0BE
:10CAF0000103136041F288330A6895075DD4013B56
:10CB0000FAD1674C674D654B674AEA60596F674ACF
:10CB1000C4F8A01EAA60596B654821F080015963D2
:10CB2000596F41F080715967196B41F4CE01196357
:10CB30005A6B5A639A6B9A631A6C02431A64596C63
:10CB40005C4A0A435A6410F07FFDD4F8B0375A4A61
:10CB5000A2FB03239B09013BB3F1807F09D24FF075
:10CB6000E022F02053610021072385F82300916122
:10CB7000136138BD43F4803313600A68940341F2B3
:10CB8000883304D4013BBCD00A689403FAD5444CE2
:10CB90004A4A4B4BB0FBF3F3B0FBF2F0B3EB400F60
:10CBA00018BF18464FF48002B3FBF0F3C4F89C2E74
:10CBB000C4F8880EC4F88C3E09E0394C00210822E4
:10CBC0000223C4F89C1EC4F8882EC4F88C3E0220B0
:10CBD0005CF034FD03280FD83A4BD4F88C1E03EBDD
:10CBE000C0008588C2884388C4F8945EB3FBF1F323
:10CBF000C4F8982EC4F8903E284B33491A6C42F082
:10CC000080521A640A6842F440420A609A689A6044
:10CC10009A6842F400429A609A6842F4A0529A607C
:10CC2000D4F89C0ED4F8882ED4F8901E024342EA21
:10CC30008112D4F8941ED4F8980E490842EA006292
:10CC4000013942EA01425A601A6842F080721A6061
:10CC50001A689201FCD51D4A40F20571116099686D
:10CC600021F003019960996841F00201A2F5806208
:10CC70009960936803F00C03082BFAD1D4F88C0E5A
:10CC80001349D823B3FBF0F39B0143F00053012079
:10CC9000C2F884308866FBF799FE33E7003802401B
:10CCA000F01E002000ED00E00005FA050000002065
:10CCB000FFC9FE36335F0700D34D621080841E002B
:10CCC00040420F002CB6070800700040003C0240B4
:10CCD0000000474210B584B000230446ADF80C3084
:10CCE0000068ADF806308DF80E3003F1804301394D
:10CCF00003F5823389B29842029114D0A3F5806380
:10CD0000984210D003F5804398420CD003F580631D
:10CD1000984208D003F58063984204D0204BD3F8A2
:10CD2000B0375B0802E01E4BD3F8B037B3FBF2F329
:10CD300001A9013BADF804305CF074FD2168194A8B
:10CD40000B8819489BB243F001030B80002301E0DC
:10CD500050F83320914208D001330E2BF8D1002037
:10CD600004B0BDE81040FBF78FBD104A02EBC303CF
:10CD700093F83D482046FBF787FD1B2C05D1192071
:10CD800004B0BDE81040FBF77FBD2E2C08BF2C205F
:10CD900004D104B0BDE81040FBF776BD04B010BD6F
:10CDA000F01E0020000001404CB6070814AE070832
:10CDB00010B5EFF3118E502383F3128803681BB371
:10CDC00084464CF8243F043300F1140252F8044B1B
:10CDD0001CB11C6052F8043C04339445F6D1002287
:10CDE0001A605FFA8EF383F31188436A2BB18B8943
:10CDF0009BB243F001038B8110BD8B8923F00103AB
:10CE00001B041B0C8B8110BD00F1240C6346DBE777
:10CE100070B50568AB0AA3F58013522B25D81F4CBB
:10CE2000234493F8F4330D2B1FD840798608E9B1D9
:10CE300003EB830C03EB4C0CB5F80CE08408B44412
:10CE40000220174EA04040EA0E0006EB8C0480B290
:10CE5000C4F84815C4F85825A881124A2C20294640
:10CE600000FB0320BDE87040A2E770BDAC8903EB76
:10CE7000830C304603EB4C0C4FF0020EB444A4B2CA
:10CE8000074E0EFA00F024EA0000A88106EB8C00A1
:10CE9000C0F84815C0F85825DFE700BF14AE0708F2
:10CEA000F01E00203424002001490248FCF7AAB8F3
:10CEB000342400200000014010B5064C064804F25E
:10CEC0004451FCF79FF804F5DA610448BDE81040CE
:10CED000FCF798B8F01E002000000140004401401B
:10CEE00002494FF08040FCF78DB800BF602400205D
:10CEF00001490248FCF786B88C2400200004004059
:10CF000001490248FCF77EB8B82400200008004020
:10CF100001490248FCF776B8E4240020000C0040E8
:10CF200001490248FCF76EB8682500200004014062
:10CF300010B5064C064804F5CF61FCF763F804F21F
:10CF400054710448BDE81040FCF75CB8F01E0020A6
:10CF500000040140001C004001490248FCF752B89F
:10CF6000942500200040014001490248FCF74AB8DE
:10CF7000EC2500200048014001490248FCF742B876
:10CF8000182600200018004001490248FCF73AB872
:10CF90007026002000200040F8B5164D1648174FA7
:10CFA00000214FF41A726DF0D0FE05F688064FF09E
:10CFB0008041A5F18C043A46002301E054F8332067
:10CFC00091420BD001330E2BF8D100201C3567F0B5
:10CFD000F9FBB5420CD055F81C1CECE7084A02EBF3
:10CFE000C3031C3593F83C0867F0ECFBB542F2D163
:10CFF000F8BD00BFD8B60708342400200000014067
:10D0000014AE070810B50C2937D8DFE801F09736C1
:10D01000363666363636373636360700038C548851
:10D02000B2F80CE023F480531B041B0C0384038C24
:10D03000B0F804C0818B21F4E6414EEA040E0904E5
:10D04000148823F40053090C41EA04211B04754C95
:10D050001B0C43EA0E33A0421FFA8CFC9BB289B230
:10D0600000F0AE8004F58064A04200F0A9809268D0
:10D07000A0F804C081830264038410BD038CB2F85D
:10D080000CC0548823F480731B041B0C0384038C92
:10D09000B0F804E0818B23F400731B044CEA040C09
:10D0A00021F073011B0C43EA0C230904B2F800C001
:10D0B000090C41EA0C0C5B4988421FFA8EFE9BB2B8
:10D0C00068D001F58061884264D09268A0F804E0DD
:10D0D000A0F81CC0C263038410BD038CB2F80CC05E
:10D0E000548823F010031B041B0C0384038CB0F83A
:10D0F00004E0018B23F020031B044CEA040C21F410
:10D10000E6411B0C43EA0C130904B2F800C0090CF9
:10D1100041EA0C211FFA81FC424988421FFA8EFE27
:10D120009BB269D001F58061884265D09268A0F811
:10D1300004E0A0F818C08263038410BD038C5488F7
:10D14000B2F80CE023F001031B041B0C0384038CD6
:10D15000B0F804C0018B21F073014EEA040E0904FB
:10D16000148823F00203090C1B0421432D4C1B0CD3
:10D1700043EA0E03A0421FFA8CFC9BB228D004F5B0
:10D180008064A04224D09268A0F804C00183426366
:10D19000038410BDD189548A23F4006343EA01213A
:10D1A000138A2EF4405E23434EEA031E94884FF602
:10D1B000FF330B4043EA04231FFA8EFE9BB284E741
:10D1C000148A2CF4804C4CEA841C1FFA8CFC4EE729
:10D1D000D489B2F810E023F008032343548A2CF4D6
:10D1E000407C4EEA040E948823F004034CEA0E0CB3
:10D1F0001FFA8CFC2343C6E7D189548A23F08003AD
:10D2000043EA0111138A2EF4406E23434EEA830E43
:10D2100094884FF6BF730B4043EA04131FFA8EFE47
:10D220009BB283E7000001402DE9F04FA24BDFF8ED
:10D23000A49293F8B63EA14EA14F8FB0CDE901392B
:10D24000013BDBB200930025DFF88CB2DFF88CA243
:10D250005B46D3469A464FEA9A23A3F58013522B96
:10D260004CD8334493F8F4330D2B47D8FC56019B2C
:10D27000012B40F00181012C35D14FF000084146CF
:10D28000204615F0A9FE15F035FF037813B1542B95
:10D2900040F0F98008F104081FFA88F8B8F1100F7F
:10D2A000EDD14FF0000E8DB3494600200CE0334421
:10D2B00093F8F4330D2B0ED8FB56A3420ED0013059
:10D2C000A84201F580711EDA8A6813689B0AA3F5EB
:10D2D0008013522BEBD90023A342F0D153799BF852
:10D2E00005209A42EBD1774B5B454BD05BF81CAFE6
:10D2F0004FEA9A23A3F58013522BB2D9009B012B3E
:10D30000F1D90024B9E7BEF1000FECD15846FBF784
:10D3100039F8C3B2022B9BF805C000F23483431CDA
:10D320005BB203EB43034FEA830E644B664903F59C
:10D33000727004E0984200F0268353F82C1F514588
:10D34000F8D11A796245F5D153F80E40002CF1D08E
:10D350005E4800234268A24203F1010300F0898085
:10D36000102B00F12400F5D14FF0FF33584A03EBA6
:10D37000C30302EB830393F82432002BB3D1029B47
:10D38000C3F808B0029B013503F58073042D0293A6
:10D390007FF45AAFDFF848B10BF59E730027ABF569
:10D3A000816A9846DAF8243ABB425FDDDBF80C501C
:10D3B000002D5BD09BF81030A88802932B68DAF818
:10D3C0000460019303F13F41B0FA80F301F57E015F
:10D3D0000393002EC3F11F034FEA9121009340F302
:10D3E0008480002302E00133B3427BD01C0259F851
:10D3F00004208A42F7D14C440099029B8BF81030EC
:10D4000003260137CBF80410CBF80C50CBF81840AA
:10D41000AE71EF71636CE26C0D4649008E401E43A5
:10D42000012303FA01F111439AF800206664E164D4
:10D430007AB303FA05F11A46236D0B432365019B6A
:10D4400089B21883D4F8A000FAF7D8FF2046FBF77A
:10D450002BF90123082F8BF81C308BF81D3088F82E
:10D4600011300BF1200B08F118089BD10FB0BDE86B
:10D47000F08FDBB2013B79E7022B7FF4FEAE082C84
:10D480003FF4FBAE2FE74FF0010E002D7FF40CAF01
:10D4900029E70399C1F12F05009903FA05F58B409F
:10D4A00099B2236D2B432365019B5883D4F8A000C8
:10D4B000FAF7A4FFCAE700BFF01E002014AE070869
:10D4C000A44A080824C00708000001409003002077
:10D4D000880100200C0000100004014044BF070830
:10D4E0000C040010032B00F31F820AEB0623320208
:10D4F00018690492002800F03F8299600131CAB295
:10D5000083F805210692542283F80421013602682B
:10D5100005924479CAF80460FAF734FF934AC3B21B
:10D52000022B92F8CDEE844600F22D82461C76B294
:10D5300006EB46068E498F48059AB600002305E0A3
:10D540000133172B00F01F8251F82C0F8242F7D1C4
:10D550000879A042F4D188590028F1D02C2101FB90
:10D5600003F30CEB4C0C03EB8C0C814B63441969FB
:10D57000049B5344C3E906017F4B00211E461C4611
:10D580006368984216D00131102904F12404F7D1C0
:10D590007A4B93F80022002A00F0E7817849794A13
:10D5A000794BCAF8681ACAF8602ACAF8703A0FB0FC
:10D5B000BDE8F08F01F1010C5FFA8CFC6F4B079610
:10D5C0000CF1FF3C0CEBCC0C03EB8C0C9CF82432E4
:10D5D0000593002BE2D1049E069B8CF82532F311B3
:10D5E00003EB262000EB001368488C2400EB83003B
:10D5F0003112674B04FB01F103EB41010AEB060317
:10D60000C3E93C145421019E8CF824123321C3F841
:10D61000AC10DE60C3F8A8005E4B04999A4209EB97
:10D62000010400F07681534B9A4200F0728103F5B9
:10D6300080439A4200F06D8103F580639A4200F0C6
:10D64000688103F580639A4200F06381474BD3F809
:10D65000B007BEF1060F4FEA500000F061814E4B5B
:10D660004E49BEF1070F18BF9C464D4B08BF8C4674
:10D670004C4918BF1946B0FBF1F1B0FBFCFC104659
:10D68000049A01390AEB020389B20CF1FF3CA3F8BA
:10D69000B0C0A3F868104FF000060193A165002305
:10D6A00002F154014944A4F85C6063655CF0BAF887
:10D6B000019B3D4A1B690193186803889BB243F0A4
:10D6C00080030380038809920A210B914FF4807232
:10D6D000022123F00103CDE90C121B04ADF82860F0
:10D6E0001B0C019E0380717909AAFFF78BFC30792E
:10D6F000002840F02281049B079E0AEB03020023CE
:10D700001069D2F818C001680A8892B242F001028A
:10D710000A807268944503F1010300F00A81102B1E
:10D7200006F12406F5D14FF0FF33144A1F4E03EBE8
:10D73000C30302EB83031E4AD3F80832B3420CBF83
:10D740004FF400134FF48003166B33431363427995
:10D7500018480C2A9BBF184B03EB42030026B3F872
:10D760003461049B53449E8200232EE0F01E00206F
:10D7700014AE07080000014090030020880100203B
:10D780005D8801085988010865880108C02D0020BE
:10D79000F03000200004014044950800105522009C
:10D7A000D0DD060040771B006000010000600240F1
:10D7B00000380240140600100CBF0708914200F028
:10D7C000E0800133042B00F0E18050F83320002A80
:10D7D000F4D1DAF80C260132CAF80C260AEBC3029F
:10D7E000DB00C2F8101603446A499A88059816436C
:10D7F0009E80049B0AEB030690222346FDF7E4FC7F
:10D80000B0690268002342F010020260C4E92533C7
:10D81000A367C4F88830C4F89C30F26962664FF49C
:10D820008062E26704214FF40032C4E923214022E0
:10D830002267D6F8AC206267F268049B1832A266B1
:10D840004FF48052C4F88020D6F8A820E26603F195
:10D8500064014FF480424944C4F884205BF05CFECC
:10D86000B069049BD0F800E0C4F81CE0D0F814E0E4
:10D87000C4F820E0D0F804E0C4F824E003F1AC01DF
:10D88000D0F808E0C4F828E00023D0F80CE0C4F891
:10D890002CE0C4E93733C4F8B830C4F8C030C4F859
:10D8A000D030C4F8E430F369C4F8AC304FF480638E
:10D8B000C4F8C4304FF4403C0423C4E935C3D6F85F
:10D8C000F430C4F8BC30F3681033C4F8B0304FF40F
:10D8D0000063C4F8C830D6F8F030C4F8B4304FF460
:10D8E0008042C4F8CC2049445BF016FEB369A88896
:10D8F0001A6822635A6962635A68A2639A68E2638B
:10D90000DA6822641A6842F010021A602B680193E8
:10D9100072E5214BBEF1060FD3F8B0077FF49FAE3E
:10D92000DFF87CC01D49A6E61B4A032382F8CC3EE3
:10D9300034E6DBB20593013BF7E60EF0CFFD06902F
:10D9400038B1019B0221DA79FEF770F8069B542268
:10D95000DA80019B1A68B2F844306FEA43436FEAF9
:10D9600053439BB2A2F84430C5E6542283F8002208
:10D97000069A83F8012211E6074A022382F8CC3E78
:10D980000CE6DB002FE700235B68FFDE00239B88AB
:10D99000FFDE00BF45840008F01E0020A0BB0D0084
:10D9A000882A11000C2911D8DFE801F0231010108B
:10D9B00019101010111010100700838B23F400634E
:10D9C0001B041B0C43EA022292B282837047838BB2
:10D9D00023F008031B041B0C1A4382837047038B3C
:10D9E00023F400631B041B0C43EA022292B202835D
:10D9F0007047038B23F008031B041B0C1A4302839C
:10DA0000704700BF2DE9F04FDFF870B29BF800407F
:10DA100087B024B90124204607B0BDE8F08F934EAB
:10DA2000D6F874580FF084FE9BF8B43A0390002B9C
:10DA300000F058828E4AA2FB05328E4B5209A3FB9E
:10DA40000213DB0803EB8303A2EB4303DAB2049275
:10DA50000BF23C6202EB830300930BF61C1306F1FE
:10DA6000DC0401934FF00009924635E03B680293D5
:10DA7000009B5C330093019B3046143301935BF0B1
:10DA8000B5FC7A4B02988C2202FB0933002583F8FF
:10DA9000D05079792A46FFF785FF22467979FFF73A
:10DAA000B1FA79790822FFF77DFF402344F83C3C26
:10DAB000A4F1480130465BF02FFD336843F01003BA
:10DAC00033609BF8B43A09F1010999450AF15C0AFF
:10DAD00004F18C0480F2D480DBF83836039AD31A30
:10DAE00004D454F8082C9342C0F2AB815F4B54F835
:10DAF000587C266A8C2202FB093393F8D030002B25
:10DB0000B4D03968736834F8542C02911FFA83FE3C
:10DB10008B89CEF1160E9BB223EA0203BEF1070FEA
:10DB20008B81A5D9DBF824390133CBF82439A36ADA
:10DB300005939C4600225CF8045B012190461BE0A3
:10DB4000DCF80000B8F1140FA0EB05031DDC13F1A5
:10DB5000080548BF03F117052B1108EB25180546EA
:10DB6000581E013102FA03F3012282408E4542EA37
:10DB700003020CF1040C08D38E45E1D8C8F115035B
:10DB8000DCF800504FF01508EAE7B8F1150F60D146
:10DB90003948C2F38423C2F3441100EB830300EB42
:10DBA0008101D3F85031D1F850111B0243EA01131F
:10DBB00002F01F0100EB8101C2F3C43200EB8202CC
:10DBC000D1F85011D2F850210B4343EA023383EAD3
:10DBD000132282EA121202F00F020F2A39D1C3F384
:10DBE0000F134FF6FF72934233D0B3F5606F00F01E
:10DBF0003681019A93819AF85820049DAA4211D047
:10DC00000098DAF800208168521ACAF80020016BE7
:10DC1000DAF80420521ACAF8042000228260026353
:10DC20008AF85850DAF8002000990132CAF800202A
:10DC30008A6801328A604FF6FF7293427FF418AF10
:10DC4000DAF804300133CAF804300B6B01330B638C
:10DC50000EE7DBF820390133CBF82039B9F1000F9A
:10DC600000F0E5804FF6FF73C5E700BFF01E00200F
:10DC70001F85EB51CDCCCCCC0CBF070804000010A5
:10DC800001228BF8202ACBF83856002B3FF4C2AE85
:10DC9000974890F88C10890700F1BE80D0F8841066
:10DCA000086849798A40018C92B289B221EA02015E
:10DCB0000184018C89B20A43012B02843FF4AAAE8D
:10DCC0008B4991F81821970700F1C080D1F81021F5
:10DCD00010685479018C012289B2A24092B221EAE3
:10DCE00002010184018C89B20A43022B02843FF4B1
:10DCF00091AE7F4991F8A421960700F1C180D1F837
:10DD00009C2110685479018C012289B2A24092B200
:10DD100021EA02010184018C89B20A43032B0284A7
:10DD20003FF478AE724991F83022950700F1B18046
:10DD3000D1F8282210685479018C012289B2A240BE
:10DD400092B221EA02010184018C89B20A43042BB8
:10DD500002843FF45FAE664991F8BC22940700F15B
:10DD6000A180D1F8B42210685479018C012289B2C3
:10DD7000A24092B221EA02010184018C89B20A43D5
:10DD8000052B02843FF446AE594991F84823900789
:10DD900000F19180D1F8402310685479018C012260
:10DDA00089B2A24092B221EA02010184018C89B2B7
:10DDB0000A43062B02843FF42DAE4D4991F8D4233B
:10DDC000920700F18180D1F8CC2310685479018C3E
:10DDD000012289B2A24092B221EA02010184018C9F
:10DDE00089B20A43082B02847FF414AE404A92F8A9
:10DDF00060349B0771D5D2F85824042311685079F8
:10DE00000A8C83409BB292B222EA03020A840A8CF3
:10DE100092B213430B84FDE5354AD2F88420106892
:10DE20005479018C0422A24089B292B23EE705994E
:10DE3000304858226CF026FF3B6802934FF6FF7380
:10DE4000D9E60024204607B0BDE8F08F284AD2F872
:10DE5000102110685479018C042289B23DE72449CD
:10DE600091F8DD2402EB420201EBC2024A4492F82F
:10DE7000ED240D2A7FF4BDAE019980228A77BAE69F
:10DE80001B4AD2F89C2110685479018C042289B273
:10DE90003CE7174AD2F8282210685479018C0422F2
:10DEA00089B24CE7124AD2F8B42210685479018C36
:10DEB000042289B25CE70E4AD2F8402310685479F4
:10DEC000018C042289B26CE7094AD2F8CC2310688D
:10DED0005479018C042289B27CE7054BD3F858248D
:10DEE00001238BE701228BF8202ACBF8383692E504
:10DEF000F01E0020CC0900102DE9F04F002299B04F
:10DF00002F21074615F04CF900B3BE4ED0F8008023
:10DF1000C6F8848E0446FDF75BF80246B0B1D0F82F
:10DF200004C0C6F880CEBCF1000F0FD0B64D002360
:10DF300029464868844501F1240103F101030FD00B
:10DF4000102BF6D1B14B93F8000218B1002019B094
:10DF5000BDE8F08F2F2283F8002283F80102F6E754
:10DF6000DBB2DFF8A892013B03EBC30309EB8303A9
:10DF700093F824A2BAF1000FE8D138469768DFF889
:10DF8000C0B22F22A3F824220EF0A8FA2F220346B3
:10DF9000CBF86C0520B1DA80E2792A21FDF746FD45
:10DFA0009B4A9C49002301E051F83320904500F042
:10DFB000228101330E2BF7D1002066F003FCD6F846
:10DFC000840E954A038823F001031B041B0C904226
:10DFD000038000F070818E4B984216D003F5804389
:10DFE000984212D003F5806398420ED003F5806307
:10DFF0009842D6F8B0270AD08849B1EB520F4FEAC1
:10E00000520340F2528100210AE0D6F8B027834B38
:10E010009A4280F017814FF0010C0021B2FBFCF313
:10E020007F4AADF804101B0A7E49A2FB03231A099C
:10E03000A1FB021252084FF000081B09ABF86A2539
:10E0400001A952000293ABF86825ADF80C80ADF839
:10E0500006808DF80E805BF0E5FBCDE90688CDF8F3
:10E060002080A379ADF81480602204929A0740F1D1
:10E07000AF80DB0003F00803ADF81E300423ADF8D9
:10E080001430D6F8840E617904AAFEF7BBFF6179DB
:10E090000822FFF787FCB0F84430D6F8808E6FEA8C
:10E0A00043436FEA53439BB2A0F8443003889BB2CA
:10E0B00043F080030380A3796179028C9B074CBFF6
:10E0C000042301238B409BB292B222EA0302028412
:10E0D000028C92B21343038403889BB243F0010382
:10E0E00003802A4600235168884502F1240203F187
:10E0F00001037DD0102BF6D14FF0FF3303EBC303A8
:10E1000009EB8309484AD9F8083248498B420CBFC9
:10E110004FF400134FF48003116B0B431363002380
:10E120006A68904505F1240503F101035DD0102BC9
:10E13000F6D13F49602200235046FDF745F840469E
:10E140005BF054F9D6F8800E036823F00103002534
:10E1500003605BF04BF9CDE91455CDE91655D6F8BF
:10E16000843E0E9512956279D6F8800E0997343365
:10E170001344304A0B9240220A930C924FF480438E
:10E180004FF48052CDE9102340F22A414FF440333E
:10E190000D91139309A94FF480630F935BF0BCF9C1
:10E1A0006379D6F8841E0C2B04D8234A02EB430370
:10E1B000B3F834518B89D6F8802E9BB21D438D81E4
:10E1C0001368012043F01003136019B0BDE8F08F0D
:10E1D0005B0003F00203ADF81C300123ADF81230F0
:10E1E0004FF48073ADF820304BE75FFA83FAA0E775
:10E1F000DBB2013B82E7114A02EBC30393F83C0810
:10E20000DBE600BFF01E0020900300208801002004
:10E21000000001404CB6070800040140006CDC021D
:10E22000598B4F01ABAAAAAA0038024000600240F5
:10E23000FD860008D88400200CBF070814AE07082C
:10E24000E82F0020254B98420BD003F580439842DD
:10E2500007D003F58063984203D003F580639842AA
:10E2600022D102F1B7731E4903F55853A1FB0313E2
:10E270009B0D013B99B2194B984201F1010C3FF4FF
:10E28000CDAE03F5804398423FF4C8AE03F58063FA
:10E2900098423FF4C3AE03F5806398423FF4BEAEAC
:10E2A0005308B3FBFCF3BBE6530803F1B7730C4907
:10E2B00003F55853DAE7D6F8B0270A4B9A42FFF431
:10E2C000AAAE074902F1B77303F55853A1FB031334
:10E2D0009B0D013B99B201F1010C9FE6000001404A
:10E2E000819F5E16006CDC02F0B50C4689B03C499B
:10E2F000BDF838609DF83C70013B054620689BB234
:10E30000049388424FF00003ADF81430ADF80E309E
:10E310008DF8163013D0334B984210D003F580435C
:10E3200098420CD003F58063984208D003F58063CF
:10E33000984204D02C4BD3F8B0375B0802E02A4B4C
:10E34000D3F8B037B3FBF2F203A9013AADF80C20D1
:10E350005BF068FA20686179A3790FB183F001035B
:10E360000022CDE90622ADF81020602203929A0720
:10E3700029D5DB0003F00803ADF81A300423ADF80B
:10E38000103003AA01910596FEF73CFE0199082280
:10E39000FFF708FB2268B2F844306FEA43436FEAA4
:10E3A00053439BB2A2F84430138811469BB243F00A
:10E3B000010321F8343B63796A60C81800222860A1
:10E3C000CA5009B0F0BD5B0003F00203ADF818308D
:10E3D0000123ADF80E304FF48073ADF81C30D0E758
:10E3E0000004014000000140F01E002010B4104A5B
:10E3F00092F8AC3703F0FF01002BF9D10D4B0E4C16
:10E40000D3F8700554F82C4CB3F884354FF0010C58
:10E4100082F8ACC74360616223889BB243EA0C0375
:10E42000238003685DF8044B43EA0C0303607047E4
:10E43000F01E0020E82F0020E04000201648174A78
:10E44000174938B5174C184D121A6CF01BFCD4F84C
:10E450008820164B164842F47002C4F888201A68C7
:10E46000002142F001021A6099601A6822F0847259
:10E4700022F480321A6058601A6822F480221A60EE
:10E480000C4AD960521B28460B496CF0FBFBA56077
:10E49000BDE83840FAF79ABA0000001004000010F6
:10E4A000C70B090800ED00E0000000200038024022
:10E4B0001030002488010020000000080548D0F832
:10E4C000303823B1DB6A13B100F503601847024806
:10E4D000704700BFF01E0020DCC0070870B50F4C6D
:10E4E0000023A4469CF800E086450CF1060C10D0F1
:10E4F0000133062BF6D10A4E56F8045C052D07D0E1
:10E5000003FB0543013546F8045C187059809A8076
:10E5100070BD062505FB0343F7E700BFB8400020A8
:10E52000E0400020002370B49C46224C224D04E0C1
:10E53000D2F8E4419C46002C37D00133DBB203EB28
:10E540004302A14205EB8202F2D10CEB4C0C05EB2D
:10E550008C051A4EB5F8E811B5F8EA21B5F8EE4188
:10E56000B5F8EC31164D048206FB01F106FB02F210
:10E57000C5F81019C5F80C2990F8281083802202DC
:10E580004FF48074C4800124002502FB03F3A142F0
:10E5900085748260C360447702D0204670BC7047A7
:10E5A000084B036070BC08467047C0E90244848091
:10E5B0000482F2E71620C2000CBF070840420F0099
:10E5C000F01E0020ECC1070830B58DB000230122F9
:10E5D00004460D46CDE90633CDE90833C221039345
:10E5E0008DF814208DF828200B9301AA02230068CF
:10E5F000049302928DF804108DF8055069F018F814
:10E6000002A920460DF03EF9206869F011F8024B8E
:10E61000C3F85C540DB030BD880100202DE9F041F5
:10E62000DFF84C80D8F80030002B19DD0E4C0F4F6E
:10E6300006460025637F63B1D7F85C34AB422946B8
:10E6400002D0706AFFF7C0FF236820465B689847D6
:10E6500038B1D8F800300135AB4204F13404E9DCBC
:10E660000120BDE8F08100BFAC2600208801002019
:10E67000E04000202DE9F041114E3368002B1BDDF6
:10E68000104D114F8046002402E03368A34213DD91
:10E69000D7F85C34A342214604F1010403D0D8F832
:10E6A0002400FFF791FF2B6828469B689847343574
:10E6B0000028EAD1BDE8F0810120BDE8F08100BF6B
:10E6C000E0400020AC260020880100202DE9F8431E
:10E6D000DFF84880D8F80030002B1ADD0E4DDFF847
:10E6E000409007460E460024D9F85C34A3422146E8
:10E6F00004F1010402D0786AFFF766FF2B68284610
:10E700001B6831469847D8F80030A34205F134051C
:10E71000EADCBDE8F88300BFAC260020E040002022
:10E7200088010020104A70B5D2F85C240F4E0C46C8
:10E730007368B1FBF3F191420D4605D0406AFFF7D3
:10E7400043FF7368B4FBF3F1094803FB1141342321
:10E7500005FB03F3C21800F2BC70D2F8BC271844C2
:10E76000BDE87040D368184788010020E0400020D1
:10E77000F01E00202DE9F0410E4F3B68002B17DD05
:10E780000D4DDFF8388006460024D8F85C34A342EB
:10E79000214604F1010402D0706AFFF715FF2B68CF
:10E7A00028461B6998473B68A34205F13405ECDC19
:10E7B000BDE8F081E0400020AC2600208801002068
:10E7C000134B70B55B68B1FBF3F30D461149124C66
:10E7D000D1F85C64C4F8B837B34282B008D01946A7
:10E7E000406A0192FFF7F0FED4F8B837019A1E464E
:10E7F000342000FB06442946D4F8BC47074D646921
:10E8000000FB0350234602B0BDE87040184700BF2C
:10E81000E040002088010020F01E0020AC260020EF
:10E82000F0B583B0104C0192089A0093FFF7C8FF2F
:10E83000D4F8B807342606FB00F0231804F2BC75A0
:10E84000D3F8BC376A469F6901A928440123B84719
:10E85000D4F8B80706FB00F004442844D4F8BC37C9
:10E86000DB69984703B0F0BDF01E00202DE9F04FA2
:10E8700083B0CDE9000393B3019EDFF878B0DFF8F1
:10E8800078A00D46914601E0F61B2AD0DBF8043053
:10E89000B5FBF3F403FB145806EB0801994294BF4F
:10E8A000C8EB0107C8EB0307DAF85C349C423D442F
:10E8B000214603D0009B586AFFF786FE342303FBF2
:10E8C00004F00A4B0A4A19181044D1F8BC474A46CA
:10E8D000A46A3B464146A047B9440028D4D100234E
:10E8E0000193019803B0BDE8F08F00BFF01E002037
:10E8F000AC260020E04000208801002038B5154CEF
:10E90000A3681B883BB9144D0023237485F828386D
:10E91000C5F8243838BD54F8042C002AF3DD012A48
:10E9200006D0E36859880C4D618201232375EBE71B
:10E93000E1688A8849880132521A9A42F3D1064D19
:10E94000D5F8303800221B69C5F85C2805F503604E
:10E950009847D9E7E0400020F01E00200748D0F893
:10E960002C3813B1064B1B7D0BB100207047D0F83B
:10E97000303800F503605B68184700BFF01E0020C8
:10E98000E040002030B4154A154D92F8283805F1C2
:10E990001804234403602B7C446092F828088342C7
:10E9A00092F8280812D8834204D3002030BCC1E971
:10E9B0000000704792F82828002BC2F180020CBF9B
:10E9C0000120022030BCC1E9002370471B1A00223D
:10E9D000012030BCC1E90032704700BFF01E0020AA
:10E9E000E04000200E4B0F4A93F82818107C93F853
:10E9F0002828904293F828280CD8904238BF93F8E2
:10EA00002828D3F824383ABFC2F1800280180020A9
:10EA100018447047D3F82438801A1844704700BF50
:10EA2000F01E0020E040002030B51B4C1B4D94F838
:10EA3000283894F8281885B005F118021344029379
:10EA40002B7C03928B421CD894F82828934210D236
:10EA500094F828180193C1F180010091CBB90122EB
:10EA600008B93F2905D90023694602A869F062FC6C
:10EA70002B7C94F82808C01AB0FA80F0400905B041
:10EA800030BD94F828180022591A019200910122F1
:10EA9000E6E719440222E3E7F01E0020E0400020F0
:10EAA0002DE9F043164685B0002933D0441E244D8D
:10EAB000244F04EB01084FF0000901E0A04529D0E4
:10EAC000287C14F8013F411C2844C9B203760B0688
:10EAD00048BF002097F8283829744ABF01460846E5
:10EAE00085F810908B4297F828388ABFC3F18003CD
:10EAF000C01AC0183F28E1D997F828388B42DDD0DA
:10EB0000114B93F8C430002BD8D00020FFF78CFFB6
:10EB1000A045D5D1694602A8FFF734FF20B1DDE951
:10EB2000003213443F2B02D805B0BDE8F083024603
:10EB3000334602A869F0FEFB05B0BDE8F08300BFD4
:10EB4000E0400020F01E00208801002030B585B094
:10EB5000694602A8FFF716FF58B9094C04F503658A
:10EB6000D4F8303828465B6898470028F8D005B0BC
:10EB700030BD0246012302A869F0DCFBEDE700BFCF
:10EB8000F01E002070B5114E1546D6F82C380A46F6
:10EB9000411999420E4988BF1D1A097C96F82838F8
:10EBA000994282B0044603D00192FFF7CFFF019A49
:10EBB000D6F8301807480023C6F85C382B468D6A13
:10EBC0002146AC4602B0BDE870406047F01E002010
:10EBD000E0400020202700208C4613460146624674
:10EBE0001846CFE738B52148214C0023C4F82C380B
:10EBF00002461178022902F1060227D00133062BC2
:10EC0000F7D11C4DD4F830380022EA60DBB1DA6A63
:10EC1000CAB119489047EB68A8609BB19A885B8895
:10EC2000D21A436802FB0333C4F82C38FAF780F891
:10EC30002A7C94F828389A42054601D0FFF786FFCF
:10EC4000C4F8245838BD0D4BAB6038BD094DD4F81D
:10EC5000302803EB430300EB4303EB6012B1D26AAD
:10EC6000002AD6D10548A860D8E700BFB8400020E8
:10EC7000F01E0020E040002020270020DCC0070814
:10EC800010B50A4CD4F830385B6A13B104F5036050
:10EC90009847074AD4F8243892685288013B1344B5
:10ECA00052421340C4F8243810BD00BFF01E0020AB
:10ECB000E04000202DE9F043DFF8E090354F93B0BD
:10ECC000FFF71CFEFFF78EFF99F828383A7C9A422E
:10ECD00001D0FFF73BFFD9F82C880025C9F824584C
:10ECE000B8F1000F11D02C4E6C462A463146204612
:10ECF00003F04AF9204669F0DBFB2035014601228A
:10ED00002046FFF7CDFEA845EFD899F828383A7C81
:10ED10009A4201D0FFF71AFFBB689B7B012B32D0D0
:10ED200099F828383A7C9A4201D0FFF70FFF002764
:10ED3000C9F82478B8F1000F28D0DFF85C903D4680
:10ED40006C462A46494609A803F01EF921220021F3
:10ED500020466BF0FAFF202221462846FFF712FFDB
:10ED60002022064609A9204615446CF02BF808B964
:10ED7000202E00D00137A845E3D8B7FA87F0400924
:10ED800013B0BDE8F083FFF77BFFC9E7012013B0A4
:10ED9000BDE8F083E0400020D0490808F01E0020C4
:10EDA000032108B5054608465AF038FC72B6104BE8
:10EDB000D3E9262352EA03010AD100242146042084
:10EDC0005AF02CFC214605205AF028FCFDF742FEA3
:10EDD0000848D0F8744829B24EF6602000FB01F1D3
:10EDE000A41843F100030C1943EBE171E7E700BFFE
:10EDF000E0400020F01E002008B5002103205AF05A
:10EE00000DFC72B6FDF726FE08B5184CD4F8A0200C
:10EE100094F8A6004AB11168938809690B40F8B9C3
:10EE2000003B18BF0123002BF4D1142013F094FDF4
:10EE300000BFD4F8A03063B11A689B88116994F8B8
:10EE4000A6200B4042B9003B18BF01230BB1FFF7CE
:10EE5000D3FFF9F79FFFEBE7B3FA83F35B09F5E71D
:10EE6000B3FA83F35B09002BD4D1DEE7E040002046
:10EE700008B561F04DFC0D490D4B91F8AD0029220C
:10EE80000128A3F8AA2BA3F8B22B01D0012008BDBA
:10EE90000848C1F8B00000F120014C3065F008F9D5
:10EEA000054B002083F8230008BD00BFE040002090
:10EEB000F01E0020E805002000ED00E02DE9F04FF5
:10EEC00041F62C728BB00021AE486BF03EFF04205F
:10EED0005AF0B4FB044605205AF0B0FB50EA040394
:10EEE00040F03F81A84B0393039BA849A548D3F862
:10EEF000F844E4226BF0C6FEA24BC3E90744C3E921
:10EF00001A445C621C67C3F8B440C3F8B840C3F845
:10EF1000BC401F4667F080F9FFF764FE00210846F9
:10EF20000DF06CFBF9F704FFB0F1000A40F38F819C
:10EF3000974D984B984E0193002407F1E4090294F1
:10EF40002746A34605F1B40804E00BF5006BDA454B
:10EF500040F3AE80019AD2F87438C2F87838F9F7E5
:10EF600019FF202241465846FFF70CFE8B4912221A
:10EF700040466BF027FF0028E7D1BB4522D002991D
:10EF8000874BCDF8149001EB410203EB82004A1C41
:10EF900084490292049002F0F7FFDDE90403D9F8F6
:10EFA0001C2043F84C0BC9E908227F4AC9F80C70B1
:10EFB000C9F82820ABEB07070122C9E90477C9F893
:10EFC00008209946039BD3F8F834C9F81C305F46F3
:10EFD0001222A918335D91F8B410994202F101028E
:10EFE0000BD00024202AF4D12037BA4541463846B8
:10EFF00054DBFFF7C7FD0022EBE70134152CF1D1FC
:10F00000D0196A492022FFF7BDFD00230A2209A971
:10F010006648CDF8248003F03FF904900998002356
:10F0200001300A2209A9099003F036F907900998DE
:10F03000002301300A2209A9099003F02DF9069056
:10F040000998002301300A2209A9099003F024F944
:10F050000590099809A9013000230A22099003F0BC
:10F060001BF9074609980023013019460A22099026
:10F0700003F012F9049989B1DDE9063243EA42123C
:10F08000059B7F0147EAC323A1F2BC7143EA6003F9
:10F0900042EA412243EA0243C9F81C30029B642B36
:10F0A00000F0F6805F460BF5006BDA453FF752AF94
:10F0B000029A642A00F0EC80BB4500F0C080384C16
:10F0C00038490C2303FB0244531C1A462046029382
:10F0D00002F05AFFD9F81C30C9F80040ABEB070525
:10F0E000C9E90375C9E90833C9F8145001232E4D45
:10F0F000C9F82850C9F80830029BDC1C4C22214E6C
:10F1000002FB04F43319184600216BF01EFE4C225A
:10F1100000216BF01AFE039A0299D2F8F8240346F4
:10F1200023483051C3E904AAC3E907225A620122E5
:10F1300004319D629A604FEA4A03B3F1805FC0F2E6
:10F140008780104A95682DB913791BB11368002B7D
:10F1500040F0A880002108460BB0BDE8F04F0DF04C
:10F160004DBA4FF47A720023214669F065FE114BC7
:10F1700040F26D11A3FB00231B0C022440F2B2727B
:10F180000D4622E0B85F0020880100201CC207085D
:10F19000E0400020F01E0020144A0808F04908084A
:10F1A000B4410020044A0808D9EB0008944100202B
:10F1B0002C4A080807452EC2013212F00304A3EBC3
:10F1C00001030CBF4FF4B77129468B42F4DA8C4926
:10F1D000002C61D003910399D1F8C8148B42C0F27E
:10F1E0009480884D01245B1A55F8041F994204F15C
:10F1F0000104F8DD013343EA4413A2F2BC7243EA8E
:10F200004223814A039DB0FBF2F102FB11024FF44D
:10F2100061603C24B2FBF0F100FB11221C20C5F818
:10F22000CC04B2FBF4F004FB1022521042EA40126C
:10F2300042EAC12242EA0343C5F8F83454E6029B8D
:10F240000321DC1C002B3FF476AF704D56E7032101
:10F250004C226F4D02FB01F42B19184600216BF074
:10F2600074FD4C2200216BF070FD0399CAF100621D
:10F270000346520067482851D1F8F8145962C3E98F
:10F28000042202225A710122C3E907119A6058E749
:10F2900064235E4D02932FE70C4603911D21C4F8B1
:10F2A000CC1498E7C2E911551564D56329462E465A
:10F2B000D46C02F14C0354B39C681E64481E844213
:10F2C000C3E91166DE6312D0481C844216D08C421A
:10F2D0007FF440AF084600283FF43CAF116CCC6B84
:10F2E0000134CC631964936401461A46E0E70029AF
:10F2F0003FF430AF884253F80C2CECD1117900293F
:10F300003FF428AF53641A64EEE7012472E74049E2
:10F310000222264613E0CB6B0A635B011DBF03F696
:10F32000FF7702F1FF3303EB17331346C1E904669D
:10F33000C1E90D3351F84C0F5A1C0135C8B10B7996
:10F34000002BE8D10F690A63002F4BD14F6910469B
:10F35000531E4863002F4ED007F6FF7703EB173399
:10F36000201A8B63C41851F84C0F5A1C0135002821
:10F37000E5D129492948C1F8C4583E220D46C1F8B3
:10F38000A0283F22013BC1F8A4284022C1F8A828A8
:10F390000191C1F8B438C1F8B8489A00990FC5F87E
:10F3A0009C0853B340F2FF10121841F10001520AB9
:10F3B00042EAC152019C02F140010A4402EBC3033C
:10F3C000C4F8B028C4F8AC18154A1149C4F8BC18E0
:10F3D000C4F8C0185802D90DC4F89838C4F8900879
:10F3E0005160B7E607F6FF77531E03EB17304F69FE
:10F3F0004863002FB0D11346B2E70122DAE700BF1D
:10F40000880100205006002080510100D9EB00083F
:10F41000B85F00203C4A0808F01E0020484A08084F
:10F42000802700200A4AD2F8D83573B11968988825
:10F43000096992F8D53508401BB1B0FA80F040094F
:10F440007047003818BF012070470120704700BF87
:10F45000E04000200020704700231B6AFFDE00BF51
:10F460000378022B12D00F4943680269D1F848088B
:10F4700010B41840D1F84048D1F83C18931E400A07
:10F4800004FB030008445DF8044B7047054B4268D9
:10F49000D3F83418D3F8300800EB410000EB5220C9
:10F4A000704700BF605700202DE9F04F83B012F085
:10F4B000020701930FD070B9864D95F8E437A5F592
:10F4C000805613B9012385F8E437012302207370B5
:10F4D00003B0BDE8F08F7F4DD5F83848D4BB4FF06E
:10F4E000FF3E7D4C7D4EF146F046F2464FF0000C5B
:10F4F0002368984200F0BC8094F80EB0BBF1000F76
:10F500003DD0BBF1010F15D10CF5B17B06EB0B1B08
:10F510009BF807B01BF0010F0CD11BF07E0F09D137
:10F520005FEADB1340F0B280D4F808B0D34501D2D3
:10F53000DA46E1460CF1010CBCF10B0F04F11004AA
:10F54000D6D1BEF1FF3F29D1B8F1FF3F20D0634EA5
:10F55000C64624E0D5F84068D5F83C3806FB0434AC
:10F56000A042BCD395F8E43713B9012385F8E437FA
:10F570005A4B012200205A7003B0BDE8F08FE646D6
:10F580000CF1010CBCF10B0F04F11004B0D1D8E761
:10F59000B9F1FF3F18BFCE4600F082804F4ED5F83C
:10F5A000C84606EB0E1841F21869013448F8090004
:10F5B00041F21C600EF5B17C48F800404FEA0C1097
:10F5C000C5F8C846345006EB0C100024446006EB26
:10F5D0000C108079042876D8DFE800F0031B621B4A
:10F5E0002F0012F001046BD106EB0C10019B90F878
:10F5F00007904FEAE20868F3C719032B80F80790D9
:10F600005CD94FF6FF70834228BF034606EB0C100F
:10F61000838097B1D5F8CC06D5F8C8360130C5F847
:10F62000CC0641F21C6406EB0E1001330351C5F801
:10F63000C83606EB0C1304209871500705D506EB6D
:10F640000C10C37943F00103C371D30608D506EB50
:10F650000C16F379C3F34502013262F34603F371EA
:10F660001F4B012003EB4E230B6003B0BDE8F08F6E
:10F670001A4E0CF5B17406EB041E4FEA04189EF8FE
:10F6800006E0BEF1000F0FD1E64688E7E0460CF138
:10F69000010CBCF10B0F04F110047FF429AF50E70B
:10F6A000002003B0BDE8F08FD5F8C8060130E6466B
:10F6B00046F80800A446C5F8C80688E72346A5E72B
:10F6C00000239B68FFDE95F8E437002B3FF4FAAE89
:10F6D000FBE600BF60570020785D002060470020F7
:10F6E0007847002070B5104E3378022B0F4B0BBFBC
:10F6F000020AC0F3D412C4B200F07F04D3F8300879
:10F7000082B010440D460023032201A9FFF7CCFE6E
:10F71000012807D13378022B019B0CBF23F814502A
:10F7200043F8245002B070BD6047002060570020AD
:10F730002DE9F04FDFF82C8198F80060032E85B09A
:10F740000C46154643D001288CBF00220122022E10
:10F750000B68019269D14FEA1329DFB24FF4807A26
:10F760000138012820D84FF0010B9D4217D93C4E9B
:10F77000D6F8A8271AB1D6F8C417994258D0D6F8A7
:10F78000300800234844092203A9FFF78DFE012811
:10F790002CD0022817D020B123689D42E8D82560DC
:10F7A000032005B0BDE8F08FF7B12D4B93F8E427A7
:10F7B00012B9012283F8E4270123022088F80130DE
:10F7C00005B0BDE8F08F022005B0BDE8F08F01283C
:10F7D0008CBF0023012301930B684FF0800AC3F311
:10F7E000D41903F07F07BBE7D346BEE798F80020A3
:10F7F0000399DDF804C0022A14D0032AE3D151F89A
:10F80000273023F07043B3FA83F35B0963455F4409
:10F81000236821D05B4457452360ECD309F10109EB
:10F820000027BAE731F81730EDE74FF4807AD6E7D2
:10F83000D6F84018013A02EB41224902B2FBF1F23C
:10F840001344B3FBFBF20BFB12320AB15B449B1A6D
:10F850009D4223608CD8A2E7AB42A2D39FE700BFB2
:10F8600060570020604700202DE9F04FDFF86CB1B1
:10F870009BF800C0BCF1020F894683B0096882463C
:10F88000174640F08C800BF58053CEB2D3F8305839
:10F89000A6EB010805EB112590444FF480739844C2
:10F8A000B94208F1FF38B8FBF3F84CD2A844BCF1D8
:10F8B000030F07EB06040CBF80224FF48072641A1A
:10F8C0009442A8EB050328BF144666B994422CBFA6
:10F8D0000A220B2201A92846FFF7E6FD012809D0DC
:10F8E00003B0BDE8F08F0B2201A92846FFF7DCFD2D
:10F8F0000128F5D19BF800C0D9F80010BCF1020F27
:10F9000001F1010323D0B44210D9019906F18042DC
:10F91000013A01EB8202043901EB840142F8043F11
:10F92000914203F10103F9D1D9F80010A61B31442B
:10F93000BAF1010FC9F8001021D08F4205F101057D
:10F940004FF00006B3D8012003B0BDE8F08FB442F9
:10F95000ECD9019806F10042013A00EB420202386C
:10F9600000EB440022F8023F904203F10103F9D179
:10F97000A61B3144BAF1010FC9F80010DDD1B9421C
:10F98000DBD1BCF1020F1DD004F18044019B013C8E
:10F990004FF0FF3243F82420D9F80010CDE70BF5E3
:10F9A000805301F07F06D3F83038BCF1030FC1F368
:10F9B000D415A6EB01081D44904414BF4FF4807386
:10F9C00080236CE704F10044019B013C4FF6FF7279
:10F9D000504623F8142003B0BDE8F08F60470020A4
:10F9E00030B50446C06983B010B9012003B030BD02
:10F9F0000D460023032201A9FFF756FD0128F5D18A
:10FA0000B4F92030002B0ADA144B93F8E4270AB932
:10FA100083F8E407124B01225A700220E6E7019AAC
:10FA2000012D4FEA431102EB431303D0022D11D1F4
:10FA3000E5255554A268DA612278032A04D1002210
:10FA40001A775A779A77DA77626A5A83120C9A820F
:10FA500003B030BDE268DA61EEE700BF6057002016
:10FA6000604700202DE9F04190F83C30002982B039
:10FA7000044614BF02210021042B7BD8DFE803F0E9
:10FA8000030C3D486900FFF7ABFF012870D1626BA2
:10FA9000002A75D184F83C00404EDFF808814FF60B
:10FAA000F77706F5805516E0BA424FD864F054FA5D
:10FAB00001284FF000011DD1206BFFF713FE012834
:10FAC00018D1019AD5F844382263511E8B4228BFC1
:10FAD0000B46C5F844383278236B032A01A918462F
:10FAE0009AB2E1D1434531D864F036FA01284FF09B
:10FAF0000001E1D002B0BDE8F081426B04F13001B9
:10FB00000020FFF7B1FE012832D1032384F83C30F6
:10FB10002348E16AD0F8C437D0F84028C0F8C417A9
:10FB20005B1A02FB03F3D0F8A82702EB4322C0F8CC
:10FB3000A827D0F8AC2702EB4323C0F8AC3700214C
:10FB400000F5F460FFF74CFF012811D1042384F87D
:10FB50003C3094F82830042B04BF002384F828306C
:10FB6000A36B8BB120469847012002B0BDE8F0811D
:10FB70000228BFD194F82830042B09D00220B9E71D
:10FB8000022384F83C30B9E7012002B0BDE8F081DF
:10FB9000002384F828300220ACE700BF6047002033
:10FBA00060570020F7FFFF0F38B590F83430044657
:10FBB000052B43D8DFE803F01E033C0F185E006BF3
:10FBC0004FF0FF31FFF78EFD012837D1E06AB8BB57
:10FBD000032384F8343000212046FFF701FF012879
:10FBE0002CD1042384F8343094F82830082B2BD0FF
:10FBF000012038BD204DD5F8382800F130010232FF
:10FC00000120FFF795FD012823D00238C0B201285A
:10FC100014D8052384F8343094F82830082B04BF16
:10FC2000002384F82830012385F8E537022038BD09
:10FC3000C06A216BFFF756FD0128C9D0002038BDEE
:10FC4000022384F83430F4E7002384F828300120BC
:10FC500038BDE368D5F84018D4E90B2003EB412305
:10FC6000C5F84408C4E9033002B96062012384F88E
:10FC70003430A5E7004DCFE76057002010B590F86D
:10FC800038300446032B59D8DFE803F0022F3843FD
:10FC90002B4AC068117802F580530329D3F8401825
:10FCA000D3F8C4270CBF4FF0800C4FF4807C01FBCD
:10FCB0000CF100EB4120C4E90302D3F8A807A0EB44
:10FCC0004120C3F8A807D3F8AC07A0EB4121E06AB4
:10FCD000C3F8AC1702EB0C01C3F8C417C4E90C213C
:10FCE00040BB6262012384F8383016480021FFF7D8
:10FCF00077FE012811D1022384F83830626B04F1B9
:10FD000030010120FFF7B0FD012806D1032384F85C
:10FD1000383000212046FFF763FE431EDBB2012B83
:10FD200000D910BD94F82830062B04BF002384F8B6
:10FD3000283010BDA2EB0C022263D3E70220ECE7CF
:10FD400060470020005F00202DE9F0434368C3F3C3
:10FD500008020A44B2F5007F83B004460D4605D27E
:10FD60002B446360012003B0BDE8F08390F91A20B2
:10FD7000501C0AD0414902F5B17201EB0212D1794F
:10FD80006FF30001D171FF22A27694F91B20511C60
:10FD90000FD03A4902F5B17201EB0212FF26D17978
:10FDA000C1F34500013820EAE07060F34601D171EB
:10FDB000E67694F800C0BCF1020FD1D0DFF8C48021
:10FDC000D8F84028B5EB422F4FEA422915DCD8F885
:10FDD00048781F407A42AA420FDCEA194A4510D2FD
:10FDE00020690028BED0254A1278032A40D080B26C
:10FDF0004FF6F7729042B3D9B4E7002003B0BDE8E4
:10FE0000F083227E206912F0080626D0D8F8C42795
:10FE1000411C8A4213D300D100214B44A5EB0905B4
:10FE2000DB1BBCF1020F60613D4421616360084649
:10FE3000D7D1D8F85028B3EB422F91D392E798F856
:10FE4000E42722B9012388F8E437636820690B4A64
:10FE50000126567094F800C0DFE701A964F07CF831
:10FE60000128CAD10199636894F800C02069D4E7D9
:10FE7000034A90427FF674AF74E700BF60470020EA
:10FE8000F7FFFF0F605700202DE9F04790F838404A
:10FE900082B00546032C00F2AB80DFE804F00219C3
:10FEA000710BFFF781FE012810D002280AD103232D
:10FEB00085F838302B6C002085F82800002B6FD097
:10FEC00098470224204602B0BDE8F08785F8380044
:10FED0002B78022B60D0474A6B68D2F8482803EA97
:10FEE0000208C8F34F282846FFF7BAFA414F0646E2
:10FEF000A8EB0008A7F5805901A90222002330468B
:10FF0000FFF7D2FA08EB060401281FFA84FA4FF42F
:10FF100000724FF000010446D4D101986AF015FF39
:10FF2000EB694FF40071284613B16B68002B3BD08E
:10FF3000D7F84038013B9A4506F101060DD2FFF78C
:10FF400003FF0028D8D197F8E43713B9012387F8C5
:10FF5000E437012389F80130CEE7C3EBC3535902DC
:10FF60002846FFF7F1FE40B997F8E43713B90123AB
:10FF700087F8E437204B01225A70022385F8383085
:10FF80002B6C002285F8282063B12846984701246D
:10FF9000204602B0BDE8F0876B68C3F34F28A2E7A4
:10FFA00002248FE701248DE7019B4FF020324FF0B0
:10FFB0002E0E4FF0100C1A605A6083F800E0C3F860
:10FFC00007206C6A1A625A6283F80BC0C3F82720B4
:10FFD00083F820E083F821E0EA6B5C835A8724FAF7
:10FFE0000CF422FA0CF29C8283F82BC09A869FE7CD
:10FFF000002467E760570020604700202DE9F041AA
:020000040801F1
:10000000B1F904300F2B82B00E460446174635D0A6
:100010002046FFF725FA94F91B80B8F1FF3F3ED048
:10002000554B41F2186203EB08118A58904211D1E6
:10003000183303EB4825B38801331BB205EB431596
:10004000B38020463D60FFF70BFA3060012002B01C
:10005000BDE8F08103F5805292F8E41700296AD0D8
:1000600001225A702278022A69D02369002B50D1CC
:10007000002301203B6002B0BDE8F0814FF4007125
:10008000FFF762FE002852D04FF6FF73B380204680
:10009000FFF7E6F994F91B80B8F1FF3FC0D1227851
:1000A000022A54D02369002BDDD033490978032973
:1000B0000EBF32499BB24FF6F7718B4294BF0023BB
:1000C0000123002BCFD138B92D4A92F8E437002B09
:1000D0004ED0294B01225A700023112201A9FFF7AB
:1000E000E3F9012842D1019D264BEB1A48BF03F2E8
:1000F000FF13B3F5B05F4FEA632230D3204A92F882
:10010000E43713B9012382F8E4371B4B01225A70FC
:1001100027E0194A1278032A0EBF184A9BB24FF6FD
:10012000F772934294BF00230123002BA0D100203B
:1001300002B0BDE8F081012182F8E41790E7104A8F
:100140006368D2F85028B3EB422F91D2EFE70C4A04
:100150006368D2F85018B3EB412FB4D3F1E74FFAEC
:1001600082F884F81B80002D7FF465AF22787AE74F
:10017000012382F8E437ACE760470020F7FFFF0F68
:1001800060570020784700202DE9F04790F8303084
:1001900088B00446042B4BD8DFE803F0030C4DD1A4
:1001A0004600C54866F010F94FF6FF72012322841D
:1001B00084F83030DFF8008304F11C0501AE04F14F
:1001C0003109324629464046FFF718FF012800F062
:1001D000DB8002282CD1B94901F5805595F9022818
:1001E000531C0AD002F5B17201EB0212D3796FF3FE
:1001F0000003D371FF2385F8023895F903385F1C9B
:100200000FD003F5B17301EB0313DA79C2F34501A3
:10021000013921EAE17161F34602FF21DA7185F8C3
:100220000318042384F830300020E36A20709847D4
:1002300008B0BDE8F087A24D95F81038002BF7D133
:100240009D4F04F11C0901AE4FF0090832464946A2
:100250003846FFF7D3FE012840F0E88001980028D7
:1002600000F0C2800378E52B01D0002BEED1954A37
:10027000821A48BF02F2FF12B2F5B05F4FEA622362
:1002800080F00E818D491B018F4A13449A7B042A0A
:100290000CD0D5F8C8260132C5F8C8265A60042209
:1002A0009A73D5F8CC360133C5F8CC3695F90238B7
:1002B0005E1C0AD003F5B17301EB0313FF2285F82E
:1002C0000228DA796FF30002DA7195F903385A1CC3
:1002D0000FD003F5B17301EB0313FF21DA7985F831
:1002E0000318C2F34501013921EAE17161F34602C5
:1002F000DA71202200216AF028FD019BD4F8312018
:10030000D4F8351059601A60B4F8392094F83B10CD
:1003100099721A81019B627EDA7205A802F070F967
:10032000BDF81430002B40F0058144F28171019A30
:1003300003201182D3811183D38284F83000237E7D
:10034000980608D5E0690023112205A9FFF7ACF84B
:1003500001287FF46DAF204666F036F82369002B44
:1003600068D0237E03F0F70213F0040322766ED1E7
:10037000122A00F083800022E36A84F828202046B5
:10038000984708B0BDE8F087019F002F00F09E80DD
:100390003B78002B00F09A8097F80BA01AF0080F1A
:1003A0007FF40FAF0B22494638466AF00BFD002858
:1003B0007FF407AF637E8AEA0303DB0640F1FB802C
:1003C0003E4901F5805595F902385E1C3FF415AFA2
:1003D00003F5B17301EB0313FF2285F80228DA79E4
:1003E00060F30002DA7108E795F8E837022B3FF472
:1003F00018AF95F81038002B7FF413AF85F820382C
:10040000C5F82438C5F8283885F81C38D5F8FC37E5
:10041000C5F81438D5F8443885F81088C5F8183868
:100420003846FFF731FD01283FF410AF02283FF4B2
:10043000F8AEFDE6237E19079DD5214B93F8C8271A
:10044000002A7FF4F5AE072283F8C82793E7A56852
:10045000E66A002384F8283029462046FFF774FC1A
:10046000002840F0A28094F82830002B7FF4E0AE02
:100470000223C4E90B6584F82830D9E6626AE16A90
:10048000A163042084F82800C4E90B22C4E90233E4
:1004900084F83C3063636362204665F095FFC7E6ED
:1004A00095F8E43713B9012385F8E43703490123AC
:1004B0004B706FF00F03E7E6485F002060470020B5
:1004C0006057002078470020785D0020584901F5EA
:1004D000805595F902385E1C0AD003F5B17301EB23
:1004E0000313DA796FF30002DA71FF2385F802381B
:1004F00095F90338581C0FD003F5B17301EB0313C2
:10050000DA79C2F34501013921EAE17161F346026A
:10051000FF21DA7185F80318237EDA067FF581AEB4
:10052000444865F051FF4FF6FF720223228484F89D
:10053000303081E6404B05A8B3F9E08501F08AFF31
:100540004FF47A72002306460F4668F075FC3C2390
:10055000054608FB0355394630464FF47A720023AE
:1005600068F06AFC4FF47A7192B20023C5FB012354
:1005700002A801F0A5FF9DF80A209DF80B109DF838
:100580000C3041EA4211BDF80820A2F2BC7241EAE7
:1005900042219DF80D20DB0243EA42139DF80E2014
:1005A00043EA520389B29BB2C1E6002E3FF440AE4B
:1005B0002046B0473CE6BA8A7B8B204D43EA024393
:1005C0006362D5F84028FB69A3605202B3FBF2F1E5
:1005D00002FB113109B113445B1AE36084F819A0DE
:1005E00095F902381249581C0AD003F5B17301EB92
:1005F0000313DA796FF30002DA71FF2385F802380A
:1006000095F903385A1C0FD003F5B17301EB0313AE
:10061000DA79C2F34501013921EAE17161F3460259
:10062000FF21DA7185F80318032384F8303086E659
:1006300060470020485F0020E04000206057002015
:1006400010B5037890F818C0023B012B044602D97C
:100650001CF0060F5DD11CF0200F3CD194F91A302C
:10066000591C0AD0314A03F5B17302EB0313FF2181
:10067000DA796FF30002DA71A17694F91B305A1C13
:100680000FD02A4A03F5B17302EB0313DA79C2F3F0
:100690004501013921EAE17161F34602FF21DA7176
:1006A000E1761CF0080F0DD0214B93F8C827072ADC
:1006B00005D093F8E427A2B31C4A0121517000220F
:1006C00083F8C827E26A0023237084F82830FAB13F
:1006D000BDE81040104700231649E0691A018A5806
:1006E000904206D001330B2BB8D01A018A589042A1
:1006F000F8D10E4A03F5B17302EB0313DA79C2F3B2
:100700004501013921EAE17161F34602DA71A5E799
:1007100010BD0121FFF764F90128F9D194F818C040
:1007200099E7012283F8E427C6E700BF604700206D
:1007300060570020785D00204FF0FF3C10B41A4A4B
:100740001A4C6046002304E001330B2B02F1100227
:1007500017D011780429F7D103F5B17104EB011119
:10076000C979C907F0D4B0F1FF3F52F80A1C01D093
:100770006145E9D2184601330B2B8C4602F1100279
:10078000E7D1431C03D101205DF8044B7047074BB0
:1007900000F5B17003EB001083880BB91B69FFDE15
:1007A0000023DB68FFDE00BF865D0020604700207D
:1007B0002DE9F04F90F82830013B83B00446082B18
:1007C0000BD8DFE803F0383C1E2305290A2E33003E
:1007D0000121FFF747F9012802D003B0BDE8F08FEF
:1007E0002378002284F82820002BF6D0D4E90113C6
:1007F0008B4238BF0B46226CA360032184F828107B
:10080000E262204603B0BDE8F04F19E7002103B0D3
:10081000BDE8F04FFFF726B903B0BDE8F04FFFF792
:100820002DBA03B0BDE8F04FFFF7BEB903B0BDE885
:10083000F04FFFF729BB03B0BDE8F04FA4E4534FDE
:100840004368D7F84858016BD7F840281D4068180E
:10085000B0EB422F4FEA42269C46C0F0938094F8BA
:1008600000E0DFF82C91A7F5805A4FF6F778BEF13B
:10087000020F14D02069002857D1D4F804C0A3680F
:10088000E26A634538BF63460021A36084F82810FC
:10089000002AA2D0204603B0BDE8F04F1047D4F89C
:1008A00004C0D7F85028BCEB422FE8D22069227E42
:1008B00012072CD5D7F8C42700F1010C624522D2CB
:1008C00097F8E42722B9012387F8E4376368216B9E
:1008D00001228AF8012094F800E0891B294433445E
:1008E0005B1B8E42C4E904C0636021639C464FF0E9
:1008F0000005BCD9BEF1020F3ED020690028BED051
:10090000DFF890B01FE0E8D14FF0000CE5E701A957
:1009100063F022FB01287FF460AF2069DDF804C09A
:1009200094F800E06368216BD7E79AF80020032A67
:10093000D3461AD082B2424594BF00220122002A37
:10094000B5D0D4F804C09BF80030032B0EBF104B79
:1009500080B24FF6F773984294BF00200120002820
:100960008DD18C44C4F804C089E7484594BF002267
:100970000122002A9BD0E4E7D7F85028B3EB422F9E
:10098000EFD37CE794F800E0B4E700BF60570020A5
:10099000F7FFFF0F6047002010B5194C194844229B
:1009A00000216AF0D2F9237804F580544FF6FF70E5
:1009B000D4F84C28A4F80208022B4FF0030118BF0A
:1009C00003234FF0100C84F8001804F5FD6000219B
:1009D000C4F8F82784F8E837C4F80C2884F801C86C
:1009E000FFF7B2F948B994F8103833B9022284F805
:1009F0001028C4F81438C4F81838012010BD00BFFE
:100A000060470020485F002000234FF6FF7201215D
:100A1000017243818381C38102828274704700BF67
:100A2000154BFF22F0B54FF0000C4FF0FF3EC270A7
:100A30000271027242724273827303F10C077646AE
:100A400065466446624602EB820281189F428454E6
:100A50004D7081F802C0CE7081F804E00BD093F99C
:100A60000620DC791D7A93F809C093F90A6093F99E
:100A70000BE00633E7E7F0BD30CD07084FF0000C80
:100A800001210222032380F805C08171C271037223
:100A9000704700BF00230222037043708370C3704D
:100AA00002717047002303704370704700230122D6
:100AB000027043708370C370704700BF40F22E4CC9
:100AC0004FF4F071A0F81EC001804FF4FA6C4FF49F
:100AD0007A71A0F820C0418440F2262C4FF4F561D1
:100AE0000023A0F81CC081844FF00E0C02210722C5
:100AF00080F826C043718371417440F2012C40F2AA
:100B00000341438240F205638270A0F814C0C182A1
:100B100003838276704700BF8388C3F30B0393423D
:100B2000A8BF134670B51A461D460C460646806897
:100B30006AF0A8F862199442B569074B08D00748D3
:100B400014F8011B00FB03F3A24283EA0103F7D16F
:100B50002B60012070BD00BFC59D1C819301000169
:100B60000023037043708370C370704700230370C9
:100B700043708370C370704700220123027042707B
:100B80008270C270037143718371C371704700BF7B
:100B9000FF23037043708370C370704700230621E6
:100BA0004FF47A72C0E9012301700373704700BFEC
:100BB00000230372704700BF00230370704700BF1B
:100BC000002303704372438183818373704700BFA6
:100BD00000234370C37003700371704710B5002386
:100BE000411CFF2200F8132001F8132001330B2BC6
:100BF000F8D10B4B4FF0FF3103F10F0400228C466C
:100C000005E093F904C093F9051013F8032F00F8D9
:100C100012C000EB420E9C428EF80110F1D110BDC3
:100C200044CD0708704700BF03230370704700BF1F
:100C3000002303704370C37083700371704700BF5B
:100C4000704700BFD0ED007AD0ED016A30EE677AD0
:100C5000E6EE877AB0EE670AC0ED007A704700BF13
:100C6000D0ED017AD0ED026A30EE677A90ED000A9D
:100C7000E6EE877A37EEC07AC0ED017AA6EE870AF3
:100C800080ED000A704700BF90ED017AD0ED036A55
:100C9000D0ED027A30EE470AA6EE807A90ED000A97
:100CA00080ED017A37EE676AE6EE867A37EEC07A33
:100CB000C0ED027AA6EE870A80ED000A704700BFF9
:100CC000DFED277AB4EEE70AF1EE10FA0CDDDFED86
:100CD000256A9FED257AF0EE407AF4EEC77AF1EEC0
:100CE00010FA30EE660AF6DCDFED207AB4EEE70AA1
:100CF000F1EE10FA0CD5DFED1B6A9FED1D7AF0EED8
:100D0000407AF4EEC77AF1EE10FA30EE260AF6D405
:100D1000DFED187AB4EEE70AF1EE10FA14DDDFED3C
:100D2000107A37EEC00A60EE006A9FED136A9FEDFD
:100D3000137ADFED137AA6EE867A20EE266AE6EEC7
:100D4000877AA6EE270A7047DFED0E7AB4EEE70A3F
:100D5000F1EE10FA44BFDFED057A37EEC00AE2E7A4
:100D6000DB0F4940DB0FC940E4CB1641DB0F49C024
:100D7000E4CB16C1DB0FC93F92E741B99730083C7D
:100D800015A82ABEDB0FC9BFD0ED056AD0ED017AE8
:100D900090ED007A90ED066AD0ED025A90ED035A7C
:100DA00080ED050A66EEA77AC0ED066AE7EE007AE6
:100DB00090ED077AE5EE867A90ED086AD0ED045A58
:100DC00080ED087AE5EE477AE5EEC67AB0EE670A7E
:100DD000C0ED077A704700BFD0ED057A90ED006A4C
:100DE00090ED067AD0ED035AE6EE007A90ED016AB6
:100DF000F0EE406AA6EE267AB0EE670AD0ED047AED
:100E000090ED026A67EEC07AA5EEC07AE6EE267A29
:100E100080ED057AC0ED067A704700BF2DE9F047F6
:100E2000089F3C460E4614F8011B002B054614BFD4
:100E30004FF030094FF0200941B3002A2CDD234642
:100E400000E0B2B113F8010B9046013A0028F8D146
:100E5000A8F102086AB1C24649462846B04753463F
:100E6000002B0AF1FF3AF7DC397828EAE872013200
:100E700049B1D71B2846B047E01914F8011B0029D7
:100E8000F8D1BDE8F0871046BDE8F087002A02F1EE
:100E9000FF38E0DC0846F4E70022EAE703685A1C62
:100EA00002601970704700BF024B186803681B6826
:100EB000184700BF80950020884210B54FF001040C
:100EC0003ED301FB04F4B0FBF4FC8C45F9D2CCB169
:100ED00022BB08E0A14203F801EBB4FBF1F211D808
:100EE000B0FBF2FC1446BCF1090F0CF1570E0CF1EB
:100EF000300204FB1C00EDDCA14203F8012BB4FB23
:100F0000F1F2EDD900221A7010BDA14203F801EBF5
:100F1000B4FBF1F2F6D8B0FBF2FC1446BCF1090FB9
:100F20000CF1370E0CF1300204FB1C00EDDCA14289
:100F300003F8012BB4FBF1F2EDD900221A7010BDB9
:100F40008446002AEAD1CEE7002870B503DA2D23C3
:100F500001F8013B4042092886464FF0010307DDB6
:100F600003EB83035B00B0FBF3F2092AF8D8EBB183
:100F7000104CBEFBF3FCA4FB0320C008BCF1090F1E
:100F80000CF130060CF15705024607D8092B01F881
:100F9000016B03FB1CEE09D90346EAE7092B01F8B4
:100FA000015B03FB1CEE01D91346E2E700230B7043
:100FB00070BD00BFCDCCCCCC0378202B024600F115
:100FC0000100F9D0092BF7D02D2B28D02B2B03BFF4
:100FD0005378B7EE000A0246B7EE000AA3F13001DB
:100FE000C8B209289FED567A10D8F2EE046A07EECF
:100FF000901AF8EEE77A12F8013FE7EE267AA3F1AD
:101000003001C8B20928B0EE677AF0D92E2B5ED035
:1010100003F0DF03452B07D020EE070A7047537813
:10102000BFEE000A0246D9E710B451782D2978D0D6
:101030002B296AD0A1F13003092B02F101026BD8F0
:101040000024002303EB830301EB430312F8011F89
:10105000A1F130000928A3F13003F3D9B3F59A7F49
:101060001A4628BF4FF49A72072B66D9DFED356A0E
:101070001346F7EE007A083B072B67EEA67AFAD8FC
:1010800002F00702DAB1F2EE046A012A67EEA67AEC
:1010900015D0022A67EEA67A11D0032A67EEA67A47
:1010A0000DD0042A67EEA67A09D0053A67EEA67A33
:1010B00005D067EEA67A012A18BF67EEA67A6CB350
:1010C00087EE277A5DF8044B20EE070A70475378C5
:1010D000A3F13001C8B2092802F1010298D8F2EE5A
:1010E000046AF0EE665A07EE901AF8EEE77A12F804
:1010F000013F87EEA66AA3F13001C8B2092866EE67
:10110000A56A37EE067AEED982E79178A1F130032D
:10111000092B02F1020293D9F7EE007A27EE277A23
:10112000D0E79178A1F13003092B02F1020288BFC8
:10113000F7EE007AC4D8012483E7F7EE007AA1E73E
:101140000000000020BCBE4CF0B5067906F0E003BC
:10115000402B03D145794FF0FF3406E0602B4FF070
:101160000105F8D1447905FA04F40023012006F0C2
:101170000706AB4200D1F0BD052E0FD8DFE806F020
:101180000308101D242448B1C85CD75C78400FE0E8
:1011900020B1C856D756C71B784278410133E8E7DB
:1011A0000028FBD031F8130032F81370784080B279
:1011B00020420CBF01200020F0E70028EED031F9DA
:1011C000130032F91370E6E70028E7D051F8230046
:1011D00052F82370DAE7037903F01803102B1CD0C0
:1011E00004D82BB1082B06D000207047182BFBD158
:1011F000B0F80B007047104BB0F80B0093F90030BB
:10120000591C06BF0D4B1B79DBB203EB830203EBCA
:10121000C20300EB830080B27047074BB0F80B00AD
:1012200093F901305A1C06BF044B5B79DBB2C3EB68
:10123000031300EB4300EEE7B0060020809500208A
:10124000114B002130B50160818003F10C054FF492
:1012500048748E460A4602EB420200EB420C00F84C
:1012600012E08CF80110DA788CF80220AB42ACF86E
:10127000044007D093F9062093F807E0197A5C89B7
:101280000633E8E730BD00BF58CD0708092900D074
:1012900001B9704701394B0003F00802930001F0D7
:1012A0000301A3EB9203C1EB0111C3EB0313C1EBE9
:1012B000011100229B0089000260818043807047F9
:1012C000002201230280C381704700BF38B5184D4A
:1012D0002B7D04463BB980F83A3095F83530B3B9E8
:1012E00084F83B3038BD052205F11801203069F043
:1012F0007DFD152205F1200104F1250069F076FD40
:10130000012384F83A3095F83530002BE8D0094DA8
:101310000FCD20606160A260E3600FCD4FF0010C43
:1013200084F83BC020616161A261E36138BD00BF08
:1013300080950020B895002010B500213822044681
:1013400069F003FD0D490E4A0E482061C4E90512FB
:101350000D480E4AE061012341F61E614FF0090C71
:10136000E18484F808C0A37384F82130A262214686
:101370000748BDE8104036F0C5BE00BF1A046C0730
:10138000001975036400DC0543080E001E7D010191
:10139000C04A0808B5EEC00ADFED347AF1EE10FA63
:1013A000CCBF30EE270A30EE670ADFED317A20EE4F
:1013B000270A70B5FDEEC07A86B017EE904A054652
:1013C00084EAE470002303A9A0EBE470CDE90033C4
:1013D000029360F0F9FA002CACBF20232D2303A860
:1013E0008DF8003067F064F801286E4628D0022896
:1013F00032D003281CD003A9304669F0AEFC304639
:1014000067F056F80338C4B222463146284669F0E0
:1014100039FC00232B55284667F04AF82E232B541D
:1014200001303119284469F0B4FC284606B070BD7B
:10143000302303A930468DF8013069F08EFCDEE7D9
:1014400043F23002302303A93046ADF801208DF875
:10145000033069F082FCD2E743F2300303A930463F
:10146000ADF8013069F079FCC9E700BF6F12033AAB
:1014700000007A440AF06EB813B568B14C1E14F837
:10148000011F21B902B0BDE810400AF077B8019001
:101490000AF060F80198F2E702B010BD08B520210B
:1014A00069F06AFC034620B11A78202A00F1010095
:1014B000F8D0184608BDF8B5D0B1104B0138C700B8
:1014C00003EBC000CA4390F85C6090F85D5002F0F6
:1014D000010282EA0604A5420AD0806D28B18588FF
:1014E0000068B24214BF058345833B4483F85D40E6
:1014F000CB0701D4FBF7C0FAF8BD00BF80950020F0
:101500002DE9F341124D134F002305F8783F0446AF
:1015100000EB8106B44203D10F4802B0BDE8F08170
:101520003946284669F019FC2146684669F031FCC5
:101530004FF000082021684669F01EFC28B9694672
:10154000284669F00AFC0434E4E780F80080F1E7FB
:1015500080950020B19F0808F8950020024BD3F831
:101560009C0044F023B900BF80950020704700BF65
:10157000084B09498B4202460AD2184602E01C3049
:10158000884205D20388C3F30B039A42F7D1704710
:1015900000207047B8E10808E4EB080870B505467C
:1015A000B0F80900FFF7E4FF064B93F8A06004468B
:1015B0002846FFF710FE16B1E368184470BDA36813
:1015C000FBE700BF8095002038B505460C46FFF7C5
:1015D000E5FF2B7903F0E002602A03F007032AD12C
:1015E000052B0CD8DFE803F0030B0F0B1B1B6A79EC
:1015F00001239340DBB2027814B11343037038BD6A
:1016000022EA0303FAE76A79012393409BB2028836
:1016100014B113430380F2E722EA0303FAE76A797D
:10162000012303FA02F2036814B113430360E6E7EF
:1016300023EA0203FAE7052BE1D8DFE803F003030E
:10164000050507070470DAE70480D8E70460D6E7E9
:1016500070B585880B460446C5F30B052A46002164
:10166000184669F072FB6169084A9142034602D349
:10167000074A914205D319B1BDE8704018460847A2
:1016800070BD2A46BDE8704069F0FCBAE4EB08087A
:1016900063EE080838B5064C064DAC4206D2A16888
:1016A00020461C34FFF7D4FFAC42F8D338BD00BF4E
:1016B000B8E10808E4EB08080A44914219D000B5E3
:1016C00001F1FF3C02F1FF3E41F221011CF8012F24
:1016D000082380EA022010F4004F81EA40020ABF8A
:1016E000400090B280B2013BF5D1E645EED15DF805
:1016F00004FB7047F8B5164D6B78BE2B26D102223D
:1017000029464FF6FF70FFF7D7FF124FAC1C228817
:101710004AB1A618BE4219D2052A17D92146FFF7A9
:10172000CBFF3446F3E721460222FFF7C5FF022232
:10173000A118FFF7C1FF0634074B641BA3F8A240B2
:1017400041F60F53C31A58425841F8BD0020FCE738
:1017500000400008008000088095002048400823D1
:1017600010F0800F82EA40010ABF4000C8B2C0B248
:10177000013BF5D1704700BF30B505688D4219D9DE
:1017800001F1FF3E6C1E00231EF801CF082183EA01
:101790000C0313F0800F82EA430C0ABF5B005FFA70
:1017A0008CF3DBB20139F4D17445EDD16A1C0260CF
:1017B0002B7030BD00236A1C02602B7030BD00BF4F
:1017C00007EE901AB8EE677ADFED7C7A27EE000A12
:1017D00060EE277ABDEEE77A17EE103A2033402B01
:1017E00000F2DB809FED767AB4EEC70AF1EE10FAD4
:1017F000B0EE677A0CDDDFED735A9FED736AF0EEA1
:10180000476AF4EEC66AF1EE10FA37EE657AF6DC56
:10181000DFED6E6AB4EEE67AF1EE10FA0CD5DFED8C
:10182000695A9FED6B6AF0EE476AF4EEC66AF1EE14
:1018300010FA37EE257AF6D4DFED666AB4EEE67A72
:10184000F1EE10FA00F39D80DFED636AB4EEE67A04
:10185000F1EE10FA44BFDFED5D6A36EEC77A27EE8F
:10186000075ADFED5E5A9FED5E6ADFED5E6ADFEDDF
:101870005E4AA5EE256A27EE054AE5EE066AF7EE12
:10188000005AA4EE267AF0EE656AE7EE646AE7EEA7
:10189000245A86EEA54A9FED4F7A77EE877ABDEE01
:1018A000E77A17EE103A2033402B6FD89FED4F7A2E
:1018B000B4EEC70AF1EE10FA0CDD9FED426ADFEDDF
:1018C000426AB0EE677AB4EEE67AF1EE10FA77EE9D
:1018D000C67AF6DC9FED3D7AF4EEC77AF1EE10FAA7
:1018E0000CD59FED386ADFED3A6AB0EE677AB4EE58
:1018F000E67AF1EE10FA77EE867AF6D49FED357A35
:10190000F4EEC77AF1EE10FA4CDD9FED397A77EEFE
:10191000677A67EEA74A9FED317A9FED315ADFED86
:10192000316AA4EE875A67EEA43AE4EE856AB7EE10
:10193000006AE3EEA67AB6EE007A36EE676AB8EE93
:10194000005A67EE857A26EE077AB7EE005AC5EEA2
:10195000256A0023836143610362C36180ED044A09
:1019600026EE877A26EE866A66EEA77A80ED095A19
:1019700080ED007A80ED016A80ED027AC0ED037A95
:101980007047DFED1B6A36EEC77A68E7DFED197A3C
:10199000B6EE007AB7EE006AD7E7B7EE004AF0EE8F
:1019A000445A78E79FED0C7AF4EEC77AF1EE10FA1C
:1019B00044BF9FED067A77EE677AAAE727D4D2363E
:1019C0000024F448DB0FC940E4CB1641DB0F49C0CB
:1019D000E4CB16C1DB0FC93FDB0FC9BF92E741B9AA
:1019E0009730083C15A82ABEF304353F00247448FC
:1019F000DB0F4940000000009FED2E7A70EE077A61
:101A0000FDEEE76A16EE903A2033402B4FD8B4EE45
:101A1000C70AF1EE10FA0CDD9FED276ADFED276AA9
:101A2000B0EE677AB4EEE67AF1EE10FA77EEC67AA7
:101A3000F6DC9FED237AF4EEC77AF1EE10FA0CD5BE
:101A40009FED1D6ADFED1F6AB0EE677AB4EEE67AAD
:101A5000F1EE10FA77EE867AF6D49FED167AF4EE70
:101A6000C77AF1EE10FA1DDC9FED177AF4EEC77A13
:101A7000F1EE10FA44BF9FED127A77EE677A27EE07
:101A8000A76ADFED125ADFED126A9FED127AE6EED9
:101A9000256A67EE865AA6EE267AE5EE877AB0EEDC
:101AA000670A70479FED0C7A77EE677AE7E79FED5C
:101AB0000B0A7047DB0FC93FDB0FC940E4CB16416F
:101AC000DB0F49C0E4CB16C1DB0FC9BF92E741B9B8
:101AD0009730083C15A82ABEDB0F494000000000E3
:101AE000F0EEC07AB0EEE07AB4EEE77AF1EE10FAFA
:101AF000B4BFB0EE676AB0EE476AB5EE406AF1EE89
:101B000010FA46D0B4EEE77AF1EE10FA8CBFF0EEA0
:101B1000675AF0EE475AC5EE866ADFED1F2ADFED01
:101B20001F3ADFED1F4A9FED1F5A9FED1F3A9FEDB1
:101B30001F4ADFED1F5AE6EEE23AA6EE834AE6EED2
:101B4000A34AB7EE006AA6EEA45AA6EE846AE6EEB1
:101B5000855AC5EE866AB4EEE77AF1EE10FA48BF10
:101B6000DFED147AF5EEC00A48BF77EEE66AF1EED3
:101B700010FA48BFDFED107AB5EEC00A48BF77EE25
:101B8000E66AF1EE10FA48BFF1EE666AB0EE660A58
:101B90007047DFED076ADEE739094E3DE3B59E3E4B
:101BA00088FA163E45FE7F3F99FB243F69A2163E08
:101BB000A7DFA834DB0FC93FDB0F494090ED005A87
:101BC0009FED4C0A35EE000A08B5FDEEC07A17EE1F
:101BD000903A2033402B7BD8FFF772F8F0EE403A72
:101BE000FDEEC57A17EE903A2033402B7FD8B0EE49
:101BF000450AFFF765F8B0EE405AD0ED014A9FED77
:101C00003D0A34EE800AFDEEC07A17EE903A20339A
:101C1000402B69D8FFF754F8F0EE405AFDEEE47A15
:101C200017EE903A2033402B5BD8B0EE640AFFF7F2
:101C300047F8F0EE404A90ED023A9FED2E0A33EE5F
:101C4000000AFDEEC07A17EE903A2033402B45D8BB
:101C5000FFF736F8B0EE404AFDEEC37A17EE903A41
:101C60002033402B37D8B0EE430AFFF729F8F0EEC7
:101C7000407A24EE233A27EEA36A24EE057A67EE33
:101C8000856AB0EE462AF0EE432AA7EE242AE6EE55
:101C9000E42AA6EE247AE3EE646A24EE254A65EE91
:101CA000E77A25EE655A65EEA35A81ED004AC1ED4B
:101CB000017AC1ED024A81ED032AC1ED042A81EDCA
:101CC000055AC1ED066A81ED077AC1ED085A08BDD3
:101CD000DFED093A84E7DFED087ACAE79FED064AAF
:101CE000BAE7DFED054AA6E7DFED035A96E79FED79
:101CF000025A82E7DB0FC93F000000002DE9F043E4
:101D000089B0541C03941478002C00F0078100253E
:101D1000074688461E46A94609E021463846C04780
:101D2000039A0135531C03931478002C3DD0252CC5
:101D3000F3D1931CCDE903395078302800F094801A
:101D4000A0F13003DBB2092B4FF0000440F2978082
:101D50006C2838D0782822D857282AD9A0F15803DF
:101D6000202B1CD8DFE803F0B41B1B1B1B1B1B1B09
:101D70001B1B1B959D1B1B1B1B1B1B1B1B1BAF1B23
:101D80001B1B1B111BA71B1BB40056F8043B049A1A
:101D90000093002341463846FFF740F80544039A74
:101DA000531C03931478002CC1D1284609B0BDE818
:101DB000F0830028F9D02528F1D125213846C047E5
:101DC0000135039AAEE7039B5A1C039219787829D0
:101DD000A8D8572958D9A1F15803202BA2D801A07F
:101DE00050F823F0E91E0108251D0108251D0108F2
:101DF000251D0108251D0108251D0108251D0108B7
:101E0000251D0108251D0108251D0108251D0108A6
:101E1000931E0108011F0108251D0108251D010849
:101E2000251D0108251D0108251D0108251D010886
:101E3000251D0108251D0108251D0108C91E0108D1
:101E4000251D0108251D0108251D0108251D010866
:101E50008B1D0108251D01080D1F0108251D010806
:101E6000251D0108E91E0108D31C03939078A0F1F9
:101E70003003DBB2092B4FF001043FF669AF04AA2F
:101E800003A962F039FB63E700298ED0252994D09D
:101E900048E756F8041B3846C9B2C0470135039AD3
:101EA00040E756F8040B05A9FFF74EF805AB009381
:101EB000049A23466EE756F8040B05AB00220A216C
:101EC000FEF7FAFFF2E7039A56F8043B1D6029E794
:101ED000A0F15802B2FA82F256F8040B520905AB8F
:101EE0001021FEF7E9FFE1E7A1F15802B2FA82F210
:101EF00056F8040B520905AB1021FEF7DDFFD5E7BC
:101F000056F8040B05A9FFF71FF8CFE756F8040BA6
:101F100005AB00220A21FEF7CFFFC7E7254644E7BD
:101F200073B5144C01920646D4F8A4000D46C0B116
:101F30001149FFF7A1FAD4F8A4003146FFF79CFA43
:101F40000E49D4F8A400FFF797FA0D49019BD4F885
:101F5000A4002A46FFF7D2FE0A49D4F8A400FFF7EE
:101F60008BFA94F8A83013B1012384F8A93002B099
:101F700070BD00BF8095002034900808D5940808F3
:101F800075140108419008080EB400B584B005AB83
:101F9000019053F8042B0649039301A8FFF7AEFE06
:101FA000019B00221A7004B05DF804EB03B0704787
:101FB0009D0E01082DE9F043002483B006460480FD
:101FC00021463046013440F015FB082CF8D100239F
:101FD000DFF8688086F8EA30C6F8EC30C6F8F030F2
:101FE000C6F8F430C6F8F8301F46FC3699463A4633
:101FF000414601A8FFF7C8FF3546032401AA12F89D
:10200000013B6BB1013C05F8013BF8D10137082FCA
:1020100085F8009006F10406E9D103B0BDE8F0832D
:102020002846224620212544013768F08EFE082FDD
:1020300085F8009006F10406D9D1EEE7CC4A0808ED
:10204000F7B5114E07463046002300F8AA3F0C466C
:102050000E4B0F49002F08BF1946154668F07DFE4C
:102060000C4F04EB4505AA36AC4202D10A4803B036
:10207000F0BD394634F8022B6846FFF785FF694604
:10208000304668F06AFEEFE7809500204E90080821
:1020900045900808579008082A960020F7B50C4E7E
:1020A0000C4F002306F8DB3F044600EB4105AC4231
:1020B00002D1094803B0F0BD394634F8022B684616
:1020C000FFF762FF6946304668F047FEEFE700BF62
:1020D0008095002078DC08085B960020F8B5084F52
:1020E0004E1E054601F11F0416F8012F28463946F9
:1020F000FFF74AFFA64205F10205F5D1F8BD00BF82
:102100005C90080803685A1C026019700368090A89
:102110005A1C02601970704702681146531C036014
:1021200011F802CB0160D31C5178036093781B0433
:1021300043EA0123111D0160D07843EA0C0343EA0E
:1021400000607047A0F13003092B07D920F0200070
:10215000413819288CBF00200120704701207047AA
:10216000303809288CBF00200120704741381928D9
:102170008CBF002001207047613819288CBF0020D7
:1021800001207047202805D0093804288CBF002082
:102190000120704701207047A0F14103192B98BF1F
:1021A00020307047A0F16103192B98BF2038704789
:1021B00010B500F100440246013C04E0B3EB0E0010
:1021C00015D1A24214D012F8013BA3F14100192805
:1021D00011F8010BA0F1410C98BF2033BCF1190F8D
:1021E00000F1200EEAD91B1A04D10028E9D110BD54
:1021F000002010BD184610BD02B310B584468418E7
:1022000004E0B3EB0E0014D1A44513D01CF8013B3D
:1022100011F8010BA3F14102192AA0F1410298BF64
:102220002033192A00F1200EEBD91B1A04D1002803
:10223000EAD110BD002010BD184610BD10467047F1
:1022400070B5044608460D4666F032F9064602E0CF
:1022500014F8013F43B1204632462946FFF7CCFF30
:102260000028F5D1204670BD1C46204670BD38B50B
:1022700007490546FFF7E4FF0649041E284618BF34
:102280000124FFF7DDFF08B144F00204204638BD09
:10229000619008081FA708082DE9F041044686460A
:1022A0009EF800C0BCF1200F7046ACF109050EF19C
:1022B000010EF5D0042DF3D9BCF12B0F5BD0BCF18E
:1022C0002D0F3BD1102A4FF0010600F1010E58D11D
:1022D0009EF800C0BCF1300F5FD04FF010086FF0D7
:1022E00070450F2742460EF1010E00200DE0ACF1C3
:1022F000300C5FFA8CFC94450FDA854274462DD37E
:102300002AD008FB00C01EF801CBBCF1390FEED972
:102310004CF0200CBCF1600F0BD801B10C600EB377
:1023200023B1B0F1004F28BF4FF000404042BDE85C
:10233000F081ACF1570C5FFA8CFCDCE7102A864682
:1023400049D04FF0FF35B5FBF2F502FB05F7FF432F
:10235000FFB290460026C6E76745D2D21E404FF036
:10236000FF30D0E7002BE2D06FF00043984228BF47
:102370001846BDE8F081102A4FF0000600F1010E6A
:10238000A6D04FF0FF35B5FBF2F502FB05F7FF4392
:1023900090F801C0FFB29046A5E79EF801C0ACF1ED
:1023A000410019280EF10104624601D80CF1200207
:1023B000782A4FF0100805D0A6466FF070450F2719
:1023C000424690E79EF802C06FF070450EF1020E93
:1023D0000F27424687E700267AE700BF01230A223B
:1023E000002159E770B50D461446FFF757F8064629
:1023F000A0B1FFF7F3FF40F634039842A8BF184698
:10240000B0F5617FB8BF4FF46170A0F5617319201A
:10241000B3FBF0F32B702378013323703046FFF7C2
:102420003DF80646A0B1FFF7D9FF40F634039842C5
:10243000A8BF1846B0F5617FB8BF4FF46170A0F532
:1024400061731920B3FBF0F36B70237801332370B1
:10245000304670BD10B40288C378174CA2F5FA62FA
:1024600002F0030140F2B55C9208013B0CFB023321
:10247000827801EB4101013A02EB810204EB420157
:1024800002798C8F4179234403EB430302EBC303AE
:1024900084790A4A0089C3EB031301EB8303C3EB7E
:1024A0000313224402EB830200214FF47A73C2FB30
:1024B00003015DF8044B704730CD070880436D3849
:1024C0002DE9F04117461E4605464FF47A72002367
:1024D0003846314666F0B0FC4349444A014482FB29
:1024E0000143C8170B44C0EB631382FB03021A4479
:1024F000D8173F4CC0EB621284FB02044FEAE27C27
:102500003C48CCEBA40C80FB0C404FEAEC74C4EBD1
:10251000E010C3EB0314A1EB8401A971C2EB02111B
:10252000A3EB81036B710CEB4C03A2EBC30240F2F3
:10253000B55303FB10CCBCF5896F2A714FEA8000BC
:1025400044DA40F2DA239C4547DCBCF5B77FB4BFE0
:1025500000220122284B02EB420103EBC1034FEAA8
:102560004208B3F8523091B2244C08EB020E04EB4F
:10257000CE0416344FF00B0E01E034F8023D6345F3
:102580001FDDBEF1010EF8D11B4B424403EBC2022A
:102590004FF0010E938F85F802E000F5FA600CF120
:1025A000010C0844ACEB030C288085F803C04FF401
:1025B0007A7200233846314666F03EFC2A81BDE837
:1025C000F0810EF1010E5FFA8EFEE4E7032140F286
:1025D00096530A464FF00608C6E7022140F2294307
:1025E0000A464FF00408BFE780BC92C789888888F4
:1025F000ABAAAA2A73B06D1630CD07086CCD0708B8
:1026000008B50C4BD3E9002352EA030C09D100238F
:1026100040F2011242808380837103800381184657
:1026200008BD054909688A1843F10003FFF748FF10
:10263000012008BD784100206427002090422DE948
:10264000F0410B46044615460AD2B0FBF5F6134A94
:1026500005FB16441846135D00F8013BBDE8F08108
:10266000B0FBF2F69642B6FBF2F706D20B4A05FB38
:102670001767D15D03F8011BEAE7BA42B7FBF2F82E
:1026800007D9064A05FB187812F8081003F8011B51
:10269000EDE74046FFF7D2FF0346F2E7D44A0808C9
:1026A00030B5874CB4F81034B4F81404B4F81614E8
:1026B000B4F81824B3F57A7F84BF4FF47A73A4F882
:1026C0001034B4F81234B3F57A7F84BF4FF47A73C0
:1026D000A4F81234B0F57A7F84BF4FF47A70A4F86E
:1026E0001404B1F57A7F88BF0021B4F81A3488BF8A
:1026F000A4F81614B2F57A7F84BF4FF47A72A4F866
:102700001824B3F57A7F84BF0023A4F81A348842D2
:102710009CBF0021A4F814149A4298BF0023B4F877
:10272000262498BFA4F81834B4F828349A4284BFF9
:102730000023A4F82634634B1B8883B02BB3627A42
:10274000614D012A48D9AA78062A97BF5F499FEDB3
:10275000607A01EB820191ED277A2979002940F016
:102760008A8094F8301407EE903A06EE901AF8EE4C
:10277000E77AB8EEE66AAB79C6EE276A002B72D12B
:10278000B4EEE67AF1EE10FA37DC6379032B14D855
:10279000504AC3EB031302EB43022379C4F83824F5
:1027A000032B12D84C4A03EB830103EBC10302EB6A
:1027B0008303C4F83C3403B030BD00236371237934
:1027C000444AC4F83824032BECD9434BC4F83C34B6
:1027D0000022227103B030BDAA79002AB3D0AA78B2
:1027E000072A2AD0B3F57A6FAED994F830140229AB
:1027F000B8BF022184F83014A6E767EE277ABCEE52
:10280000E77A8DED017A9DF8042007EE102AB8EEE4
:10281000C77AF4EEC77AF1EE10FAC4BF0132D2B231
:10282000002A3CD0102AA8BF1022D2B28A421346F6
:1028300038BF0B4684F83034A7E70622B3F57A6F29
:10284000AA702ED82A79002A9FD194F8301407EE66
:10285000903A07EE101AF8EEE77AB8EEC76A9FEDE5
:102860001F7AC6EE276A37EE077AB4EEE67AF1EE03
:1028700010FA8ADDC1E7042A02D8002A85D002E0D6
:10288000053A032A81D9B7EE000A80EE070A67F0FD
:1028900081FC2B88984228BF1846288075E70122C2
:1028A000C3E794F830242979022AB8BF022284F8B9
:1028B000302400297FF469AF9FED087A51E700BF0B
:1028C00080950020C00A0010942D002030CD07080C
:1028D0006F12033884960020FC96002017B7D13879
:1028E0002DE9F04FB24E85B096F84034A3F11702AF
:1028F000022A00AF00F2DA82AE4BBB60DFF8D8925A
:1029000096F85814DFF8D4B2AB4D09F16C0A4C4676
:102910004FF0000834E010F0010C4ED1142A00F002
:10292000C1824308820802F0333203F07733134444
:10293000C20802F01132C31A9B1A03EB131303F0FF
:102940000F33ABFB03E2D209C2EB02229A1A8303D4
:1029500002D5012A00F0A682012A0ED9082A00F227
:10296000A182BCF1000F01D0284206D1F96064F0C9
:1029700005F9F968002800F095820C34544521D0FF
:1029800094F904202068A2F11E03DBB2012BC2D807
:10299000A379022BA8BF0223A371E379022BA8BF5E
:1029A0000223E371237A022B20F04100A8BF022307
:1029B000206023724FF0000CB3E708F101085FFAC2
:1029C00088F8AEE708F1FF38B8F1020F00F26A822A
:1029D0000024022086F8F84415F078F896F8FC34C4
:1029E000022B00F00D83002800F07483734B96F8DF
:1029F000C98503F5247B4FF47A7E4FF0000C5A888A
:102A0000B2F57A7FB3F8462088BFA3F802E0B2F5AA
:102A10007A7F9A8888BFA3F846E0B2F57A7FDA8891
:102A200088BFA3F804E09988B2F57A7F84BF0022BA
:102A3000A3F806C09142B3F85A10B3F85C2098BFCF
:102A4000A3F804C0914293F86B2088BFA3F85AC042
:102A5000013A632A84BF642283F86B2093F86C20C8
:102A60000132D2B2092A88BF83F86CC003F1660034
:102A7000194600228D7A10F8014B0132A54238BF69
:102A800000F801CC032A01F10601F3D1B8F1010FDE
:102A900018BF83F885C0A4339B45B0D1484B9B78C1
:102AA000042B00F0EA823BB9454A1388B3F5F07F66
:102AB00084BF4FF4F0731380FFF7F2FD414896F89E
:102AC000DC15FEF7E3FB96F8FB151030FEF7DEFB96
:102AD00096F809160E30FEF7D9FBB6F81626B6F8AA
:102AE00014361343B6F8182613431BB213B101234F
:102AF000A6F81A36D6F8B835334A1A40002A00F03C
:102B0000FF82D80700F15982590440F1ED812F4925
:102B1000D6F8BC250B400A40C6F8B835C6F8BC2527
:102B20009C0408D52A49D6F8BC250B400A40C6F8B3
:102B3000B835C6F8BC25180440F12182002286F879
:102B40005F2486F86F24D90440F1248296F8273652
:102B5000DFF880B0022B04BF012386F827360BF183
:102B600078045B4602E00633A3420CD01A78072AA9
:102B7000F9D19978DA78914202D35A79002AF2D0C1
:102B8000072026F051F800234FF4806086F8F834CF
:102B900014F09CFF002800F08A820E4DA84698F899
:102BA000051041B398F8000018B35B461BE000BF66
:102BB0008095002030CD0708BC020200FC96002062
:102BC000942D00206C9B002009600002F6DFFFFDC1
:102BD000F6BFFFFDAC9B0020089A0020818080801A
:102BE00006339C4207D01A788A42F9D15A79002AD2
:102BF000F6D026F019F808F106084445CFD1BC4BB1
:102C000093F802B0BBF1080F00F0E58196F8C935E2
:102C1000A3F10103B3FA83F35B0986F8A43696F8AF
:102C2000CA35A3F10103B3FA83F35B0986F8A8362A
:102C3000D6F8BC3513F00072C3F3C03106D096F855
:102C4000B826A2F10802B2FA82F252090A4386F8C3
:102C5000A62696F80D24B17C032A84BF002286F8AC
:102C60000D24D6F8B82523F4005322F40052C6F8F8
:102C7000BC35C6F8B825002900F0E681B6F8CC3698
:102C8000002B40F0ED81D6F8D03613F07F4F1CBFFB
:102C90000023C6F8D036D6F8D83623F4007323F0D4
:102CA00002031BB140F20223C6F8D83696F8D43698
:102CB000013B042B84BF012386F8D436ABF1050B0E
:102CC0008C4BBBF1030F93F8901540F24F8111B379
:102CD0000023FB60864B7C606FF00702A2EB0308C9
:102CE000444603F1080B884604E004EB0B039845C7
:102CF00040F212811BF8010B0028F6D010F034F9D5
:102D00000028F2D083799B07EFD5FA687C6801230D
:102D1000002A40F00781764B9B7913B1744A002357
:102D20009371B6F8E23613F00C0F03D1C3F303131B
:102D3000022B03D94FF42063A6F8E236B6F8E43646
:102D400013F00C0F03D1C3F30313022B03D940F686
:102D50000123A6F8E43696F8613796F855279A428B
:102D600096F8543705D9002286F8552753B1A6F8AE
:102D7000582796F860279A4204D2002386F85437E1
:102D8000A6F8583796F84A3896F856275A49FC60FC
:102D90009A4288BF0023BC6888BF86F8563701F185
:102DA000780B11F8013C03EB430323444FF0030875
:102DB00093F870E293F871C293F872020B461A7896
:102DC0007245A8BF724603F8012B5A796245A8BF25
:102DD00062465A719A788242A8BF0246B8F1010849
:102DE0009A70ECD11E318B45DBD1D6F88024FC687B
:102DF000002A00F02381002001212B78282B07D105
:102E00006B78043301FA03F313421CBF9A43012089
:102E10000635AC42F1D108B1C6F88024374D05F132
:102E200008042B4613F8012B072A00F288809C42E5
:102E3000F8D1EB4688B06B46FF211846202267F098
:102E400084FF2E49034611F8012B53F8220001306C
:102E50007CD18C4243F82220F5D1B6F8C225B6F8D1
:102E6000C0359A42DD4602D3254BC6F8C035FF2354
:102E7000244986F87C3899F90430142B05D0D9F808
:102E8000002031EA020200F0F58009F10C09D14579
:102E9000F1D11D4B5A79022A00F0A8801437BD46A3
:102EA000BDE8F08F194811F0C1FC91E5184ABA60ED
:102EB0001146DA0001EBC30393F8B81021B1D3F83F
:102EC000BC30002B00F0EF80BB68134493F8B920AE
:102ED000002A3FF413AD93F89831002B7FF40EAD28
:102EE000182386F8403409E51A076FD509491AE610
:102EF000942D0020C00A001087960020A72D0020E6
:102F0000AE014A010100020088410020089A002019
:102F100030CD0708FE9FFFFDFA687C680023002A79
:102F20003FF4F9AE7C494A7C002A7FF4FAAE4A7934
:102F3000012A3FF4F0AE002B7FF4EDAEF1E6EB4654
:102F400088B02022FF21684667F0FFFE05F8018B5C
:102F500008F10108B8F1080F3FF47FAF05F8018BC5
:102F600008F10108B8F1080FF0D176E76A4A0023AA
:102F70001371002900F0BB800123FB60AAE696F8DC
:102F80005F24002A00F0A0800022D90486F86F2474
:102F90003FF5DCAD1A067FF5D9AD96F84014182937
:102FA00006D85E4B01228A401340002B7FF4CEAD41
:102FB000DFF87CB10BF17804E5E55949D6F8BC257A
:102FC0000B400A40C6F8B835C6F8BC259D017FF510
:102FD000A7AD5449A7E51A469B79002B3FF416AEDE
:102FE000537C012B04BF022353740FE696F8842808
:102FF000002A7FF453AF14375A71BD46BDE8F08FF5
:1030000000283FF4F3AC484B96F8491590F904506A
:103010004FF0FF0C03F16C0093F90820AA4204D191
:10302000013983F808C0C9B201240C338342F3D1BB
:10303000002C3FF4DBAC86F84915D7E4282025F0B6
:10304000F3FDD6F88024D6E638490B43C6F8BC35E4
:10305000B6F8CC360A43C6F8B825002B3FF413AEB9
:1030600096F8C8060FF080FF00287FF40CAEA6F893
:10307000CC0608E686F87C380BE7D6F8B835264A41
:1030800023F48053C6F8B835D6F8BC3523F4805302
:10309000C6F8BC35538CB3F57A7FBFF40DAD4FF451
:1030A0007A73538408E5172386F840340CE7D6F882
:1030B000B83523F00063C6F8B835D6F8BC3523F030
:1030C0000063C6F8BC3568E542F2010213427FF4A2
:1030D0005BAF38E5D6F8B825D6F8BC3522F08002CB
:1030E00023F08003C6F8B825C6F8BC357EE4537CCF
:1030F000002B7FF416AE5379012B7FF412AE0AE653
:10310000D6F8BC2543F0080342F00802C6F8B835EB
:10311000C6F8BC25F5E400BF942D00200041000155
:10312000F79FFFFDF69FFFFFCC9A00202006370097
:10313000AC9B00202DE9F04F884F97F88838013B71
:10314000012B83B040F2F280D7F8BC28844B02F206
:10315000DC52C7F8BC28834A934280F0FB8003F11D
:103160001C059B46804B814E4FF0010A03F102087B
:103170007D4B5A88002A00F0C28008EB0203B3425C
:1031800080F0BD80444608E01A881C461344002A9B
:1031900000F0B580B34280F0B280052A40F2AF80E3
:1031A00035F81C2C6188C2F30B029142ECD1627994
:1031B0009207E9D1238855F8141C94F804900193E0
:1031C0005846FEF745FA35F81C2CB9EB123F00F0D3
:1031D0009E804FF0000A35F8181C55F8140CC1F306
:1031E0000B015FF0D7FE55F8043C18605D4B0BF106
:1031F0001C0B9B4505F11C05BAD3D7F8B835C7F8A9
:10320000BC35FFF76DFB3B79594D5A4C03EB8302FC
:1032100003EBC2037A79A5F17801C2EB021201EB4C
:10322000420205EB8303C7F83824C7F83C3424F086
:103230006BFF4FF0FF33D7F83C04636032F03EFF82
:1032400025F046FD05F5966305F5A56102E0063318
:103250008B4266D01A78002AF9D19D78D8788542B9
:1032600002D358790028F2D097F82436227203EB63
:10327000830303EB83039B00632BD8BF6423B7F85E
:103280002826C7F8B438642303FB02F2632AD8BFA8
:103290001A463949CCBFC7F8B828C7F8B838C7F8B4
:1032A000D0280023354AC7F8BC38C7F8C038C7F85B
:1032B000C438C7F8C838C7F8CC38A7F8D43887F866
:1032C000D638C1F8402735F0AFF997F8DA18B7F8D3
:1032D000D80826F083FB42F01BFB1AF073FD97F829
:1032E0008838013B012B2DD9254A1268C7F8BC2824
:1032F0000123504687F8D53803B0BDE8F08F55F864
:10330000141C5846FEF7A4F94FF0000A63E7019B2E
:10331000A11D9A1F5846FDF7FFFB00287FF45BAF05
:1033200057E7FA7C003A18BF01229DE70AF000FA3D
:1033300000F5B71000F558700223C7F8A80887F801
:10334000AC3801E70AF0F4F90223C7F8A80887F8B7
:10335000AC38C9E74FF0010A4FE700BF8095002065
:10336000B8E10808E4EB0808004000080080000805
:10337000FC960020B0060020C00A0010949B00209C
:10338000642700201C4B0122032870B51B4D83F8D5
:10339000482706461ED9711CC9B249004029184A5F
:1033A00028BF4021002302244FF0140ED4540233CE
:1033B00002EB030C99420CF801ECF7D8FF2E08BF82
:1033C00002212944FF2381F8DC38BDE870400E203B
:1033D00014F0FEBC00EB800005F5BE7306EBC000E8
:1033E00003EB8000C5F83C042E7132F067FE26F036
:1033F000ABFE26F07FFFCEE7C00A001080950020CC
:103400005C9E0020054BD3F82029012142F40012D4
:1034100083F81D19C3F82029704700BF809500204C
:10342000F8B50468C4F30D0406460F460CB33568BE
:103430003F6856F09FF8092840F08780444C236984
:1034400023F440732361236943F4007323612369E8
:1034500043F0010323612F6056F08CF8236909289B
:1034600023F00103236170D13368043333600020FB
:1034700034E0384B384A93422AD302F580429342D3
:1034800025D302F58042934229D3344A934228D966
:1034900002F58032934226D902F50032934224D9B4
:1034A00002F50032934222D902F50032934220D92C
:1034B00002F5003293421ED902F5802293421CD9B4
:1034C000B3F1016F1BD305200FF0E6FBFBE70824E7
:1034D00056F050F8092814D04FF0FF30F8BD1024F2
:1034E000F6E71824F4E72024F2E72824F0E7302454
:1034F000EEE73824ECE74024EAE74824E8E75824DC
:10350000E6E7134D2B6923F440732B612B6943F4D9
:1035100000732B612B6923F0F8032B612B691C438B
:1035200044F002042C612B6943F480332B6156F084
:1035300021F82B6923F002032B612B69092823F062
:10354000F8032B613FF473AFC6E76FF00100C5E7E6
:10355000003C02400040000800400008FFFF000857
:103560002DE9F041574F3B78B12B8AB06FD1FEF770
:10357000C1F880F00104E4B2534B544DB3F87F32EC
:10358000534EADF8003004F00104B54261D3002C75
:1035900000F096801022002106A867F0D6FB4D4B64
:1035A0000497DB1B05934C4B1A69002A04DA4B4A3B
:1035B0005A6002F188325A6001228DF82420F322E9
:1035C000DA606946022204A80025089564F0B2FB7F
:1035D000022269464FF6FF70FEF76EF83B4F044635
:1035E000B74243D3022201A904A80025ADF8045034
:1035F00064F0A0FB022201A92046FEF75DF840BA64
:10360000C043ADF80800022204A802A964F092FBAE
:10361000079868B106ABC0F104022946184467F068
:1036200094FB089818B906A904A8FFF7F9FE0890BA
:103630009DF82430089823B1274A136943F00043CA
:103640001361B0FA80F040090AB0BDE8F0810124AE
:1036500092E7A988A868C1F30B015FF09BFCAB69F6
:103660001B681C35834218BF01248EE7B7F804801D
:103670008DF80D50C8F30B0808F10603ADF80830BB
:103680003B88C3F30B02ADF80A201B0B062202A9EC
:1036900004A88DF80C3064F04DFB062202A92046E8
:1036A000FEF70AF8B9680446424604A864F042FBF3
:1036B000B96820464246FDF7FFFF1C3704468FE7F6
:1036C0000120C1E70040000830CD0708B8E1080834
:1036D000E4EB080800800008003C02402301674535
:1036E00010B5264CFFF7FCF894F88838013B012B05
:1036F00030D9D4F8BC38012203F2DC53C4F8BC380A
:1037000084F82429FFF72CFF10B9FFF729FFE0B157
:103710001B4B1B78B12B02D1FDF7ECFF10B9052034
:103720000FF0BAFA94F88838013B0022012B84F894
:1037300024291BD9134B01221968C4F8BC18002393
:1037400084F8D52884F8253910BDFFF709FF002833
:10375000DED1E4E709F0ECFF00F5B71000F5587092
:103760000223C4F8A80884F8AC38C2E709F0E0FFE7
:103770000223C4F8A80884F8AC38DBE78095002061
:10378000004000086427002008B5044B5B6A984796
:10379000034B01229A74BDE80840A1E7B00600205F
:1037A0008095002038B50C4A0C4B0D4C5B6A012506
:1037B00082F848579847A574FFF792FFFFF7BAFCC5
:1037C000FF2341F20242A4F8DC2884F8DE380E2000
:1037D000BDE8384014F0FCBAC00A0010B006002062
:1037E0008095002090F88730DFED6A5A03EE903A1A
:1037F00090F88B3006EE103A90F8893004EE103ACB
:1038000090F88A30F8EEE33A04EE903A90F88D3072
:1038100063EEA57AB8EEC66A03EE903A26EE256A04
:10382000B8EEC44AF8EEE44AF8EEE33A26EE276A28
:1038300024EE254A64EEA54A63EEA53AF0B5564D4E
:1038400024EE064A64EEA74A63EEA73A0021062654
:10385000F7EE002AA5F10C0C00F1660E06FB01F252
:10386000B7EE005AAC1890F886700244F0EE456A44
:1038700015E0012904F1060402F10602EED190F8E8
:10388000883007EE903A90F8903006EE903AF8EED5
:10389000E77AF8EEE66A27EEA55A66EEA56A23787F
:1038A00007EE103A66EE867AB8EEC77A27EE277AE8
:1038B000FDEEC77A17EE903AFA2BA8BFFA2323EA57
:1038C000E3731372637807EE103A66EE847AB8EE0B
:1038D000C77A27EE277AFDEEC77A17EE903AFA2BD1
:1038E000A8BFFA2323EAE37353725CF8213007EE92
:1038F000903A002BF8EEE77A49DDA37807EE103A0C
:10390000B8EE477A90F88C3037EE677A03EE103ACB
:1039100087EE272AB8EEC33AB0EE627A23EE253A54
:10392000A2EE037A64EEA77A66EEA36A67EE857A62
:1039300027EE877AFDEEE77ABDEEC77A17EE103AEA
:10394000FA2BA8BFFA2323EAE373937217EE903A97
:10395000FA2BA8BFFA2323EAE3730EF80130A388F9
:1039600007EE903AF8EEE77A013167EEA67AFDEEBF
:10397000E77A17EE903AB3F57A7FA8BF4FF47A73DF
:1039800023EAE3738F429381BFF673AFF0BDB7EEC6
:10399000007AC7E70AD7233C50D2070890F88E3048
:1039A0006BB3B0F85A308BB190F88F2002EB8203E2
:1039B0006421C3EB0313B3FBF1F3A0F85A30962351
:1039C00012FB03F3B3FBF1F3A0F85C3043884BB177
:1039D00090F88F3003EB8303C3EB03136422B3FB34
:1039E000F2F34380B0F846304BB190F88F30962216
:1039F00013FB02F36422B3FBF2F3A0F846307047E6
:103A000090F821304BB3438B83B190F82230FA22E7
:103A100013FB02F203EB8303B3F57A7FA8BF4FF4E5
:103A20007A7364218383B2FBF1F24283838843B1CA
:103A300090F82230FA2213FB02F36422B3FBF2F374
:103A40008380C3884BB190F8223003EB8303B3F536
:103A50007A7FA8BF4FF47A73C380704770B50B4C60
:103A6000002504F5247694F8863013B12046FFF73C
:103A7000B9FE2046FFF792FF01353046FFF7C0FF41
:103A8000042D04F1A404EED170BD00BFFC9600200B
:103A9000034B53F8EC0C08B107F070BD704700BF42
:103AA00078A6002008B50B460549024651F8EC0CF3
:103AB00028B10449FEF722F9BDE80840E8E708BD4F
:103AC00078A6002075140108024B014653F8EC0C4F
:103AD000FDF7D2BC78A6002008B504460848FFF7D9
:103AE000F3FFFFF7D5FF074BD3F89C0014F0EEF877
:103AF0000EF0E0FE012C01D162F086FBF8F7BCFF6E
:103B000069900808809500200048DDE7209C08089F
:103B10000CB4C30607B500D561B9049805A9019195
:103B2000FFF7C0FFFFF7F0FF012003B05DF804EBE3
:103B300002B070470020F8E708B5FFF7C5FFBDE801
:103B40000840E1E710B504460348FFF7BDFF2046F3
:103B5000BDE81040F0E700BF7590080808B50848B8
:103B6000FFF7F0FFFFF794FF064B002403F8E84C43
:103B70009C611C7726F0F6FC2046FFF7ADFF00BFE6
:103B80007A90080878A60020034B014653F8EC0C05
:103B900008B107F0DFBC704778A600200CB407B569
:103BA00010F020000BD079B92320FFF7EDFF049827
:103BB00005A90191FFF776FFFFF7A6FF012003B0EB
:103BC0005DF804EB02B070470020F8E70FB407B5CA
:103BD00004A951F8040B0191FFF764FF03B05DF8ED
:103BE00004EB04B0704730B52B4885B0FFF76CFF8D
:103BF0002A4B93F8843823B9294805B0BDE83040F2
:103C00009AE7FBF70FFC08B92648F6E7FBF722FC1A
:103C100008B92548F1E7254B1B68DB699847002860
:103C2000F7D0FBF719FC0268037D81790446407CDC
:103C30000290207C0190608A009052081C48FFF797
:103C4000C5FFE51D0C3415F8010BFFF79DFFA542DC
:103C5000F9D1184C1848FFF737FF6378022B06D0CC
:103C600007D9032B10D11548FFF72EFF0CE014489D
:103C7000FAE704F580541348FFF726FF94F8E43779
:103C8000022B05D0032B05D005B0BDE830403BE743
:103C90000D48E9E70D48E7E7A19008088095002066
:103CA000AB900808BA900808C8900808BC4A0808F1
:103CB000D79008086047002005910808159108086A
:103CC0001B910808289108082E91080847910808B8
:103CD000154B1B6870B52BB31448154EFFF72CFF1E
:103CE000FFF7D6FEFAF70AFE0025FAF737FE04467C
:103CF00040B1132014F06CF8FFF706FFBDE87040E8
:103D00000C4819E73046FFF761FF782D06D80135DA
:103D1000FFF7BEFE64200EF01FFEE6E7FFF7F4FE9D
:103D20002546F5E770BD00BF1C2700205991080803
:103D3000A2C20808739108080FB407B504A951F886
:103D4000040B0191FFF7AEFEFFF7DEFE03B05DF856
:103D500004EB04B070472DE9F041037903F0E00271
:103D6000402A50D004D85AB1202A29D0BDE8F08189
:103D7000602A4BD0802AF9D182794179254812E016
:103D800003F00703052B16D8DFE803F01015101514
:103D90000309D0F805102048BDE8F041CCE7D0F881
:103DA000052051421D48BDE8F041C5E7B0F80720A5
:103DB000B0F80510F6E7B0F90720B0F90510F1E703
:103DC0004679174D174805EBC605FFF77DFE95F8B8
:103DD000387500240123A74202D8BDE8F04193E6DC
:103DE000D5F8346556F824204FEA84084AB113B94F
:103DF0000D48FFF769FE56F808100C48FFF7E6FE7D
:103E000000230134E7E741790948C5E7BDE8F041FF
:103E1000084891E7C8910808799108088F91080827
:103E200030CD0708A69108081E950808C6A5080801
:103E3000B7910808DF9108082DE9F04387B0FAF739
:103E40003DFB02698389018802928268019242885F
:103E5000009242681B4EDFF880801B4FDFF87C9099
:103E600004461A48FFF768FF002515B94046FFF7DA
:103E700063FE3B689D4213DA33781548052B96BFE5
:103E800009EB83030022D3F81C27B388009329464B
:103E900073880135FFF750FF062D06F10606E4D1C1
:103EA00060F050FB81884388CB1A616803FB0111E5
:103EB0000591FAF797FD05990246064807B0BDE857
:103EC000F04339E7B8400020DC400020F7910808B3
:103ED00061920808709208085592080830CD0708CA
:103EE0000249034801F521610EC925E70070FF1F53
:103EF0008D92080810B57521044637F017FA01466F
:103F00000948FFF719FF1A21204637F00FFA01463A
:103F10000648FFF711FF1B21204637F007FABDE8DE
:103F200010400146024807E7A1920808B492080829
:103F3000C792080838B50C4D95F80F0410F0FD0431
:103F400005D10A48FFF7F8FE2046FFF7D3FF95F8A2
:103F50000F34013B012B06D80548FFF7EDFEBDE805
:103F600038400120C6E738BD80950020DA92080865
:103F7000E59208082DE9F04F2DED028B794B7A4937
:103F80001A687A4BB2FBF3F299B008EE100A78483F
:103F9000FFF71CFE774BDFF850C20FCBDCF8087040
:103FA0000CAD85E80F00744B0793BC08734B089366
:103FB00014F00204C7F3810718AB18BFDCF80460E3
:103FC00003EB870318BFC6F3805653F8301C002C50
:103FD00000F0C58018AB03EB860353F8442C684C03
:103FE0006848694D694EDFF80482DFF8C8A1FFF721
:103FF000EDFDE28B4FF47A73B2FBF3F103FB112278
:104000000A20B4F9203092B2B2FBF0F26048FFF718
:1040100093FE604A60496148FFF7D8FDFFF774FDE1
:10402000A97C5F4A5F4B604806EB8101D31AD1F847
:104030004417B5F8A220FFF77FFE5C48FFF744FD68
:1040400094F822105A48FFF7C1FD5A48FFF73CFD8B
:1040500094F823105848FFF7B9FDFFF755FD57486E
:10406000FFF732FD00210A4695F82B340B4113F07F
:10407000010F01F1010708D012B15046FFF724FDEE
:1040800039464046FFF7A2FD0122072F3946EBD102
:104090004B4F97F86A1507F5EC7307F13C020129BD
:1040A00018BF134693F8DC30032B02D04548FFF7C6
:1040B0008DFD454B97F86A15A3F5CE72012918BFFF
:1040C000134693F8DC30012B02D14048FFF77EFD08
:1040D0003D4B97F86A15A3F5CE72012918BF134618
:1040E0001B695B7B012B02D93948FFF76FFDDFF8B5
:1040F00000A1FFF709FD636A03934FF000080AF17E
:10410000200B5AF8041B002974D0012303FA08F984
:10411000039B19EA030F1FD019F01F0F1CD02D4B62
:104120005BF8282013F8080052F82020B8F1000F9F
:1041300006D02948CDE90412FFF7C6FCDDE90412D8
:104140002648FFF743FDB9F1020F05D197F86D1A24
:1041500011B12348FFF73AFD08F10108D1E7214AE0
:104160003DE700BFA0260020F892080840420F005B
:10417000FD92080864D407081A9308081F930808DA
:1041800078A60020249308088095002030CD0708E9
:104190002C930808F0FF0010000800004D93080859
:1041A000008000080040000871930808A0930808E8
:1041B000B2930808BA930808BC930808C493080887
:1041C000C00A0010DD930808980C0010E593080859
:1041D000EA930808D80600201E950808F2930808FC
:1041E000F8930808229C080800380240D493080875
:1041F0007CD40708FFF788FC95F8721ED5F8742E5A
:104200007B48137A527A06EB8101D1F88017FFF7C9
:1042100093FD784B784819684FF47A73B1FBF3F14A
:10422000FFF7D4FC09A8FEF7EBF938B109A910A8EB
:1042300063F07CFE714810A9FFF7C8FCFFF764FC2F
:10424000D4F8B020002A00F08F8007EE902ADFED2E
:104250006C6AB8EEE77AC6EE877AFDEEE77A17EE7B
:10426000903AB4F8680858B107EE900ADFED646A36
:10427000F8EEE77A86EEA77AFDEEC77A17EE900A97
:10428000216B59B107EE901ADFED5D6AF8EEE77A1F
:1042900086EEA77AFDEEC77A17EE901AB7F8A87ADD
:1042A000642FCDE9000139465648A8BF6421FFF7C5
:1042B00043FD94F86A3894F86B28B4F86C185248A7
:1042C00006EB8303D3F89437FFF736FD4F4B504886
:1042D000198889B2FFF730FD4E4918EE100AFFF732
:1042E00082FCFAF7EBF8016921B182684A48120DA5
:1042F000FFF722FD4948FFF7E7FBD5F8BC351B0661
:1043000062D594F89838032B8CBF45484548FFF791
:10431000DBFB95F8FC34022B28D14348FFF7D4FB94
:1043200094F89838042B46D84048FFF7CDFB94F812
:10433000A838002B46D006EBC303D3F8EC173C4853
:10434000FFF744FCFFF7E0FB3A4F3B48FFF7BCFBAD
:10435000D5F820490125002C3AD1FFF7D5FB19B03B
:10436000BDEC028BBDE8F08F13467AE7022013F014
:10437000CFFB074608B93148D0E741F0AFFA97F9CB
:10438000041006EB80000131D0F8A8272C48FFF775
:104390001DFC95F8FF34012B04D12A48FFF794FB4C
:1043A0002948BBE7BB79294806EB8303D3F8A81754
:1043B000FFF70CFCF4E795F8FE340BB92448B4E79A
:1043C0002448B2E72449BAE72448FFF77DFBB9E760
:1043D00094FAA4F3B3FA83F305FA03F206EB83032A
:1043E0003846D3F8201824EA0204FFF7EFFBB2E7BF
:1043F000FC930808642700200E94080828940808F5
:10440000002474493B940808819408086C2D00200E
:10441000A8940808229C0808B7940808D2940808B1
:10442000D8940808E4940808F49408086EC30808AF
:10443000319508083D9508084D950808FA94080834
:1044400004950808189508081D950808A79E0808EF
:1044500021950808AF900808F092080841950808CF
:104460002DE9F04FDFF8788198F8073099B0002BEC
:1044700000F098805148524EDFF868B1DFF868913B
:10448000DFF868A1FFF758FB00252F460BA9E8B21B
:1044900019F0F6FE9DF83430002B53D0139C54B124
:1044A00007EE904A9FED470AF8EE677A80EE270AFA
:1044B00065F070FE04460B9A29465846FFF786FBC6
:1044C000109A002A70D002FB04F04FF47A73B0FB0C
:1044D000F3F30993DDF848C0BCF1000F66D00CFB84
:1044E00004F142F21073B1FBF3F198F80730082D94
:1044F00018BF7F18002B5BD017980790159806906F
:10450000169805900A2311984FF47A7EB0FBFEFEB0
:104510000998CDF810E0B1FBF3FE03FB1E11CDE9C5
:1045200002E10999B1FBF3F103FB1100CDE90010A1
:10453000BCFBF3F321465046FFF7FEFB0023C6E920
:104540000D33B3620135212D06F140069ED198F856
:10455000073023B31C4C1D48D4F8B028D4F8AC184D
:10456000D2084FF47A73B1FBF3F3D4F8B418FFF721
:10457000E3FB0A221648B7FBF2F102FB1172FFF7C8
:10458000DBFB144B1B78432B06D1D4F8B828D4F8A6
:10459000BC181148FFF7D0FB0023C4F8B43819B099
:1045A000BDE8F08F0D4866E7099293E761469CE706
:1045B00021464846FFF7C0FBC0E700BF63950808E7
:1045C000A0A600208096184B78A600200A9608081E
:1045D0002A960808C42800204E960808C1950808A5
:1045E00080950020CB95080862A50808DA95080890
:1045F0000EB403B503AA52F8041B0192FDF790FC18
:10460000074B53F8EC3C2BB9064B0749D3F8A400F1
:10461000FCF732FF02B05DF804EB03B0704700BF57
:1046200078A6002080950020209C08082DE9F047FE
:1046300098460B7903F0E004402C81460F4616465D
:1046400031D1684DDFF8A081DFF8C091002422E06D
:104650003B7903F00703013B042B04D8DFE803F0A8
:1046600006080B0E2000315D28460AE03157FBE7B3
:1046700036F81410F8E736F91410F5E756F8241058
:104680004046FFF7A3FA7B79013BA34202DD48468F
:10469000FFF71AFA01347B79A342D9DCBDE8F08731
:1046A00056F82410E0E703F00703052B58D8DFE89D
:1046B00003F0030C141619313578602C5ED045D800
:1046C000002C66D0202C7CD0E8E796F90050602CB6
:1046D00054D03BD8002CF5D148E03588EDE7B6F949
:1046E0000050F4E7D6F800A0202C554669D02BD80E
:1046F000002CD3D151463C48FFF768FAD7F8051093
:104700008A4518D8B8F1000FC8D03848BDE8F0473E
:10471000FFF75CBA202C356853D015D8002CBDD1DA
:1047200029463048FFF752FAD7F80510A94202DBB4
:104730004B42AB42E6DDFFF7E7F93A682C492B46DE
:104740004846BDE8F04753E7602C17D0802CA5D130
:104750003178284B2848002914BF31461946D5E73F
:10476000202C2DD007D8002C98D12546B7F905402C
:10477000B7F9076011E0602CE8D100257B7945FA94
:1047800003F3DB07BDE8F0474CBF1C481C48FFF7AC
:104790001DBAB7F80540B7F8076012482946FFF779
:1047A00015FAAC42C7DCAE42C5DBB8F1000F3FF4EE
:1047B00075AF324621461348BDE8F047FFF706BA09
:1047C00000257A79104B03EBC20393F83825954204
:1047D000B1DAD3F8343553F82500BDE8F047FFF7D8
:1047E00073B900BF79DC08088C910808789608082E
:1047F0007E9608083EC30808C6A50808F491080874
:104800004FDD0808999F080830CD0708BA930808BB
:1048100013B50446084601920091FCF7BFFEDDE99E
:1048200000130246204602B0BDE81040FEE60EB47A
:1048300003B503AA52F8041B0192FDF771FB054B67
:104840000549D3F8A400FCF717FE02B05DF804EBAD
:1048500003B0704780950020209C0808014902465B
:10486000E5E700BF98960808F8B5064608460C46E6
:10487000FDF7B4FD20210546204666F07DFA04468A
:1048800018B93046BDE8F840E8E7114F114E3B78C3
:1048900032789A4201D0FAF759F90F4B20461D6041
:1048A00063F006FE012201462046FAF7F9F83B784C
:1048B00032789A4201D0FAF749F9204663F0F8FDC0
:1048C0002A460146BDE8F8400448FFF735BA00BF64
:1048D00018270020F040002014270020AF96080879
:1048E0002DE9F041064688B008460D46FDF776FDF5
:1048F00020210446284666F03FFA20B9304608B029
:10490000BDE8F041AAE7FDF769FD224605460146EC
:104910000F48FFF711FA85B1202D2A46694628BFB6
:1049200020222046FAF72EF9E84606460027B7422D
:1049300008DBAD1B3444002EEDD1FFF7E5F808B0DD
:10494000BDE8F08118F8010BFFF71EF90137EEE71B
:10495000C596080810B504460748FFF7EDF8FAF7C2
:10496000A9F920B1BDE810400448FFF7E5B820469A
:104970000349BDE810405AE7DD960808E7960808A5
:10498000EF9608082DE9F041144BD3F85C3B88B052
:104990000446F3B11A6804A9D56A18466A46A847BE
:1049A000064688B1DFF8408004AC6D46002735F834
:1049B000022B34F8021B40460137FFF7BDF9BE4217
:1049C000F5DC08B0BDE8F08105492046FFF72FFF70
:1049D000F7E7044908B0BDE8F04128E780950020DA
:1049E0001097080828970808F69608082DE9F0415E
:1049F000074608460D4663F05BFD064688B31C4C2F
:104A000094F82080B8F1000F15D0237D9BB104F1FC
:104A1000200063F04DFDB042024605D1294604F165
:104A2000200066F0CFF930B13846124B124A1349D4
:104A3000BDE8F041FBE694F8A03093B9237D13B1B3
:104A4000B8F1000F0DD115220A48294666F0CEF9BB
:104A50000B4B0C48012283F8C02883F8C128FFF7CC
:104A600071F8BDE8F04103490748FFF765B900BF99
:104A700080950020A09500202F9708083A970808F5
:104A800078A6002064970808749708082DE9F0417B
:104A9000074608460D4663F00BFD064688B31C4CDE
:104AA00094F81480B8F1000F15D0237E9BB104F167
:104AB000180063F0FDFCB042024605D1294604F11E
:104AC000180066F07FF930B13846124B124A13498C
:104AD000BDE8F041ABE694F8A03093B9B8F1000F0F
:104AE00001D0237E6BB905220A48294666F07EF97B
:104AF0000B4B0C48012283F8C02883F8C128FFF72C
:104B000021F8BDE8F04103490748FFF715B900BF98
:104B10008095002098950020829708083A97080809
:104B200078A6002092970808A79708082DE9F04377
:104B300006469BB008460C4663F0BAFC00270546C3
:104B40001C22394602A8019766F0FFF825B3402DD4
:104B500007D03A4940232A4630461BB0BDE8F0430F
:104B600065E60DF1040804F1400902222146684679
:104B700066F03CF90023102209A968468DF80270FE
:104B8000FDF78AFB099B0DF10202934223D1023407
:104B9000A14508F8010BE8D100213D220AA809919E
:104BA00066F0D3F8002D3BD0254C94F83550D5B1A4
:104BB000202204F1380101A866F09DF898B104F1B3
:104BC000380109A8FDF78AFA1E4A1F4909AB304689
:104BD000FFF72DFE04E01A781C493046FFF727FE48
:104BE0001BB0BDE8F08394F8A030CBB9C5B901ADD6
:104BF0000FCD174C0FC495E80F0084E80F00154B3C
:104C0000012209A8A4F1100183F8C228FDF766FA71
:104C10001148FEF797FF114809A9FFF78DF8DFE764
:104C20000C4B93F8C23823B9054B93F83530002B61
:104C3000F1D0074909A8FDF751FAECE7BA9708083F
:104C400080950020F89708083A970808DC9708082C
:104C5000B895002078A60020029808081198080846
:104C60002DE9F74F834608460D4663F021FC374F88
:104C70000446D7F8B895B8B93548364D364FFEF7E3
:104C800023FF012655F8041B49B106FA04F313EA81
:104C9000090F02D03846FEF799FF0134F2E703B05E
:104CA000BDE8F04FFEF730BF02462C492846FDF71D
:104CB000A3FA78B92A48274C2A4DFEF705FF54F885
:104CC000041B0029EBD00B78002BF8D02846FEF708
:104CD0007DFFF4E72B782D2B1E4B03BF013504F12C
:104CE000FF344FF0010A4FF0000A002653F8048BFE
:104CF000B8F1000F06D11C492A46584603B0BDE85A
:104D0000F04F94E52246414628460193FDF774FA98
:104D1000019BC0B90123B340BAF1000F0DD029EABD
:104D200003031248C7F8B835FEF7CEFE0D484146DA
:104D300003B0BDE8F04FFEF7FFBF49EA03030C489C
:104D4000C7F8B835F0E70136D0E700BF80950020FE
:104D50001E980808B8D5070828980808C6950808B6
:104D60002C9808083D9508083798080848980808BE
:104D7000519808082DE9F74F814608460E46174618
:104D8000984663F095FB0446E8B93F483F4DFEF76F
:104D90001DFF204612F084FC3B68184206D02046D6
:104DA00012F090FC01462846FEF710FF0134182C43
:104DB000EFD13B6813B93648FEF786FE03B0BDE875
:104DC000F04FFEF7A1BE024632493046FDF714FA15
:104DD0000546A8B93048FEF777FE2C462F4D2046F1
:104DE00012F05EFC10EA080F06D0204612F06AFCB2
:104DF00001462846FEF7EAFE0134192CEFD1DDE723
:104E000033782D2B48F0807303BF013604F1FF3453
:104E1000012500254FF0000A0193504612F052FC84
:104E20002246834601463046FDF7E6F900BB504670
:104E300012F036FC019B03421AD08DB1BAF1180F63
:104E40001CBF3B6840EA03081548C7F80080FEF71E
:104E50003BFE1248594603B0BDE8F04FFEF76CBF69
:104E6000BAF1180F1CBF3D6885433D600D48EEE761
:104E70000AF1010ABAF1190FCFD10B49324648465F
:104E800003B0BDE8F04FD2E4599808083C950808F3
:104E900063980808C69508082C9808083D950808E6
:104EA000489808085198080837980808014A40F2BD
:104EB00002235FE7589C0020014A6FF07F4359E7C7
:104EC000509C002010B50446012033F08FF920B922
:104ED00020460449BDE81040A9E4BDE8104002485E
:104EE000FEF72ABF6A9808087998080870B5054641
:104EF00008461646FDF772FA0D4B93F8902590423E
:104F0000044605D201460B48FEF716FF204670BD49
:104F10002EB1FF2803D10848FEF70EFFF6E7074938
:104F2000013A2846FFF783FC4FF0FF34EEE700BF5D
:104F3000C00A00108498080895980808A8980808DE
:104F40002DE9F04F074691B08248834D0E46FEF79B
:104F5000F3FE8249C5F8C4D8002385F8C838062274
:104F6000012391F890153046402485F8C9480DF08A
:104F700069FC0A200DF0F0FC95F8C8380C2BDAB269
:104F800040F2E4809DF80C50FE2D30D0FF2D0BBF79
:104F900015240F2401260026944240F0D780611E7C
:104FA000C9B268464EF0D2F904F140030DEB030498
:104FB00014F8413C834240F0C48006F1FF385FFAA8
:104FC00088F8B8F1010F9DF80D3012D903F01F07D2
:104FD00061375C096248FEF777FD022E6AD0013C1A
:104FE000042C65D8DFE804F00B5E606462000226E2
:104FF000D2E79DF80E709DF80F401D46EAE759482C
:10500000DFF8BC91DFF8BCB1FEF796FD5648FEF71D
:105010005BFD6C464FF0000A14F8011B48460AF18C
:10502000010AFEF7D3FDBAF10C0F49D1FEF76CFD72
:10503000022E4FD06422B5FBF2F102FB11524B4815
:105040003B46D2B2C9B2FEF777FEB8F1010F71D874
:10505000474A484B9DF810104748484D002914BF57
:1050600011461946FEF768FE9DF81110444B45485D
:10507000002914BF19462946FEF75EFE022E59D1BB
:105080009DF812404048FEF71FFD4CB3FF2C37D06F
:105090000A22B4FBF2F102FB11423C48D2B2FEF705
:1050A0004BFE20E03A48ABE73A48A9E73A48A7E781
:1050B0003A48A5E700238DF83F300DF11F009FE728
:1050C000374B03FB0AF2B2F1553FA5D85846FEF71D
:1050D000FBFCA1E733483A462946FEF72DFEB7E729
:1050E0002846FEF729FD9DF813402F48FEF7ECFCFB
:1050F00044B1FF2C21D02D482146FEF71DFE04E0CF
:105100002B48EEE71D48FEF717FD1C4E284FDFF831
:1051100070800DF11305002415F8013F7BB1FF2BC2
:105120000CBF3A464246214622480134FEF704FEAF
:10513000042CF1D111B0BDE8F08F1D48E3E73246F1
:10514000F1E71D493846FFF772FBF3E71B48FEF70E
:10515000F3FCEFE7EE98080878A60020C00A0010DC
:10516000FF9808080A990808309908084299080821
:10517000CE980808D798080879990808DE98080892
:10518000F2A608089099080897990808AB990808AA
:10519000119908081999080821990808F092080837
:1051A000ABAAAAAA5E990808B399080879DC08088E
:1051B000E2980808C3990808CE990808DE990808FB
:1051C0005C9008083EC308082DE9F84FDFF8A88076
:1051D000DFF88890DFF8A4A007460C46204663F06D
:1051E00067F9064660B91D4B1D4893F840241D4BD6
:1051F00003EB8203D3F80019BDE8F84FFEF79CBD1E
:10520000024641462046FCF7F7FF60B1DFF860B088
:1052100000255BF8041BB1B9224638461249BDE8A7
:10522000F84FFFF704BB1148114C124DFEF74CFC30
:1052300054F8041B19B12846FEF7C8FCF8E7BDE88E
:10524000F84FFEF761BC32462046FCF7D5FF01352A
:105250000028DED189F840545446BFE780950020ED
:10526000E799080830CD0708379808082C980808EF
:1052700034D607083D950808C6950808229C0808FA
:1052800038B50D4604461A4905222846FCF7B4FFF6
:1052900068B9184B93F8A82022B9012183F8A81007
:1052A00083F8A920BDE838401348FEF745BC1349F0
:1052B00003222846FCF7A0FFA0B90E4D95F8A830B0
:1052C00063B195F8A9304BB10D492046FFF7AFFA0D
:1052D000002385F8A83085F8A93038BD0948FEF7C5
:1052E0002BFCF5E720460849BDE83840FFF79FBA98
:1052F00049A6080880950020F19908089BA708088E
:10530000079A08083E9A0808529A0808F8B5224CED
:1053100094F8A83005467BB194F8A93063B11F49D1
:10532000FFF785FA28461E49FFF781FA002084F826
:10533000A80084F8A900F8BD1A4E96F8C1389BB1B0
:1053400096F8C03883B11849052206F6EC0065F0DE
:105350004DFD1649152206F6F10065F047FD0123C3
:1053600086F806390DF066FF96F8C27897B194F882
:1053700035000028DFD10E4D0E4C0FCD0FC495E83F
:105380000F0084E80F00012386F807390DF052FF63
:105390003846D0E70120CEE780950020079A08081C
:1053A000619A080878A6002098950020A095002012
:1053B000B895002044AF002008B5FFF7A7FF38B12B
:1053C000FEF7E2F90348FEF7BDFB0020FEF784FB81
:1053D00008BD00BF7F9A080808B5034610462AB1E9
:1053E000DB0600D511B1FEF7ADFB002008BDF8B516
:1053F0000D4E96F8A030054693B9F8BD25B1238827
:10540000C3F30B039D4204D0D4E90201A28865F0E6
:1054100039FC1C34BC42F1D3002386F8A030ECE701
:10542000024C034FF6E700BF80950020B8E1080862
:10543000E4EB08082DE9F04F85B0164601911A46B5
:10544000824600213046FFF7C7FF324C06F01003BA
:1054500005464FF000090293FEF71AFB2379019AE3
:1054600003F01803934203D0002A48D1182B46D1E9
:10547000284B4FF00D0B0BFB0933B3F80900FCF779
:1054800077F880462046FBF7A6FED8E902210746BA
:10549000024401442046FBF757FE80F001012A46F2
:1054A0000390C9B23046FFF797FFDDE902230546B6
:1054B00002B123BB174A0BFB09FB52F80BB0B20633
:1054C0000FD573B9144803935946FEF77FFBD8F8FC
:1054D0000820039B3A4421465046FFF7A7F8FEF701
:1054E00013FB0E485946FEF771FBD8F80C20002339
:1054F0003A4421465046FFF799F8FEF705FB09F1BB
:10550000010940F28D23994504F10D04A4D105B0A1
:10551000BDE8F08F5CE50708869A0808879A0808B6
:105520000149FFF784B900BF919A080838B50C46C5
:10553000054615492046FCF73BFE30B9FEF78EFACA
:105540001248BDE83840FEF7F7BA11492046FCF78B
:105550002FFEA0B90F4A82F8020282F80A0282F8EE
:10556000A60282F8AE0282F84A0382F8520382F859
:10557000EE0382F8F60382F82D040748E1E7284697
:10558000BDE83840CCE700BFA09A0808A69A0808F2
:10559000C19A080880950020C99A08082DE9F043AF
:1055A000064687B008460C4662F082FF082843D1C1
:1055B000671E03AD073429463A46A84612F8010F84
:1055C000FCF7F0FDA24201F8010BF7D10023DFF850
:1055D0007C908DF8143017F8010FFCF7E3FDC1B291
:1055E00005F8010B4846019165F0C6FB20B1019911
:1055F000284665F0C1FB28B13046FFF791FF07B0A0
:10560000BDE8F083A742E6D10F49404632F07AFD6B
:105610000D480E49082310F8012B11F8014B1832E0
:105620006A44013B02F80C4CF5D109488DF814305E
:1056300003A9FEF781FBE2E70028E9D0304607B076
:10564000BDE8F043FFF70AB9D0990020205B0808B5
:10565000E59A08082DE9F74F064601AA08462F49A2
:10566000DFF8C880DFF8C890DFF8B0A065F040FB35
:105670004FF0000B04465D4601271CBBBBF1000F39
:1056800028D1274C002D44D026482946FEF754FB4C
:1056900094F8A0300BB905F091FAFBF7FBFF00235B
:1056A00084F8A930FEF7DAF915B12846FFF79FFE16
:1056B0009FB13046FFF72AFE78B1FEF711F80020BF
:1056C000FEF70AFABBF1000F0AD02046FCF786FE6F
:1056D00085B2C5B93046FFF723FF03B0BDE8F08FB0
:1056E00041462046FCF7ACFD80B949462046FCF710
:1056F000A7FD0028EED05F4601AA5146002065F0C4
:10570000F7FA0446B9E74FF0000BF5E74FF0010B4D
:10571000F2E70548FEF716FABFE700BFB19F080899
:1057200080950020F59A0808189B0808EC9A08084C
:1057300080A6080807B5009313460A460249FFF7FA
:1057400076F803B05DF804FB2E9B080820B10078C2
:10575000B0FA80F040097047012070472DE9F3410D
:1057600006460846FFF7F2FF0D46074670B10024D3
:1057700001A920465CF028F9013401463046FFF7C4
:10578000EDFF122CF4D102B0BDE8F0810846FCF721
:1057900025FEC4B2112C71D8681CFBF77FFE3B4D6F
:1057A0008046E8B93A4B03EB440393F808198A1E84
:1057B00051425141364B03EB440393F80829AA5C4C
:1057C000002954D093F80939192040F2EE2100FB4A
:1057D00003133048214602B0BDE8F041FEF7ACBAF1
:1057E0000178284665F0C8FA70B1032C94BF0022F6
:1057F0000122294902EB4202431B0A4452FA83F375
:1058000093F87079032F04D1304602B0BDE8F0411F
:1058100086E64046FBF742FE08B3022FF4D1FCF7C0
:10582000DDFD40F6CA0280B29042194BA8BF104677
:1058300040F2EE22904203EB4403B8BF1046A0F2C0
:10584000EE201922B0FBF2F083F80909BB1E594281
:1058500059410F4B03EB440383F80879AAE7022F61
:10586000F4D1304602B0BDE8F041FEF7F7BF0B4877
:10587000214602B0BDE8F041FEF75EBA08491123A7
:105880003A46304602B0BDE8F04153E7405D0808B3
:1058900078A60020479B080830CD0708579B0808CA
:1058A000649B08082DE9F04F024691B00846FFF7C7
:1058B0004DFF0B46044628B1104611B0BDE8F04F2D
:1058C000FEF7CCBF4FF0FF32CDE90820A74ADFF842
:1058D000E482D2F89C20DFF8E09292F83810DFF8EA
:1058E000DCA2CDE90C10CDE90E02CDE90A00A049F9
:1058F00007AA184665F0FCF9274605460494264693
:105900004DB9089A0C9FBA4262D19A48FEF714FA30
:1059100011B0BDE8F08F062F12D8DFE807F0041EA3
:105920002328454C510051462846FCF789FC78B1A4
:105930004FF4806012F0ECF890F9043008930124E1
:105940008B4907AA002065F0D3F901370546D7E750
:105950002846FCF743FD0890F2E72846FCF73EFD99
:105960000990EDE72846FCF782FC0A90E8E7284614
:1059700062F09EFD4146024605902846FCF73CFC3D
:1059800018B3059A49462846FCF736FC0646002817
:10599000D6D02846FCF722FD04280646D0D9014679
:1059A0007548FEF7C9F9B3E72846FCF717FD002351
:1059B0000C900F93C4E72846FCF710FD0D90BFE74D
:1059C0002846FCF754FC0E90BAE701230493B7E78E
:1059D000DFF8EC8151B2434613F9010B884208D03D
:1059E0000135092DF8D1002164480131FEF7A4F9F1
:1059F0008EE763480121FEF79FF97AB2002318F978
:105A0000011B8A4200F00D810133092BF7D13A4680
:105A10000121E9E7A7F1140253425341059308AD70
:105A2000002303F10108EB68A3BB95F900B05846C9
:105A300012F036F8D5F804A020B1D0F80090B9F1F2
:105A4000000F5ED1BAF1000F19D14FF461436B60C2
:105A50004FF0010AAB680BB90323AB600023D5F804
:105A6000049002932A7A1946CDE9009258461A46C4
:105A700012F0B3F8E86028B94248414691E74FF088
:105A8000000AE7E74A464146BAF1000F37D03E48E0
:105A9000FEF79CF8B8F1020F05F110054FF0010375
:105AA000BFD1059BDDF83C800B9D53B13748FEF715
:105AB00043F8D8F800301B6A1BB135492A464046E6
:105AC0009847049B002B4ED03249334B142F18BFFC
:105AD00019463248FEF730F9142F09D1049B03B957
:105AE00036B12B68DB691BB12D49324628469847F1
:105AF000002C67D10022414628465BF019FF294857
:105B0000C6E7C5F80C90BAF1000F25D026484146EB
:105B10005246FEF75BF85146484602F0AFFED5F814
:105B200008A0BAF1000F0FD099F8042092450BD0CD
:105B30001E4853464146FEF749F8D9F800305FFA4F
:105B40008AF19B6948469847D9F82C30002BA1D0A0
:105B50000023C9F82C309DE7D9F8082014484146A5
:105B6000FEF734F8DBE70C49B3E700BF809500206F
:105B7000B19F0808A29B08088A9B0808E69C0808B1
:105B8000BB9B0808C79B0808E39B08089A9C080869
:105B90007D8801086C9B0808229C0808C39C0808A3
:105BA000B7140108079C0808239C0808759C08087E
:105BB000509C0808849B080865980808799B080889
:105BC000ECD0070806F052FD05200CF0C5FE1A4F78
:105BD000DFF86C9000264FF0030A99F89035B34235
:105BE00088D917F801BBBBF1000F15D058460DF04E
:105BF000BBF9044680B1584606F070FC08B1A0F825
:105C000006A001210490F5F709FCA379049813F08C
:105C1000010F03D0F4F7ACFD0136DEE7F4F798FD91
:105C2000FAE706483A460221FEF786F8099B002B60
:105C30003FF4F0AE0023F1E69C2D0020BB9B08084A
:105C4000C00A001010B5044608460B46FFF77EFD5B
:105C500028B9094903221846FCF7CEFA28B90748A3
:105C6000FDF770FF0120FDF737FF20460449BDE82E
:105C70001040FEF7DCBD00BFF89C0808FC9C08083B
:105C8000529A08082DE9F74F05460846FFF75EFDD2
:105C90000B46044618B9334A92F82C7927B928469E
:105CA00003B0BDE8F04F3BE42F49DFF8C880DFF8D0
:105CB000C890DFF8C8A001AA184665F019F8264672
:105CC00010B906F0E1FC08E056B901220146284669
:105CD000FFF70CF9421C04461BD103B0BDE8F08F5E
:105CE000FCF77CFB2F28834636D80FB106F0BEFCAC
:105CF000BBF1060F14D01D49012391F890155FFAEE
:105D00008BF2E0B20CF09EFD59464846FEF714F8BF
:105D10000027154901AA0020013664F0E9FFCFE70A
:105D2000DAF8BC351B0113D5FF2C0FD0E1B22846A1
:105D3000FFF706F9E8E72846FFF702F901370B4BB2
:105D400093F89025F9B28A42F5D8DDE70027F6E707
:105D50000748FDF7F1FED7E72F2241462846FEF718
:105D600066FDD6E778A60020B19F0808C00A00109B
:105D70006A9808082F9D08081E9D08088095002035
:105D80002DE9F04F064685B00846FFF7DFFC0B46CD
:105D9000044628B1304605B0BDE8F04FFEF75EBDC1
:105DA0003149DFF8D490DFF8D4A0DFF8D4B003AAEB
:105DB000184664F09DFF27460546A04665B92B4B63
:105DC0003A46D3F89C00A1B261F04DF868BB28496F
:105DD0003046FEF72CFD28E0B8F1000F06D0B8F1F0
:105DE000010F25D03046FEF739FD1EE0284662F04F
:105DF0005FFB4946024601902846FCF7FDF950B387
:105E0000019A51462846FCF7F7F930B3019A5946F2
:105E10002846FCF7F1F910B3019A16492846FCF719
:105E2000EBF9F0B13046FFF77BFB05B0BDE8F08F32
:105E3000BB1E5A425A4129463046FFF757F8421CCA
:105E40000446F2D0084903AA002064F051FF08F18B
:105E500001080546B2E74746F4E70127F2E70227C3
:105E6000F0E70327EEE700BFB19F08088095002008
:105E70005B9D0808589D08084F9D0808529D08081A
:105E8000559D08082DE9F74380460846FFF75EFC5C
:105E90000B46054628B14046FEF7E0FC03B0BDE8DE
:105EA000F0832E49DFF8B49001AA184664F020FF71
:105EB0002F4604462E467CB9022DECD1A7F57A7305
:105EC000B3F57A7F21D926494FF4FA634FF47A72F9
:105ED0004046FFF72FFCE1E74DB1012D10D001AA9C
:105EE0004946002064F004FF01350446E3E701223F
:105EF00021464046FEF7FAFF431C0646EFD1CDE7A8
:105F00002046FCF76BFA0746E9E7164DD5F84C3A00
:105F1000B8B25B689847FF2EBCEEC00A124B0BD19B
:105F200095F89025F8EE407AA24212DC10EE101A95
:105F30000E48FDF701FFB1E7F8EE407A03EB860368
:105F400010EE102A0A48C3ED007A3146FDF7F4FE40
:105F5000A4E7E3EC017A0134E6E700BFB19F08084B
:105F6000699E0808C00A0010A8AF0020869D080896
:105F7000799D0808F8B507460846FFF7E7FBC8B162
:105F80001F4B1E6B0136304611F09CFB3446054614
:105F9000F0B90134192CA8BF0024204611F092FB5F
:105FA0000546A8B9B442F4D138461649BDE8F840D0
:105FB000FEF73DBC0846FCF711FA044611F082FBDF
:105FC000054628B921461048BDE8F840FDF7B4BEA3
:105FD0000B4B1C6311F0C6FE0C482A462146FDF708
:105FE000ABFE182C09D80A480C2101FB040090F8DC
:105FF0007809BDE8F84011F0EBBE0020F9E700BFDA
:10600000B0060020959D0808A99D0808BF9D0808B6
:1060100030CD070838B5124D04460846FFF796FB09
:1060200060B1104B104893F900104B1C0ABF0F4B86
:10603000C9B21979BDE83840FDF77EBE0846FCF7C5
:10604000CDF9032804D8C0B2FDF79CF92946E4E74E
:1060500020460749BDE838400322FEF7E8BB00BFF1
:10606000229C0808B0060020D89D080880950020D2
:10607000E89D080838B5124D04460846FFF766FB50
:1060800060B1104B104893F901104B1C0ABF0F4B25
:10609000C9B25979BDE83840FDF74EBE0846FCF755
:1060A0009DF9032804D8C0B219F022FB2946E4E781
:1060B00020460749BDE838400322FEF7B8BB00BFC1
:1060C000229C0808B0060020D49D08088095002076
:1060D000E39D08082DE9F74F444BDFF828A11A7912
:1060E0008AF800205A7993F8A0308AF801200546F2
:1060F00088460BB904F062FDFBF7CCFA00263C4C55
:10610000B1460D233A4A7343414652F803B058460C
:10611000FCF796F8002841D0B9F1000F01D0FDF747
:10612000F3FC34485946FDF751FD0022214628462C
:10613000FEF76EFBFDF7E8FC237903F01803082B4C
:1061400046D0102B49D02046FDF705FE284A0D23E6
:1061500003FB0623B3F80900FBF70AFA0746D8B198
:106160002046FBF738F8D7E90221009002440144A9
:106170002046FAF7E9FF78B9019059461E48FDF725
:1061800025FD019AB9681346009A28460A4421461B
:10619000FEF74CFAFDF7B8FC09F10109013640F2AF
:1061A0008D239E4204F10D04ABD10020FFF71FF9AF
:1061B000FF238AF800308AF80130B9F1000F11D1BD
:1061C0000E494246284603B0BDE8F04FFEF72FBB0C
:1061D0000B492846FFF71EFFB5E709492846FFF798
:1061E00049FFB0E703B0BDE8F08F00BF8095002005
:1061F0005CE507088B9A0808039E0808379808088A
:10620000229C0808B00600202DE9F74F07460846F3
:106210000E4662F04DF9044620B1012826D13278AD
:106220002A2A23D1B348B44EDFF8E892FDF784FC64
:106230000025B2464FF00D0B40F28D280BFB05F305
:1062400048465AF80310FDF7C1FC221E18BF012270
:10625000314638460135FEF7DBFAFDF755FC45457A
:1062600006F10D06EAD103B0BDE8F08F3D213046BE
:1062700064F082FD002800F0378101460A4611F8DB
:10628000014D202CFAD0921B0130814610F8011BE1
:106290002029FAD0DFF860B25FFA82FA4FF00008E6
:1062A0000D2303FB08F10BEB010452465BF80110D0
:1062B00000913046FBF7A0FF0546002857D1009912
:1062C000084662F0F5F8824551D1267906F0E001E2
:1062D000402900F0CC800ED8002956D0202900F0AB
:1062E0009E8038468549FEF7A2FA204603B0BDE8F5
:1062F000F04FFDF730BD602900F092808029F0D189
:10630000484662F0D5F8E379A679DB0705460CD557
:106310002046FBF743F90378014633B12A46484645
:1063200064F050FD002840F0D980002D00F0D680A8
:10633000AE42C0F0D3800D2303FB08B3204693F890
:1063400005A0FBF72BF93246002164F0FEFCAA45BC
:106350002CD86B492A46484664F034FD30B32046B9
:10636000FBF71CF92A46494664F08CFC1EE008F154
:10637000010840F28D23984592D162493246384651
:1063800003B0BDE8F04FFEF752BA06F00703042B46
:106390001CD10B460A224846FBF77EFFD4F8053095
:1063A000834201469DD32046FBF70EF90D2303FBE4
:1063B00008F855485BF80810FDF708FC0022214654
:1063C000384603B0BDE8F04FFEF722BA052B0FD1D7
:1063D00001230A224846FBF75FFFD4F805308342C9
:1063E0000146FFF67EAF5B4283423FF77AAFDAE7C2
:1063F0004846FBF7F3FFB4F80550B4F8071016F061
:10640000050FAAB218BF2AB28BB218BF0BB29042C6
:10641000FFF667AF98423FF764AF0146C3E765797F
:106420003A4A02EBC505002695F838250092B24697
:106430003346009AB24202D9BAF1000F03D0002BC2
:106440003FF44FAFB2E7D5F8341551F8260060B1EC
:1064500049460193FBF7ACFE019B30B9314620461B
:106460004FF0010AFBF7B0F853460136E1E76379D4
:10647000009306F00706013E009BAB4296DD4846BE
:10648000814610F8013B202BFAD02046FBF786F816
:106490008246042E04D8DFE806F0031010161F0011
:1064A0004846FBF79BFF0AF8050048462C2164F09C
:1064B00063FC013500F10109DEE74846FBF78EFF7A
:1064C0002AF81500F1E700230A2200214846FBF7CD
:1064D000E3FE4AF82500E8E70123F5E70C493246D8
:1064E0003846FEF7A4F9FCE63146384603B0BDE86D
:1064F000F04FEFE5139E08085CE50708619E080869
:106500003EC3080837980808569E080830CD07088B
:10651000269E08088B9A08082DE9F04F914689B00D
:106520000C461A4600218046FEF756FFDFF8ECB015
:1065300006464D460027B9F1000F6CD029460622C9
:10654000204664F0D8FB0028324614BF0121002108
:1065500040460CBF4FF0010A4FF0000AFEF73CFF27
:106560000646287817F002FC079010B3687917F0F8
:10657000FDFB079BEA785B790793AB7895F801E020
:106580004FF461714FF0190C1CFB03131CFB02123A
:10659000297900B14079CDF804E0CDE90232079BBA
:1065A0000093CDE904103B465A4651464046FDF75C
:1065B000F5FA207817F0DAFB079010B3607917F03E
:1065C000D5FB079BE2785B790793A37894F801E009
:1065D0004FF461714FF0190C1CFB03131CFB0212EA
:1065E000217900B14079CDF804E0CDE90232079B72
:1065F0000093CDE904103B465A4651464046FDF70C
:1066000087FA0137142F04F1060405F1060592D12B
:1066100009B0BDE8F08FCA46CBE700BF6F9E0808FF
:106620002DE9F041064686B00846FFF78FF80F4681
:10663000054638B100235D491A46012006B0BDE881
:10664000F04169E70846FBF7C9FE1328044600F34A
:10665000A38006264643781C8DF81750FAF71EFFD4
:10666000534D074670B1FBF7B9FEC0B217F094FB6B
:1066700040B1AB19027983F82C269DF8173001330D
:106680008DF817303846FAF709FF074668B1FBF76F
:10669000A5FE0D2809D8062303FB045383F82D0615
:1066A0009DF8173001338DF81730DFF80081B11CE9
:1066B0000DF1170241443846FBF794FEFAF7EEFE5F
:1066C000074668B1FBF78AFE012809D8062303FBB9
:1066D000045383F830069DF8173001338DF81730D6
:1066E0003846FAF7DBFE80B1FBF778FEC0B217F050
:1066F00053FB50B1062303FB0453027983F8312680
:106700009DF8173001338DF817309DF81720042AB3
:106710004FF006032FD103FB04530022A3F83026C9
:1067200022F0D6FA062303FB04554FF4617695F860
:106730002C0617F01BFB95F82F2695F82E761923BB
:10674000804695F8310613FB076713FB026617F0C6
:106750000DFB437998F80520039395F830360097A0
:10676000CDE90163134895F82D362146FDF7E4FA8B
:1067700006B0BDE8F081052A05D103FB04530022D1
:1067800083F83126CCE7062ACAD008EB060200239C
:1067900048F806309380C3E7074913232A4630465A
:1067A00006B0BDE8F041FEF7C5BF00BFAC9B0020BE
:1067B000809500206F9E0808889E08082DE9F04FFC
:1067C000174689B01A460C4600218146FEF704FEA2
:1067D0003B4EDFF8F4B007F16C0380463D4607936B
:1067E00094F90410374A002392F90800884263D0D4
:1067F0000133092B02F10C02F6D1079B0C359D42A7
:1068000004F10C04ECD109B0BDE8F08F29460C224C
:10681000204664F070FA0028424614BF012100218E
:1068200048460CBF4FF0010A4FF0000AFEF7D4FDB6
:10683000EA7995F9043006EB82028046D2F8A8275F
:1068400004922A7A06EB82025146D2F8A8270392D4
:10685000AA7906EB82024846D2F8A82702926A7902
:1068600006EB8202D2F8A82701922A6800925A46C3
:10687000FDF794F9E27994F9043006EB820251466F
:10688000D2F8A8270492227A06EB82024846D2F870
:10689000A8270392A27906EB8202D2F8A8270292D7
:1068A000627906EB8202D2F8A82701922268009250
:1068B0005A46FDF72DF9A0E7002FA7D1BA46D9E730
:1068C00030CD0708CC9A00208E9E08082DE9F047AD
:1068D00007468AB00846FEF739FF044638B1002360
:1068E00054491A4601200AB0BDE8F04766E70DF1A9
:1068F0001C080790C8E9010008464E1CFBF76EFD16
:106900004C4B40B21A4693F90410814200F08B8040
:106910000134092C03F10C03F5D10024254630463F
:10692000FAF7BCFD064638B100230A221946FBF7E8
:10693000B3FC01350790EDB2DFF800A14FF000097C
:106940003046FAF7ABFD064640B3FBF747FD3A4940
:10695000002251F804CB6045D3B203D00132102A93
:10696000F7D100230AEB8302D2F8A827904215D171
:10697000B9F1020F1FD0B9F1030F21D05A1EB9F19E
:10698000010FD2B212D00B2A03D88DF82130013575
:10699000EDB209F10109B9F1040FD1D1052D15D8D6
:1069A00038460AB0BDE8F047FDF758BF042AF0D8D2
:1069B0008DF82230EBE7052BEBD88DF82430E6E795
:1069C0009A1E0D2AE5D88DF82330E0E798E80700F5
:1069D0001A4B84E807009DF8232003EB8202002174
:1069E000D2F8A82704929DF8242003EB82020846DF
:1069F000D2F8A82703929DF8222003EB8202D2F856
:106A0000A82702929DF8212003EB82030C4AD3F8B9
:106A1000A8370193079B00939DF92030FDF778F884
:106A20000AB0BDE8F0870C2303FB04248DF8200096
:106A3000012574E7089A0020D8D4070830CD07084C
:106A40008E9E08082DE9F04F8BB00C46089200216D
:106A50001A460746FEF7C0FCDFF8B4B0089D09905F
:106A600000264FF019094FF46178089B002B4BD09A
:106A700029460A22204664F03EF90028099A14BFEC
:106A80000121002138460CBF4FF0010A4FF0000AE7
:106A9000FEF7A2FC2A890692EA8805922A790492D6
:106AA000EA780392AA78099019FB028202926A7826
:106AB00019FB028201922A78009233465A465146C7
:106AC0003846FDF76BF822890692E2880592227912
:106AD0000492E2780392A27819FB02820292627811
:106AE00019FB0282019214F80A2B009233465A468F
:106AF000514638460136FDF70BF81E2E05F10A0502
:106B0000B3D10BB0BDE8F08FDDF820A0DBE700BF0C
:106B1000AB9E08082DE9F04380468BB00846FEF78F
:106B200015FE0F46044638B1002365491A46012078
:106B30000BB0BDE8F04385E70846FBF74FFC1D2886
:106B4000054600F3B3800A264643781C8DF827409B
:106B5000FAF7A4FC044630B1FBF740FC9DF827305F
:106B600001338DF827302046FAF798FC554C07463C
:106B700068B1FBF733FC0D2809D80A2303FB054352
:106B800083F850099DF8273001338DF82730DFF85E
:106B90003091711C0DF1270249443846FBF722FC65
:106BA000FAF77CFC074668B1FBF718FC222809D8E5
:106BB0000A2303FB054383F853099DF8273001336B
:106BC0008DF827303846FAF769FC074668B1FBF7BD
:106BD00005FC0D2809D80A2303FB054383F8540953
:106BE0009DF8273001338DF827309DF82730062B8C
:106BF0000CD009EB0602002349F8063040465360EA
:106C00001381FDF72BFE0BB0BDE8F0830A2606FBCF
:106C1000054600233846A6F85639A6F85839FAF73B
:106C20003DFC074640B1FBF7D9FB9DF82730A6F89D
:106C3000560901338DF827303846FAF72FFC58B142
:106C4000FBF7CCFB0A2303FB0543A3F858099DF887
:106C5000273001338DF827301B4B4FF0FF325A603D
:106C60000A2202FB05424FF46170B2F858390693CC
:106C7000B2F85639059392F85439049392F853397F
:106C8000039392F85219192313FB0101029192F810
:106C9000511913FB0103019392F85039009300211D
:106CA0000A4A2B460846FCF733FFACE708491D2388
:106CB000224640460BB0BDE8F043FEF73BBD00BFA7
:106CC000C8AF002078A60020B0060020AB9E0808C0
:106CD000889E08082DE9F04F2DED088BDFF82CA1D8
:106CE00095B0804691461F460C4616464FF0000B65
:106CF00094ED008AB5EE408AF1EE10FA7FD0D4ED23
:106D0000019A94ED029AD4ED038AB9F1000F49D0AB
:106D1000D6ED00BA96ED01BAD6ED02AA96ED03AA19
:106D2000B4EE6B8AF1EE10FA6ED1F4EE4B9AF1EEFE
:106D300010FA69D1B4EE6A9AF1EE10FA64D1F4EE69
:106D40004A8AF1EE10FA0CBF012100213A460D46A5
:106D5000404681F00101FEF73FFBB0EE6B0A0746AB
:106D600011A8FAF717FBB0EE4B0A07900EA8FAF736
:106D700011FBB0EE6A0A06900BA8FAF70BFBB0EE17
:106D80004A0A059008A8FAF705FB0599069A079B99
:106D9000039002910192009352465B462946404679
:106DA000FCF7FCFEB0EE480A11A8FAF7F3FAB0EED1
:106DB000690A05460EA8FAF7EDFAB0EE490A069000
:106DC0000BA8FAF7E7FAB0EE680A059008A8FAF7F8
:106DD000E1FA069B059A0390CDE9005302925B46C7
:106DE0005246002140460BF1010BFCF791FEBBF12E
:106DF000080F04F1100406F110067FF479AF15B006
:106E0000BDEC088BBDE8F08F00219FE7CE9E0808FF
:106E10002DE9F74FDFF898A1DFF898B107460D4646
:106E20002846FEF793FC064638B1002359491A4616
:106E3000012003B0BDE8F04F4CE70522514628463B
:106E4000FBF7DAF960B9534B00221A601A611A6233
:106E50001A631A641A651A661A6703B0BDE8F08FE0
:106E60004D4904222846FBF7C7F904462846002C62
:106E700044D1FAF713FB80460028EED061F018FBEE
:106E8000464BC2B253F8049BB9F1000F07D14449F5
:106E90002A46384603B0BDE8F04FFDF7C8BC494666
:106EA0004046CDE90023FBF7A7F90134DDE90023D3
:106EB00006460028E6D1374A03461546002101332D
:106EC000082B42F8101BFAD10BEBC404D4F8BCC059
:106ED000BCF1000F03D094F8B8E0764505DB3148EB
:106EE000314D4946FCF728FF9AE70CEB06130FCB10
:106EF00005EB061484E80F000136EEE7FBF76EFAA7
:106F0000072804463DD82846FAF7C8FA064658B37B
:106F1000FAF752F81F4B03EB041383ED000A012527
:106F20003046FAF7BBFA064638B1FAF745F8194B7E
:106F300003EB041383ED010A01353046FAF7AEFA8C
:106F4000064638B1FAF738F8124B03EB041383ED19
:106F5000020A01353046FAF7A1FA38B9384603B0CB
:106F6000BDE8F04FFDF77ABC0546D9E7FAF724F8FB
:106F70000848032D00EB041484ED030A3FF455AFD9
:106F8000ECE70A4907233246384603B0BDE8F04F24
:106F9000FEF7D0BBEC9E0020E29E080834D607081E
:106FA00037980808E79E0808229C0808889E080869
:106FB000849B080830CD07082DE9F74F92460C4610
:106FC0001A4600218146FEF707FADFF870B08046C6
:106FD00056460025BAF1000F2ED031460422204635
:106FE00063F089FE0028424614BF01210021484673
:106FF0000CBF01270027FEF7EFF9738801933AF8D9
:107000002530009380462B465A4639464846FCF7C1
:10701000C5FD6388019334F8043B00935A462B4620
:10702000394648460135FCF773FD042D06F1040688
:10703000D0D103B0BDE8F08F5746EAE7F19E0808CB
:107040002DE9F34105460846FEF780FB0C4607464E
:1070500038B1002333491A46012002B0BDE8F0419F
:10706000AAE731492046FBF7A3F8034670B92D4A39
:107070004FF47A704FF4FA610133042B1080518081
:1070800002F10402F8D102B0BDE8F0812046FBF71E
:10709000A5F90328064641D82046FAF7FFF9074626
:1070A00070B1FBF79BF94FF0010804463846FAF738
:1070B000F5F948B9284602B0BDE8F041FDF7CEBB6E
:1070C00040F2EE248046F1E7FBF788F9B8F1000FB3
:1070D000F0D0A4F2EE2240F2DC539A4203D8A0F2A0
:1070E000EE229A420AD9114940F6CA0340F2EE2232
:1070F000284602B0BDE8F041FEF71CBB0C4B0D4A20
:1071000003EB86030021A3F87C4AA3F87E0ACDE9AD
:10711000004033460846FCF7FBFCB4E7064903236E
:107120003A46E5E7F4B00020849B0808029F08086F
:1071300078A60020F19E0808649B08082DE9F04F0E
:1071400089468FB0174600211A460646FEF744F9D5
:10715000DFF878A0054600240DF1240B59F82430FF
:107160000293594602A85AF091FB67B357F82430AE
:10717000029A0393934218BF01212A4608BF0021B7
:1071800030460CBF4FF001084FF00008FEF724F91D
:1071900004A9054603A85AF079FB04A900912346E7
:1071A000524641463046FCF7F9FC2346CDF800B084
:1071B0005246414630460134FCF7AAFC202CCDD182
:1071C0000FB0BDE8F08FB846EFE700BF109F08088A
:1071D000F0B5074689B00846FEF7B8FA0E460546F0
:1071E00038B1002319491A46012009B0BDE8F04022
:1071F000A4E70846FBF7F2F81F2804461DD83046DE
:10720000FAF74CF9014620463EF0F4FC78B10F48FD
:1072100003AE314600EB84005AF038FB0C4A00966E
:10722000234629462846FCF773FC09B0F0BD3846D2
:1072300009B0BDE8F040FEF773B906491F232A469E
:10724000384609B0BDE8F040FEF774BA04B100203A
:10725000109F0808889E08082DE9F04F924685B0D7
:107260000C461A4600218146FEF7B6F8DFF874B0E6
:10727000804655460026BAF1000F31D02946042237
:10728000204663F038FD0028424614BF012100214A
:1072900048460CBF01270027FEF79EF8EB780293C3
:1072A000AB7801932B880093804633465A46394683
:1072B0004846FCF773FCE3780293A378019334F813
:1072C000043B00935A463346394648460136FCF79C
:1072D0001FFC102E05F10405CDD105B0BDE8F08FDF
:1072E0005746E8E71A9F0808F0B5074685B00846F4
:1072F000FEF72CFA0E46054638B100231C491A4603
:10730000012005B0BDE8F040A6E70846FBF766F8A7
:107310000F28044623DC3046FAF7C0F80146204621
:107320003EF0E8FBA8B1134B04F1200203EB82030B
:10733000294693F88F2A029293F88E2A0192B3F885
:107340008C3A00930C4A23462846FCF7E1FB05B033
:10735000F0BD384605B0BDE8F040FEF7E1B807499A
:107360000F232A46384605B0BDE8F040FEF7E2B9E3
:1073700084B1002078A600201A9F0808889E08087B
:107380002DE9F04F87B0144603911A4600210546B7
:10739000FEF722F8DFF830B106464FF0000806236A
:1073A00003FB08F7C0374FF00009039BDB5D049334
:1073B000002C00F08580E35D049A05939A4218BF83
:1073C0000121324608BF002128460CBF4FF0010AB8
:1073D0004FF0000AFEF700F8059B0646CDE9009342
:1073E0005A46434651462846FCF7D8FB049B5A466A
:1073F000CDE9009351464346284609F10109FCF7BF
:1074000087FBB9F1060F07F10107CED108F101089A
:10741000B8F1060FC3D1DFF8B0B0E427039BA7F1A2
:10742000E40913F807A0002C4CD0E35D04939A45BF
:10743000324614BF0121002128460CBF4FF001083D
:107440004FF00008FDF7C8FF049B0646CDE9009306
:107450005A46062341462846FCF7A0FBCDE9009A90
:10746000194A0623414628460137FCF751FBEF2F06
:10747000D4D1039B93F8EF70B4B194F8EF804745F3
:10748000324614BF0121002128460CBF01240024EC
:10749000FDF7A2FF002300930B4ACDF804800723D9
:1074A00021462846FCF77AFB00230093064A019701
:1074B000072321462846FCF72BFB07B0BDE8F08FD9
:1074C000A24693E7A046C9E72C9F0808F0B50546F9
:1074D00087B00846FEF73AF90B46044638B1002358
:1074E0001C491A46012007B0BDE8F04048E71A4998
:1074F000194F02AA184663F0FBFB03AEB8B1032C88
:1075000004D12846FDF7AAF907B0F0BDFAF766FFE7
:1075100002AA46F8040B39460020013463F0E8FB68
:10752000ECE70E4832462146FCF706FCECE7032C5C
:10753000E7D1DDE90346059B01931A463146E0B2E7
:107540003EF01CFB019B0028EBD12846FDF7E8FF2D
:10755000DAE700BF04B10020B19F08082C9F08089B
:107560002DE9F04F0F4689B0164600211A46054610
:10757000FDF732FFDFF83CB10790B84634464FF0D4
:107580000009002E7ED021460C22404663F0B3FB5A
:107590000028079A14BF0121002128460CBF4FF094
:1075A000010A4FF0000AFDF717FF94F90B2004922F
:1075B00094F90A200392B4F908200292B4F9062043
:1075C0000192B4F90420079000924B465A46514666
:1075D0002846FCF7E3FA98F90B20049298F90A2060
:1075E0000392B8F908200292B8F906200192B8F97E
:1075F000042000924B465A465146284609F101099B
:10760000FCF786FAB9F1080F08F10C0804F10C0434
:10761000B7D1DFF8A49000240C2303FB04FA9EB337
:107620004FF00008012303FA08FB56F80A2057F828
:107630000A3053403BEA030314BF0121002112EA40
:107640000B0F08D0CDF8008023464A462846079104
:10765000FCF7A4FA079957F80A301BEA030F06D083
:10766000CDF8008023464A462846FCF751FA08F137
:107670000108B8F10E0FD5D10134082CCCD109B0D6
:10768000BDE8F08FB246A6E7B04657F80A200123BE
:1076900003FA08F3134207D0CDF8008023464A4688
:1076A00001212846FCF734FA08F10108B8F10E0F61
:1076B000EBD1E1E7409F0808589F0808F0B506465F
:1076C0008BB00846FEF742F80D46044620B300236F
:1076D0003F491A4601200BB0BDE8F04040E72D2B92
:1076E00003D0A3F13002092A4BD8052C05DD304622
:1076F0000BB0BDE8F040FDF7B1B82846FAF76EFED2
:107700000AAB621C03EB440424F80C0C15F8013F8F
:10771000303B092BFAD914462B78002BDFD1062CED
:10772000E5D1BDF81C20BDF91C30072ADFD8BDF912
:107730001E10A1F5FA7292B2B2F5FA6F1AD8BDF91D
:107740002040A4F5FA7292B2B2F5FA6F12D8BDF9E0
:107750002270B9420EDCBC420CDBA1420ADCBDF94E
:1077600024C00CF1640292B2C82A03D8BDF9265095
:10777000112D11DD174930460BB0BDE8F040FDF783
:1077800056B8202B02D101352246C4E730460BB053
:10779000BDE8F040FDF7C4BE0F4A0C2000FB0322F9
:1077A0006DB2A2F8801BA2F8824BA2F8847B82F80B
:1077B00086CB82F8875B00910021CDE903C5CDE936
:1077C0000147064A0846FCF7A3F90BB0F0BD00BF1D
:1077D000F4B100206D9F080878A60020409F08089B
:1077E0002DE9F04F89468DB0164600211A4607460E
:1077F000FDF7F2FDDFF8DCA005460024C4EBC4036E
:1078000009EB030259F8030091889279089040F33C
:107810000748ADF824108DF82620B8F1000F54D099
:10782000002E55D0F218F058918893790A90ADF84F
:107830002C1007220AA908A88DF82E3063F05BFAF5
:1078400000282A4614BF0121002138460CBF4FF002
:10785000010B4FF0000BFDF7BFFD9DF82E30069396
:107860009DF92D3005939DF92C3004939DF82B3014
:1078700003939DF92A3002939DF8293001939DF8D6
:107880002830009305462346524659463846FCF7B1
:1078900085F99DF8263006939DF9253005939DF9CD
:1078A000243004939DF82330CDE902839DF82130E4
:1078B00001939DF82030009352462346594638469E
:1078C0000134FCF725F9102C98D10DB0BDE8F08FEC
:1078D000B346DEE7839F08082DE9F04F9D4FDFF8A0
:1078E000A882DFF8A8928DB006460D46284660F0C3
:1078F000DFFD034630B99849024601200DB0BDE8CE
:10790000F04F6DE7052239462846FAF775FC044624
:10791000C8B9924D0146702205F6DC3063F015FAC5
:10792000C5F87C4BC5F8884BC5F8944BC5F8A04BFF
:10793000C5F8AC4BC5F8B84BC5F8C44BC5F8D04B2F
:107940000DB0BDE8F08F042241462846FAF754FCFA
:10795000044638BB2846F9F7A1FD82460028EFD03F
:1079600060F0A6FDDFF828B202465BF8041B39B9C7
:107970007B492A4630460DB0BDE8F04FFCF757BFB3
:107980005046CDE90012FAF737FC019A40B920467B
:107990002EF062FC0099734D4846FCF7CDF9A5E73F
:1079A0000134E2E7704907222846FAF725FC07462A
:1079B00000287AD12021284663F0DEF9044670BB06
:1079C0006A486B4DFCF702F9214628460134FCF762
:1079D000FDF80E2CF8D1FCF797F8DFF8B891654F59
:1079E000DFF8B481002421464846FCF7EFF80C2666
:1079F000DFF8A8A166430025F2595F480123AB4098
:107A0000134214BF414651460135FCF7DFF80E2DF5
:107A1000F2D10134FCF778F8082CE4D190E757490B
:107A2000564D03AA63F064F904AC002848D0022F35
:107A300011D1049A072A07D805990D2904D803788B
:107A4000722B13D06E2B22D04D49082300223046D2
:107A5000FDF770FE74E7FAF7C1FC03AA44F8040BC3
:107A600029460020013763F043F9DEE73B4B0C2049
:107A700000FB0233012000FA01F1D3F87C0B08432C
:107A8000C3F87C0B38493046FFF726FF58E7334BE5
:107A90000C2000FB0233012202FA01F1D3F87C2B07
:107AA00022EA0102C3F87C2BECE728463349334F26
:107AB00003AA63F01DF904AD0024A8B1082C03D17A
:107AC0003046FCF7CBFE3BE7FAF788FC03AA45F803
:107AD000040B39460020013463F00AF9EDE7294927
:107AE0003046FCF7A4FE2BE7082CE9D1049B0F2BB2
:107AF000F5D8DDF814E0BEF1070FF0D8DDF818C0B6
:107B0000BCF10D0FEBD8079F07F16402C82AE6D835
:107B1000089DFF2DE3D809986428E0D80A996429C4
:107B2000DDD88842DBDA0B9C032CD8D8C3EBC30228
:107B30000A4B134483F8E11B83F8DCEB094983F813
:107B4000DDCB83F8DE7B83F8DF5B83F8E00B83F823
:107B5000E24B98E7849B080854B2002078A60020E6
:107B600037980808229C0808A09F0808C7A508089D
:107B7000A89F0808F4B10020AD9F0808B19F08082D
:107B8000B39F08086D9F0808E29E0808E79E080852
:107B900034D6070879DC08086B9F080846A808084F
:107BA0002DE9F04F89B00C46079200211A4607468E
:107BB000FDF712FC0026079DDFF8A0B00690B24644
:107BC0004FF019094FF46178079B43B32946062209
:107BD000204663F090F80028069A14BF0121002186
:107BE00038460CBF4FF0010A4FF0000AFDF7F4FBD6
:107BF0006A79069019FB028205922A7919FB0282A2
:107C00000492EA780392AA7802926A7801922A781A
:107C1000009233465A4651463846FBF7BFFF627919
:107C200019FB02820592227919FB02820492E27802
:107C30000392A27802926278019214F8062B0092C5
:107C400033465A46514638460136FBF761FF0A2E45
:107C500005F10605B8D109B0BDE8F08FB99F080855
:107C60002DE9F04F80468BB00846FDF76FFD894641
:107C7000074638B1002355491A4601200BB0BDE82C
:107C8000F04F8DE7524C084694F84A3894F860B7A4
:107C900094F861A70793FAF7A1FB0928054600F3BA
:107CA0008B800626464309F101008DF82770F9F70D
:107CB000F5FB074658B1FAF791FB0D2807D8A31931
:107CC00083F8740B9DF8273001338DF82730384640
:107CD000F9F7E4FB074668B1FAF780FB834509D35F
:107CE000062303FB054383F8750B9DF8273001330A
:107CF0008DF827303846F9F7D1FB074668B1FAF717
:107D00006DFB504509D8062303FB054383F8760B2A
:107D10009DF8273001338DF827303846F9F7BEFB40
:107D2000074670B1FAF75AFB079B834209D3062333
:107D300003FB054383F8770B9DF8273001338DF85B
:107D40002730DFF88890311D0DF12702494438466D
:107D5000FAF748FB9DF82730062B0BD009EB0602FB
:107D6000002349F8063040469380FCF777FD0BB0BE
:107D7000BDE8F08F03FB05444FF4617194F8792B53
:107D8000192313FB0212059294F8782B13FB0213AC
:107D9000049394F8773B039394F8763B029394F81A
:107DA000753B019394F8743B00930021094A2B46DC
:107DB0000846FBF7ADFEDAE7074909233A46404695
:107DC0000BB0BDE8F04FFDF7B5BC00BFF4A000203C
:107DD00080950020B99F0808889E08082DE9F04F7B
:107DE0000F4689B0144600211A460646FDF7F4FAFC
:107DF0000546002C00F0DB8022783B789A4218BFC1
:107E00000121024608BF002130460CBF4FF0010897
:107E10004FF00008FDF7E0FA23789B4A05464146FB
:107E20003046FBF7BBFE3B78974A41463046FBF7AE
:107E30006FFE002C00F0BD8062787B789A4218BFFC
:107E400001212A4608BF002130460CBF4FF001082F
:107E50004FF00008FDF7C0FA63788C4A05464146AA
:107E60003046FBF79BFE7B78884A41463046FBF75D
:107E70004FFE07F1CA030493822304F1CA0B059352
:107E80004FF002094FF0000A3B78534500F393800E
:107E9000002C00F0F38097F8EA3094F8EA209A4238
:107EA00018BF01212A4608BF002130460CBF4FF001
:107EB00001084FF00008FDF78FFA94F8EA30744A91
:107EC000054641463046FBF769FE97F8EA30704AAE
:107ED00041463046FBF71CFE07F1EC09002C00F090
:107EE000CF8004F1EC034A4604F1FC014FF0010895
:107EF0009A4633F802CB32F8020B844518BF4FF094
:107F000000088B42F5D188F001012A46C9B23046FB
:107F1000FDF762FA082105465046FAF7BFF85D4AB8
:107F2000034641463046FBF739FE97F8EA104846CB
:107F3000FAF7B4F8574A034641463046FBF7E8FDE6
:107F4000002C00F09F804FF0FC094FF0010807EB78
:107F5000090104EB0900FAF72BF909F104090028DB
:107F600018BF4FF00008B9F58E7FF0D188F00101FD
:107F70002A46C9B23046FDF72FFA082104F1FC0069
:107F8000F9F7BEFA444A034641463046FBF706FE7F
:107F900097F8EA1007F1FC00F9F7B2FA3E4A0346F7
:107FA0004146304609B0BDE8F04FFBF7B1BDA046F1
:107FB00039E7A04657E7059B3B440693002C5BD06E
:107FC000059B0698234419460793FAF7F1F8049B9A
:107FD0001A789BF800309A4206BFB0FA80F84FEA50
:107FE00058184FF000084B4609F11002F85AE15AB0
:107FF0000233884218BF4FF000089342F6D188F050
:1080000001012A46C9B23046FDF7E6F9627804EB71
:10801000090105469BF81800FAF712F802909BF840
:1080200000300193079B00931C4A0AF1010341466B
:108030003046FBF7B3FD049B7A78187E079307EB75
:108040000901F9F7FDFF079B049A02901B78019341
:108050000132069B04920AF1010A00930F4A53462B
:1080600041463046FBF754FD059B09330BF1010BEC
:1080700009F11009059307E7A046DCE7A04624E7CD
:10808000A04652E7A04683E7D29F0808E49F08086D
:1080900012A008082AA0080841A00808F99F0808AB
:1080A0002DE9F04F8FB0044602AA0846AF4962F0AE
:1080B0001FFE064640B903460246AD494120FFF780
:1080C0008DFE0FB0BDE8F08FAA49FAF771F80746A8
:1080D00020BBA64902AA62F00BFEFAF77FF9082836
:1080E000054606D9A44908233A462046FDF722FB57
:1080F000E7E7A24C94F86037834202DC84F86057CB
:10810000DFE7064604F5EC67314638463AF072FA86
:1081100094F860370136B342F6DCEFE79849304611
:10812000FAF746F80546E0B9904902AA62F0E0FD88
:10813000FAF754F90828064603D9924908232A4633
:10814000D3E78E4C94F86137834202DC84F8616790
:10815000B7E728463146013559F070FB082DF8D1B4
:10816000F4E789493046FAF723F8074600BB7F4910
:1081700002AA62F0BDFD0028A3D0FAF72FF9082863
:10818000054603D9814908233A46AEE77B4C94F86B
:108190004A38834209DD014604F5EC603AF074FA8E
:1081A000294604F5EC603AF07DFA84F84A5888E7ED
:1081B00077493046F9F7FCFF054618BB6F4BDFF8EF
:1081C000AC9193F84A7806AE01461022304662F030
:1081D000BCFDB046BD4202AA80F20E814946002095
:1081E00062F086FD10B96B493A460EE1FAF7F6F8EF
:1081F000013528F8020BEDE796E80F00664C84E89D
:108200000F005EE765493046F9F7D2FF05460028C2
:108210003BD15A4B0DF1180893F84A984646074649
:108220004F45524902AA4FF0000080F2F28062F0FE
:108230005FFD014610B95A494A46E6E0032230463E
:1082400062F0D4FDB2464FF0000B304660F030F9DA
:10825000584502D801370436E2E79AF80000F9F7EA
:10826000A1FF0BF1010B0AF8010BEEE74D494A465D
:10827000CBE04146204603223AF0A4F9013504340C
:1082800008F10408AF42F4D11BE747493046F9F73B
:108290008FFF0546002840F0AC80384F334997F8EF
:1082A000608702AA62F024FD00283FF40AAFFAF7C3
:1082B00095F8461E01D4B04503DC3C4943460122F3
:1082C00013E72A4902AA002062F012FD01460028A5
:1082D0003FF4F7AE4FF00008082203A8CDE9038869
:1082E0008DF8148062F082FD0DF10C0903A860F096
:1082F000DFF840451CD81D4902AA002062F0F8FCB6
:1083000000283FF4DEAE90F800A097F86197DFF800
:10831000ACB04FF000084D45144902AA4FF00000E0
:108320007EDA62F0E5FC024658B921494A466CE023
:1083300099F80000F9F736FF08F1010809F8010B78
:10834000D4E7002D40D11378303B092B3CD9194993
:108350000192F9F72DFF019A90B310465946F9F7AB
:1083600027FF019A002838D013494EE0B19F080832
:10837000E09C002058A008085EA008088095002016
:1083800069A0080872A0080880A008088CA0080846
:108390009EA008088DA10808CC9D0020C8A0080850
:1083A000ADA10808D4A00808F2A00808F7A00808A2
:1083B000CDA10808469008080AA1080803A10808EA
:1083C0004FF001084FF0FF3510460192FAF706F81A
:1083D0000028019A03DA214917E0A846F2E70EAB1C
:1083E00003EB4503013523F8200C94E71C494A466A
:1083F0000BE01C49324608E01B49002062F078FC83
:1084000000283FF4F9AE19493A462046FCF70FFA26
:1084100057E662F06DFC00287FF428AF144C31E77A
:1084200062F066FC0028E1D1124C06EBC6008230F7
:10843000082203A920443AF0C5F85046F9F7B2FEE5
:1084400037446A0087F82A0804EB061006A90230B0
:1084500062F018FC87F8428833E600BF3FA10808A5
:1084600054A1080877A10808B19F0808AAA0080825
:10847000DC9D0020E09C00202DE9F04F89B00F46E4
:1084800091460021139A98460646FCF7A5FF87EA15
:1084900009096FEA0903DFF8849006930446002572
:1084A00028460FF0FDF8129B184230D0069BDFF8EB
:1084B00070B0034014BF4FF0010A4FF0000A04935C
:1084C00010EA070314BF4A465A4628460593079206
:1084D0000FF0F8F8079A0390009043465146304653
:1084E000FBF75CFB049BB3FA83F122464909304653
:1084F000FCF772FF059A039B009304464346002A4B
:1085000014BF5A464A4651463046FBF701FB013537
:10851000182DC5D109B0BDE8F08F00BFDC9E08085A
:10852000F2A1080837B50446084601915FF0C0FF84
:108530000199054602462046F9F75EFE70B9625D74
:108540001046F9F71FFE00B932B901352C44204618
:1085500001340378202BFAD003B030BD0020FBE7B4
:10856000F0B5032985B005460C46164614D80B4FC6
:108570003970FBF7C9FA0A492846FDF74BFD09494E
:10858000224601A8F9F700FD01AB32460821284632
:10859000FCF750FFFF233B7005B0F0BDB006002094
:1085A000229C0808D89D0808F0B5032985B0054627
:1085B0000C46164614D80B4F7970FBF7A5FA0A49FA
:1085C0002846FDF757FD094922466846F9F7DCFCC5
:1085D0006B46324610212846FCF72CFFFF237B70A8
:1085E00005B0F0BDB0060020229C0808D49D080804
:1085F00030B587B0134B0493134B0393134B144CB8
:108600000293144B0193144B144A154900930546E9
:1086100004F10B031348FBF7D9FAFBF775FA75B1B0
:10862000237E63B194F820304BB10F4804F120024F
:1086300004F1180107B0BDE83040FBF77DBB07B07F
:1086400030BD00BF39A208083EA2080846A20808AB
:10865000809500204FA208085BA20808F9A108082D
:1086600003A208080EA2080861A20808224BB0F570
:10867000FA6F1A680346A8BF4FF4FA63B3F57A7F1E
:10868000B8BF4FF47A73D20416D540F2DC52904250
:1086900015D007EE903A40F2DB529042F8EE677A3E
:1086A0001FD8DFED166A9FED167A9FED160A77EE5A
:1086B000E67AA7EE870A7047B0F57A7F02D89FED79
:1086C000120A704707EE903ADFED106A9FED107ABC
:1086D0009FED100AF8EE677A77EEE67AA7EE870A42
:1086E0007047DFED0D6A9FED0D7A9FED0D0A77EE75
:1086F000E67AA7EE870A70473C9B002000007A4488
:10870000D62000C000E082440000000000407A440F
:10871000661000400000404200A0BB44D62000404C
:108720000000834410B584464FEA810E102312F4F2
:10873000004F14BF0E2407245200013BCCF8004028
:1087400092B2F444F3D100EB81128C01035142F850
:108750002130122010BD00BF10B584464FEA810EB3
:108760000424130B03EB430318331201013CCCF830
:10877000003092B2F444F4D100EB01130A018450AA
:1087800043F82140062010BD704700BF704700BF6E
:10879000034B00EB400003EBC000407C704700BF80
:1087A000480500102DE9FF471E46C368BDF830702C
:1087B000DDF8348004468946924643B3CBB20D2B94
:1087C0009ABF1A4AD5560025BAF1FF3F21D0236837
:1087D000174A3146CDE9005A3846C04752462079FB
:1087E0005FFA89F1F2F780FB024600B10288D3B24A
:1087F0000393C2F30323120BCDE9005202930D4AF7
:10880000236831463846C04704B0BDE8F0874D1CA8
:10881000DAE77B06F8D42368074A0C9531463846D8
:10882000C44604B0BDE8F047604700BFA44A08084A
:108830008EA208089BA20808BFA2080800230370A4
:1088400043708370C3707047704700BF002070474B
:10885000704700BF0020704701207047704700BF7D
:10886000704700BF704700BF704700BF9FED010A0F
:10887000704700BF000000000020704703681B69BC
:10888000184730B5084B002293F900405D78011974
:108890000132CD729D780555062ADC788C7503F17E
:1088A0000403F1D130BD00BF88060808002383709F
:1088B0000370C37043707047C36B33B15B68426D24
:1088C0009BB29A4205D3D01A7047D0E907239A4247
:1088D000F9D2C0681044C01A704700BFD0E909122D
:1088E0000369914238BFC9188A1A016C39B14968C5
:1088F000013B12FA81F2934204D9981A7047013B66
:10890000981A704700207047036C13B190F8640008
:108910007047D0E90903181AB0FA80F0400970478F
:10892000C26B10B4034662B1426DC1685C69881ABB
:10893000013A205C5DF8044B08BF0A46C0B25A6594
:108940007047006A5C69411C205CDC68A14238BF4A
:108950000A46C0B25DF8044B1A627047836E70B568
:1089600004460D460BB19847B8B1636AA269D55465
:10897000636A2169226C01338B4228BF0023636242
:1089800032B3EFF31183502282F31288226C116804
:10899000C90703D5DBB283F3118870BD516889B272
:1089A00071B9D4E90950854218D0A6690644D66049
:1089B00018D9281A80B25060A562002184F864108A
:1089C000116841F00101DBB2116083F3118870BDC1
:1089D000226ED36843F08003D36070BD012284F817
:1089E0006420D7E72569281A80B25060A162E4E7C5
:1089F000836E03B118477047F8B590F87C30012BAF
:108A00001CD0002A164619DD0269436A05460F4646
:108A1000D41AB442A869A8BF34463946184422463D
:108A200062F030F96B6A2A692344361BB3FBF2F01B
:108A3000002E02FB10336B622744E9DCF8BD00BF57
:108A400090F87C30012B0DD0036C43B3EFF311830E
:108A5000502282F31288026C1168C90703D5DBB279
:108A600083F311887047516889B270B471B9D0E945
:108A70000954A54219D086692644D6601CD92C1BFE
:108A8000A4B254608562002180F86410116841F03E
:108A90000101DBB2116083F3118870BC7047026E74
:108AA000D36843F08003D3607047012280F86420CC
:108AB000DBB283F31188F0E705692C1BA4B2546084
:108AC0008162E0E70849002301E0152B09D003EBA0
:108AD0004302013311F802C084450A44F5D110461F
:108AE00070470020704700BFF429002010B311B375
:108AF00010B5124C4FF0100C22464FF0010E00231F
:108B000004E001334E2B0ED092F804C0604502F110
:108B10001C02F6D1714508D001330EF1010E4E2B27
:108B20005FFA8EFEF0D1002010BDC3EBC30304EB4F
:108B3000830010BD70470846704700BFBCB60708E9
:108B40002DE9F04188B01E4603090E9F9046403340
:108B500000F00F0451B30793FFF7C8FFC279079BDA
:108B6000CDE900420546164A41463046B847D0B1E5
:108B70002868F2F7DDFBA9796A79DFF854C0ED794E
:108B8000079B009411F0020F4FEA92020D4902F187
:108B9000010208BF6146CDE90102CDE903150A4A89
:108BA00000213046B84708B0BDE8F081074A0E946E
:108BB00041463046BC4608B0BDE8F041604700BFC2
:108BC000CEA20808F5910808E0A2080802A3080848
:108BD000229C08082DE9F047DFF85CA0BAF80030C5
:108BE000043388469EB201F10909012518F8014BAA
:108BF000B4460021ACF1040305FA01F29BB2224015
:108C0000C2B1878900EB830E01339BB29C45CEF83D
:108C10001470F5D101310CF1040C08291FFA8CFCF9
:108C2000E8D12036C845B6B2E0D10023AAF800301A
:108C3000BDE8F0871746E5E700E500202DE9F04F95
:108C4000DFF89490B9F802300B330F4601F10608B3
:108C50001FFA83FB0125002117F801EB5A464FF05C
:108C6000000C0126A2F10B039BB206E001339BB27C
:108C70008489CAF8144093420BD000EB830A002E7B
:108C8000F4D100EB830A01339BB29342CAF814601B
:108C9000F3D1043300EB8303BCF1090F596010D00A
:108CA000BCF1080F0BD005FA0CF313EA0E0F14BF3A
:108CB000012600260C320CF1010C92B2D2E70026FC
:108CC000F8E70BF1780447451FFA84FBC4D1A9F8F3
:108CD0000210BDE8F08F00BF00E500202DE9F04153
:108CE000057B0E780446C0E90555C0E90755C0E983
:108CF0000955C0E90B55C0E90D55F643282200215E
:108D00003C3062F022F8F6B24FF0140C4FF0050E32
:108D10004FF0000846FA0EF303F00103002B14BFD6
:108D200019270A2743441EF001000CEB07015FFAE4
:108D300083F818BF284689B2634604EB83020133E7
:108D40009BB299425061F8D10EF1FF3EBC44BEF196
:108D5000FF3F1FFA8CFCDDD118F0010F14BF192062
:108D60000A200CEB000189B2634604EB8302013355
:108D70009BB28B425561F8D10CEB00039BB21A1DDC
:108D80000549013304EB82029BB2002050608B80C6
:108D90002361BDE8F08100BF00E5002070B5094CFB
:108DA000A36873B10546002606E099681A681E7329
:108DB000A1609047A36823B15A68AA1A002A1846EE
:108DC000F3DA70BD00E50020914B1B68D90600D492
:108DD0007047F0B58F4C2DED028BE36987B013B16E
:108DE00004F10C009847236A002B70D08A4894ED58
:108DF000188A9847C21C054675D0002877DA431CAC
:108E000000F0F9806FF00102A262844E3368EB1A21
:108E100003FB03F34FF609218B42DCBF8049A1FB22
:108E2000031394F87D1004EB4100D4BF43F3CF0348
:108E30004FF4C853A0F880304B1CDBB2052B84F8EC
:108E40007D3000F0888094F88A303560002B00F087
:108E50008E80B4F88200B4F88030B4F8841094F8AE
:108E600034600344B4F886000B44B4F8881003441B
:108E70000B441BB2B3F5FA4F1946A8BF4FF4FA41A1
:108E800021EAE171A1873EB9002A05DDB3F5167F1D
:108E900078DB012684F83460624B18781B2844D0B4
:108EA0001C2837D1E76A604DA36B2A80002F6E80A3
:108EB000AB802DDD002A2BDDB1F5167F28DA002EE0
:108EC00000F0A1809342D4BF0023012321E0554943
:108ED0004FF0FF330878A3621A461B28E36202D1E1
:108EE000514D6A80AB8007B0BDEC028BF0BD636E64
:108EF0004E4904EB8302013309682163052B906618
:108F000063664DD094F87C30002B4ED102467BE74F
:108F10000023EB80D4ED097AB4EEE78AF1EE10FA83
:108F20000CD54FF0FF33E362DDE7D4ED097A3E4D17
:108F3000B4EEE78AF1EE10FAE98014D4002A64DB7B
:108F400007EE902AF8EEE77A67EE887AFDEEE77A88
:108F500017EE903AC1E7002384F87D30012384F8AE
:108F60008A30356075E74FF0FF33E362B9E794F874
:108F700034604FF6FF73A3874FF0FF31002E8BD183
:108F8000002A89DDA36B93423BDA294802EB820376
:108F9000C3EB0313A0FB03035B09A36300267BE77A
:108FA00000220123626684F87C30224F0FCF01AE8D
:108FB0000FC6029A3B683360904202DC13460246B9
:108FC0001846DDE90413994202DC1E460B46314681
:108FD0008142A8BF01469A42B8BF1A46039B8B4202
:108FE00002DB0846194603468A42A8BF0A469A424F
:108FF000B8BF1A4608E70D4BA0621B682363024600
:1090000003E7002648E7012383E74FF0FF3364E7D7
:109010009CA6002000E500200CE500201807002099
:10902000CDCCCCCCC4280020C82800206427002048
:109030001F85EB5168E500200120FFF7D9BA38B54C
:109040000B4B03EBC0050C4695F88821094803EB50
:1090500082039969FAF7BAFD95F88E3133B1611C34
:109060000548BDE83840C9B2FAF7B0BD38BD00BF09
:1090700088060808C6A5080878DC080813B52B4838
:10908000FAF722FD2A4B93F82130002B4CD0294CC3
:109090002948FAF751FD94F894302BB194F89630A2
:1090A00013B194F8953073B994ED280A23488DEDE7
:1090B000010AFAF709FD224B9DED010A1B8833BB1B
:1090C0002048FAF739FDB4F898101F48FAF77EFDEA
:1090D00094F8943013B31D48FAF72EFDB4F89C10A1
:1090E0001B48FAF773FD94F89630CBB11748FAF79E
:1090F00023FDB4F89A101748FAF768FD94F89530F4
:1091000083B1124802B0BDE81040FAF715BD61F016
:1091100041F881B21048FAF70FFED4E70F48DBE7B9
:109120000E48E4E70D48EDE70D48EBE714A3080807
:10913000D0990020701500102AA3080831A3080850
:10914000E0AE00204BA308085AA308087AA3080839
:109150008AA30808A4A3080855A3080883A308083D
:109160004FDD080808B5254B1B68DB040AD5B5EEB2
:10917000400AF1EE10FA12D19FED210A61F00AF8CF
:1091800080B208BDDFED1F7AB4EEE70AF1EE10FA07
:109190001CDA9FED1D0A60F0FDFF80B208BDDFED17
:1091A000197AB4EEE70AF1EE10FAE5D49FED177ADA
:1091B000B4EEC70AF1EE10FA14D870EE677A9FED9C
:1091C000147A9FED140AA7EE870AE4E770EE677A37
:1091D0009FED117A9FED110AA7EE870A60F0DAFF82
:1091E00080B208BDDFED0E7A9FED0E7A70EE677AE1
:1091F0009FED0D0AA7EE870ACDE700BF3C9B00203C
:109200000080BB440000404200007A4400E08244F9
:1092100066BEFFBE0060BB4438DFFF3E00407A44BC
:109220000000834466BEFF3E00A0BB44F8B5C64BB9
:109230001D6815F004072DED048B40F00081DFED73
:10924000C38AC34C15F0200505D094F8585115F089
:10925000020540F0908094F890319FEDBE8A13F0A3
:10926000010340F0AC8094F89121002A7ED1D4ED26
:10927000657A9FEDB97ADFEDB96A67EE877A94ED8A
:10928000677AE8EEA67A38EEC77AC4ED657A84ED9F
:10929000667A65B194F8A421D4F85C31C4F8A031A1
:1092A00001218A4284F8921118BFC4F89831AC4B5E
:1092B0001E780E2E00F00781DFEDA47A002794EDD2
:1092C0006D7A94ED6E6A77EEC76AD4ED6C7AA6EE8D
:1092D000267A77EE676A84ED6D7AE6EE267AC4ED3B
:1092E0006C7AC4ED6B7A0FB1C4ED667AD4ED6F6A17
:1092F00094ED717A9FED9B5A94ED726AC4ED6F7A8A
:1093000077EEE66AF0EE475AD6EE855AF0EE477AE7
:10931000E6EE257A94ED700AC4ED717A37EEC07AE4
:10932000A6EE070A84ED700A60F034FF02B282EA0A
:10933000E273A3EBE2739BB2092B7ED9002AACBF88
:109340000A380A3005B20E2EA4F8CC5160D0242E73
:1093500009D1DFED857A94ED660A20EE270A60F0E8
:1093600019FF824B5880BDEC048BF8BD84F8923114
:1093700084F891317BE7D4ED5A7AB4F86C31F8EE89
:10938000E77AC4ED577A002B00F08A8007EE903A16
:10939000DFED746A9FED767AF8EEE77A86EEA78ABB
:1093A000B4EEC78AF1EE10FA88BFB0EE478A94F89F
:1093B000903113F001034FF001053FF454AF94F8DE
:1093C0009131002B56D094ED679A78EEC99A002D12
:1093D0003AD094F89231002B54D0D4ED577A94EDD2
:1093E000680A5F4B1E7877EEC07A0E2EC4ED6B7A5A
:1093F0005FD094F8A431002B75D0022B02D00FB1AE
:10940000012B31D0D4ED6B7AF0EE698A012756E753
:10941000DFED547A554C9FED540A28EE278A28EE4A
:10942000800ABDEEC88A18EE103A238060F0B2FEC2
:10943000BDEC048B6080E580F8BD002583E7444CDB
:109440000127D4ED538AFDE6454B1E780E2E2AD017
:1094500094F892519FED3D8A002DCAD1002FD1D0B2
:1094600094F8A431002BCBD1F0EE697A0127F0EE0D
:10947000698A24E794ED659A012384ED679A84F85C
:109480009131A2E7002F56D0D4ED577A37EEE80A93
:10949000012330EE090A84F8923184ED680AA0E7CE
:1094A0009FED2C8A83E7D4ED6B7A94F892519FED6F
:1094B000278A9FED2D0A27EE800A60F06BFE2B4B6A
:1094C0000E269880C8E7DFED2B7A94ED577A274B6C
:1094D00027EE277A0027BDEEC77ADFED1C7A17EE5C
:1094E000102A9A80EBE6002F8CD094ED6B6A94F8EA
:1094F000A531DFED216A07EE903A76EE688AB8EE84
:10950000E77A78EE897AF0EE698AF0EEE77A67EE2C
:10951000877AF4EEE67AF1EE10FAC4BF68EE266AB6
:1095200086EEA78AF7EE007A77EEC87A67EEA97A18
:10953000E6EE087AC3E60A4B1E780E2E7FF462AF81
:10954000D4ED6B7A3D46B4E79CA6002000000000F5
:1095500000E500209A99993ECDCC4C3FCDCC4C3EB5
:10956000C42800200000C842CDCCCC3DC828002033
:109570006666663F0AD7233C00401C462DE9F04F43
:109580000A4687B000210646FBF726FF3B4C0590B4
:109590003B4A2378608802EB8303D3F818A0F7F7DF
:1095A000E7FF83680493374BC1681A78002A4BD0D1
:1095B000DDF810800491002721796279049B07FB74
:1095C000012213F80290B8F1000F3FD018F80250B2
:1095D000059A4D4514BF0121002130460CBF4FF0C4
:1095E000010B4FF0000BFBF7F7FE013705907DB341
:1095F00005F00F022D0940350292CDE90075224A8F
:10960000534659463046FAF7C9FAB9F1000F2AD045
:1096100009F00F024FEA1919029209F14002CDE94F
:1096200000725346184A59463046FAF771FAA27941
:10963000012A38BF0122BA42BEDC144B0834A342CF
:10964000A6D107B0BDE8F08F9046B4E74546BFE726
:10965000B8F1000FD9D00E4A00975346594630460C
:10966000FAF79CFAD1E77306E1D4094A009753460A
:1096700059463046FAF74CFAD9E700BF10080808F7
:109680008806080820960020C4A30808C80908080E
:10969000DAA308080246531C084605D1044B1A6891
:1096A0001B790A600B7170470249F8F76DBC00BF67
:1096B000C9A2080879DC080810B501311446FFF783
:1096C00015FA28B9064B1A681B792260237110BD60
:1096D000C27904492046BDE81040F8F755BC00BFE8
:1096E000C9A20808DBA208082DE9F041154686B09A
:1096F0006A1C8846BDF830600D9F194623D00309C7
:1097000000F00F044033CDE90045164A059330467A
:10971000B847A8B198F80510D8F800002A46F1F724
:109720002BFC68B1028801780391C2F30321120B6C
:10973000CDE900420291059B0B4A00213046B84713
:1097400006B0BDE8F0817306FAD40309074A00F0B9
:109750000F000C9040333046BC4606B0BDE8F041E7
:10976000604700BFEEA3080800A4080829A4080861
:109770002DE9F04F2DED028B0A468BB00021824679
:10978000FBF72AFE6D4D814605F1800B00266C4BE0
:109790001C78AB7AB34200F393801035AB45F5D11A
:1097A00040F21620F7F7E4FED0E902530CB12C4644
:1097B0001D460DF1100B15220021584661F0C5FA27
:1097C00000272E78002E42D069783046FFF78EF9B8
:1097D00095F9023002935A1C534208EE100A534185
:1097E000002C00F0A880002214F802C0B44504EB5D
:1097F000020040F09C8090F90280029A424540F0BD
:10980000948042788A4208BF012301220BF8072086
:1098100003F001034A4683F0010150460393FBF72E
:10982000DBFD039B81464CB1464A18EE101ACDE988
:1098300000A230464246FFF757FF039B424A18EE0C
:10984000101ACDE900A23046029AFFF74DFF01370A
:10985000152F05F10305B4D16CB33A4FDFF8E8805A
:1098600004F13F061BF8013B02930BBB2078F8B1D3
:1098700094F9022001321BD06178FFF737F94A468C
:10988000054601215046FBF7A7FD94F90220029BF3
:10989000294681462078CDE900A7FFF725FF2078EB
:1098A000029BCDE900A84FF0FF322946FFF71CFFCD
:1098B0000334B442D6D10BB0BDEC028BBDE8F08FBF
:1098C000E888F7F755FED0E902230CB114461A4692
:1098D000297A6B7A06FB013312F9038014B3E75639
:1098E000B8450CBF012300234A4614BF01210021C3
:1098F00050460293FBF770FD029B814644B1114A2A
:109900003146CDE900A228463A46FEF74BFF029BBE
:109910000D4A3146CDE900A228464246FEF742FFF5
:10992000013634E74FF0FF37DAE700236DE7033203
:109930003F2A7FF459AF4FF0FF386BE71C07002038
:10994000209600209D3B0108113B01082DE9F04FB6
:109950006E4B1B7887B0002B00F0D1806C4D6D48AA
:10996000A968DFF8F4A1FAF7E7F969686A48FAF735
:10997000E3F96A4B6A48D3E90031C91A694BD3F855
:10998000D021B1FBF2F2FAF7D7F9FAF7BDF8664841
:10999000FAF7D2F86548FAF7CFF84FF00008644BB1
:1099A0001B785FFA88F4A34222D8624C624FFAF720
:1099B000ABF82646002556F8041B38460135FAF761
:1099C00005F9162DF7D1FAF79FF85B4E01252346CE
:1099D00061681B683046C91A0135FAF7F7F8162D89
:1099E00004F10404F3D107B0BDE8F04FFAF78CB8E6
:1099F000524B142603EB840306FB045693ED2D0A09
:109A0000B6F80E9060F0C6FB96F81EE01EF0010F4F
:109A100014BF52222D221EF0020F14BF54232D23F7
:109A20001EF0040F07EE903A14BF56232D231EF0AC
:109A3000080F14BF4FF0430C4FF02D0C81B21EF0F5
:109A4000800F4FF03C0BB1FBFBF105914FF064012F
:109A500014BF4FF0530E4FF02D0E80B201FB09F1F1
:109A6000671CCDE902E10093049017EE903ACDF81F
:109A700004C039465046FAF7A9F8B37FDB073AD558
